:020000040800F2
:10000000F8FF01209D92090845170908ED7A0408B8
:10001000491709084D170908511709080000000081
:100020000000000000000000000000005517090853
:1000300059170908000000005D170908B95E040897
:10004000299309082993090829930908299309087C
:100050002993090829930908BD250408C525040822
:10006000CD250408D5250408DD2504086900000015
:10007000790000008900000099000000AD00000038
:10008000C1000000D500000029930908000000000D
:10009000000000000000000000000000E52504084A
:1000A000299309082993090829930908F14E04089E
:1000B000014F0408114F0408214F0408C917040810
:1000C000C1170408D9170408D1170408299309088F
:1000D00029930908A1BD0000B1BE0000E9BF0000DE
:1000E000ED25040829930908000000002993090858
:1000F0002993090829930908AD4F0408E900000075
:100100002993090871380408314F04082993090814
:1001100021C1000059C2000029930908414F040879
:10012000FD00000011010000250100003901000060
:100130004D010000299309082993090800000000D7
:1001400000000000000000000000000000000000AF
:1001500061010000750100008901000091C30000E9
:10016000E9170408E11704082993090829930908E5
:10017000FD1F09086517090829930908299309082B
:100180002993090861170908C9C4000001C60000C5
:10019000299309082993090829930908299309082B
:1001A000299309082993090829930908299309081B
:1001B000299309080000000000000000F917040856
:1001C000F11704082993090800000000000000004E
:1001D0000000000000000000299309080000000052
:1001E000000000000000000000000000000000000F
:1001F0000000000000000000299309082993090865
:100200002993090829930908299309080000000087
:100210002993090829930908299309080000000077
:100220002993090800000000299309080000000034
:10023000953904082993090800000000299309084A
:1002400000000000000000000000000000000000AE
:10025000000000000000000000000000000000009E
:1002600000000000299309080000000000000000C1
:10027000000000000000000000000000000000007E
:1002800029930908299309080000000000000000D4
:1002900000000000000000002993090829930908C4
:1002A00029930908299309082993090800000000E7
:1002B000000000000000000000000000000000003E
:1002C00000000000299309082993090829930908C7
:1002D00029930908299309082993090829930908EA
:1002E00029930908299309082993090829930908DA
:1002F00029930908299309082993090829930908CA
:100300002993090829930908000000002993090886
:1003100029930908299309082993090829930908A9
:100320002993090829930908299309082993090899
:100330002993090829930908299309082993090889
:100340002993090829930908299309082993090879
:100350002993090829930908299309082993090869
:100360002993090829930908299309082993090859
:100370002993090829930908299309082993090849
:100380002993090829930908299309082993090839
:100390002993090829930908299309082993090829
:0403A000299309088C
:020000040804EE
:10000000084A0346D0F8E4005268D3F8F010121AF8
:1000100000209142B8BFC3F8F020012283F81C21D0
:10002000704700BF001000E02C2370B400FB03F306
:10003000754DEA582B445268946902F1180C116806
:100040008E0601D5A60667D4CB0601D5E6067AD47E
:100050004E0628D5630626D52C2303FB0053997F33
:10006000F9B105EB800090F8B110D1B190F8B31060
:100070000129CDB215D1116821F0F60111600021DE
:1000800080F8B010022180F8B310997E187F1C7F91
:10009000C9B2C0B204F0FF06002C40F09D801D766E
:1000A0005E7670BC70474E071DD48E07F9D5A10748
:1000B000F7D52C2101FB00514B7F002B5ED18B7FAC
:1000C000002BEED005EB800393F8B1000028E8D1B7
:1000D000C97E0120C9B2916283F8B100136823F090
:1000E00002031360DDE76307DFD505EB80012C23F6
:1000F000546A03FB005391F8B020187F52B2824239
:10010000CFDA91F8B020E4B2586A53B25A1C52B216
:1001100081F8B020C454C4E72021D161E10603D5A1
:100120001021D161012119761368002105EB8004AB
:1001300023F0F60313602C2384F8B31003FB005361
:1001400070BC5976704710212C23D161012103FB2B
:1001500000531976116821F0D60111609169890662
:100160009FD52021002405EB8000D161116821F08A
:10017000F601116080F8B3405C7692E705EB8003EE
:10018000840093F8B060FF2E36D093F8B030097F2A
:100190005BB28B420BDB2C442C2194F8B03001FB7A
:1001A00000515BB2097F8B42FFF67BAF96E7DCF82C
:1001B00000309B07FBD52C2305EB040C03FB0053FD
:1001C0001E6A9CF8B0305BB2591C49B28CF8B01072
:1001D000F35CDBB29362DEE7BFF34F8F0B4B41EA78
:1001E00000410B435360BFF34F8FBFF36F8F136812
:1001F00043F0B403136054E7C97EC9B29162002191
:1002000083F8B010C7E700BF802800240024000254
:10021000D0E9001300221A60037A032B10D84FEAAA
:10022000530C06203D224FEA8C0C10FB03C310B484
:1002300002FA03F38C6823435DF8044B8B6070472C
:10024000043BC868DAB2C3F3400302EB4202520037
:1002500002EB83023D2393400343CB60704700BF12
:1002600030B41B4B1B4D1C4CA84298BF2346C01AF0
:100270000B6070281FD00BD8402824D0582816D0E7
:10028000A0F12800B0FA80F0400930BC106070473F
:10029000A02814D0B82806D088280CBF052000203C
:1002A00030BC10607047072030BC106070470320DE
:1002B00030BC10607047042030BC106070470620CE
:1002C00030BC10607047022030BC1060704700BF27
:1002D00000040240FF030240000002401F4A204B7E
:1002E000904202F1010210B41E4C98BF2346A4F1C3
:1002F000140498BF2246801A702820D00AD84028BB
:1003000027D0582816D0282800D118335DF8044B80
:1003100019607047A02817D0B82806D08828F5D1D2
:1003200078335DF8044B19607047A8335DF8044BCF
:100330001960704748335DF8044B196070476033AB
:100340005DF8044B1960704790335DF8044B1960F9
:10035000704730335DF8044B19607047FF0302406B
:100360001404024014000240002A4FEA014C0346E4
:1003700030B508BFE64600F1C00514BF8E468C4676
:10038000002419680C3353F8042C43F8084C41EA54
:100390000C0142EA0E02AB4243F80C1C43F8042C59
:1003A000EFD1D0F8C03043EA0E03C0E93144C0F8C1
:1003B000C03030BD10B40C4C2368002B11DD002080
:1003C00004F1040C0146DCF8B03003F1C0025960BE
:1003D0000C339342FBD1013023680CF5887C8342B7
:1003E000F1DC5DF8044B704704000020F0B5414C8F
:1003F00004EB401393F8603403B9F0BD3E4B420167
:1004000093F8C05093F8C1C065450CD00CEB4C0E6E
:1004100003EBCE0E9EF8C4604FEA4C0E771E012F00
:100420005BD9032E53D02244A2F84414EFF3118178
:10043000902383F3128892F84634C9B2B2F8440488
:1004400043EA400300209BB282F8460481F31188FE
:10045000190994F8440581EA13215940D8B1C943D8
:100460001B01D2F85C540124D2F848049BB201F07D
:100470000F01D5F8B02084400B4302F1C0005900B1
:1004800013F4004F8BB202D15168214351600C32FA
:100490009042F4D1F0BDD2F848041B01D2F85C249C
:1004A00001F00F0110309BB20124D2F8B0200B43B1
:1004B000844002F1C000590013F4004F8BB202D106
:1004C0005168214351600C329042F4D1F0BD0CF1DF
:1004D000010606F00306AE42A5D0E64403EBCE03C8
:1004E000034493F8D11000299DD0A318012083F86C
:1004F000460498E70400002080280024704700BFCD
:10050000024B03EB401393F8610470470400002092
:1005100010B582B00C466A4601A9FFF7A1FE21681A
:10052000DDE9002302EB420203EBC20319616268BA
:100530005A61A2689A61E268DA6122695A6202B07D
:1005400010BD00BF184B194A10B4194CA04298BFF7
:100550001346C01A702820D013D8402821D058281C
:1005600019D0282800D118331A695DF8044B0A60A5
:100570005A694A609A698A60DA69CA605B6A0B6183
:100580007047A0280BD0B82803D08828ECD1783346
:10059000EAE7A833E8E74833E6E76033E4E7903377
:1005A000E2E73033E0E700BF000402400000024011
:1005B000FF03024038B5026D044643689A61EFF3C9
:1005C0001182502383F312884168D2B2656C0B68A4
:1005D000C06C23EA050303430B6082F3118804F126
:1005E0001C012069FFF794FFA268B4F87010002383
:1005F0001268D162237638BD30B540F2FF5405460B
:100600008463C06820F48050E86041F48050AA60A0
:10061000E8607ABB73BB4FF0FF334FF0800E4C4A5B
:1006200010684FF4081200F1340C00E02AB3DCF833
:100630000040013A14EA0E0FF8D0002B29DD446B7C
:10064000640721D4032B24D0426BD20725D4022B7C
:1006500021D00269C9B2D2B2914223D1012B4269A1
:1006600022D0062B17D112F4604F49D1394BC3F871
:10067000242110E04FF0450ED1E7002B04DD426B42
:10068000520701D4032BDFD1032040F2FF53AB63A9
:1006900030BD002AF8D00020F7E740F2FF530120D8
:1006A000AB6330BD1020F0E72B4B1340002BF2D092
:1006B000002A39DB53002BD494002FD4D0002BD444
:1006C00011012FD453012BD4D40133D410021DD4E3
:1006D0005102E7D4930231D4D4022DD4100319D49B
:1006E000510323D4930331D4D4032DD4100429D43B
:1006F000510425D493041BD41407CCD51A20C4E785
:10070000900407D45104CDD41304C4D50F20BCE702
:100710000920BAE71320B8E70B20B6E70A20B4E7B0
:100720000D20B2E70C20B0E71C20AEE71420ACE7A8
:100730001920AAE70E20A8E71220A6E71120A4E7B7
:100740001820A2E71720A0E716209EE715209CE7B7
:10075000A40300248028002408E0FFFDF0B5454DE7
:1007600083B095F82831022B70D8434E37687B69E7
:1007700013F0007302D00E2003B0F0BD04460093C6
:10078000082201234FF488713846FFF735FF00280F
:10079000F2D10123D5F8242140F237113846FFF772
:1007A0002BFF0028E8D1354B024640F23311384682
:1007B0007B620823BB62FB6A43F03303FB620123C5
:1007C000FFF71AFF0028D7D13668684640F22A5151
:1007D00006F1340302E01A6812033CD51A680A4293
:1007E000F9D0736B18073ED4736B99073DD4736BC4
:1007F0009B063CD4B4F5804F009B18BF4FF4803269
:100800001BBA08BF4FF480221A4222D00123D5F828
:10081000242140F237113046FFF7EEFE0028ABD11D
:10082000A4F5804201234FF483713046B2FA82F27C
:1008300052099A40FFF7E0FE00289DD1736823F427
:100840004043736073682343736095E7282003B0C7
:10085000F0BD262090E71A689704BFD5D6F880200F
:1008600040F8042BBAE7042086E7022084E706203C
:1008700082E700BF80280024A403002400E1F505DE
:100880000B4890F8481589B101EB4101002300F2B3
:100890004C50490010B41C4650F82320063302B1D6
:1008A00014608B42F8D15DF8044B7047704700BF6D
:1008B000040000200B4890F8481589B101EB410174
:1008C000002300F24C50490010B41C4650F823207D
:1008D000063302B114608B42F8D15DF8044B7047C7
:1008E000704700BF0400002000EE100AB8EE400A76
:1008F000704700BFBCEEC00A10EE103A98B27047C5
:10090000D0E90920131A58425841704790F84F38DF
:1009100030B53BB990F84D18012490F84E38DAB252
:10092000914200D830BD04FA03F2B0F856580133B2
:100930002A43A0F85628F2E70379024613F0010093
:1009400006D0D2E90731D2685B1A013A03EA020005
:10095000704710B50379044613F001030ED0FFF77A
:10096000EBFF034650B1226A6369E1689B5C013288
:10097000B2FBF1F0DBB201FB10222262184610BD7F
:1009800003799B070AD5436A8269D154436A026995
:100990000133B3FBF2F102FB11334362704770473E
:1009A000017170470379014613F0020007D00B690B
:1009B000D1E90921013B521A1A40D2B2981A704764
:1009C000072808D8044B03EB401393F8602412B1B6
:1009D000012283F84624704704000020072808D825
:1009E000054B03EB4013B3F84404B0FA80F0400920
:1009F00070470020704700BF04000020054B93F8AB
:100A00000C26824204D903EB4013D3F850047047FC
:100A10000020704704000020704700BF704700BFEF
:100A200000EB4000024B03EBC00393F85D057047F9
:100A300004000020064B93F80C26824206D900EBF6
:100A4000400003EBC003D3F86005704700207047F7
:100A500004000020072808D8054B03EBC013B3F8A7
:100A60001006B0FA80F0400970470020704700BFC0
:100A700004000020072805D8034B012203EBC01314
:100A800083F81226704700BF04000020F8B54FF02D
:100A9000B0431D685A69154005405D617DB1084F3E
:100AA0000126B5FA85F4C4F11F0407EB840306FAA6
:100AB00004F4D3F82C0103689847A543F1D1F8BD9D
:100AC000802800240269C3682DE9F04712EA03096F
:100AD0002AD006460D4600F110074FF00048B9FA3B
:100AE00089F328FA03F21B3BD24309EA02093A6070
:100AF000042B16D8DFE803F04134271A0300AB6A51
:100B0000002B47D003F1FF3A00231FFA8AFAAB62A9
:100B10006C6A34B123682046514698476468002CBB
:100B2000F8D1B9F1000FDAD1BDE8F0876868002884
:100B3000F7D00368002BF4D0716B89B29847B9F1F4
:100B4000000FCCD1F0E7A8680028EAD00368002B9A
:100B5000E7D0B16B89B29847B9F1000FBFD1E3E795
:100B6000E8680028DDD00368002BDAD0F16B89B289
:100B70009847B9F1000FB2D1D6E728690028D0D044
:100B80000368002BCDD0316C89B29847B9F1000FC2
:100B9000A5D1C9E7F36A1FFA83FAB9E770B505462C
:100BA0000B260A4C013E00D170BD94F9000017F0ED
:100BB00027F9031E08DB6178EA18072B9172A178E8
:100BC000E95401DCE37813750434EBE768BB0908EA
:100BD000F8B52C232D4E054600FB03F3F2583344A1
:100BE0005468A269606812F4F85F41D00127211DA2
:100BF0001F7612F40077236823F0F603236002F4D3
:100C0000807318BF43F4007312F4806F18BF43F46D
:100C1000806312F4006F18BF43F40063D20448BF2E
:100C200043F48053E361AFB9830422D542F21073D9
:100C300001E0013B02D00A689704FAD4636843F4E8
:100C40008043636042F2107301E0013B19D00A68EF
:100C50005004FAD4A3699B0601D52023E3612C2319
:100C6000002206EB850103FB056381F8B3205A7669
:100C7000F8BD63685A04EDD4636843F4804363604D
:100C8000E8E720464EF060FAE4E700BF8028002441
:100C90002DE9F04FDFF854A387B09AF844351BB91B
:100CA000012007B0BDE8F08FDAF80030C54A002B0C
:100CB000D2F86C5119DD0AF104040020C249D4F8BD
:100CC000F830BFF34F8F03F59072C1F85C322033D8
:100CD0009342FAD1BFF34F8FBFF36F8F0130DAF831
:100CE000003004F588749842E9DBB84A4FF00009F7
:100CF000B74BA2FB05125209A3FB0213DB0803EB5F
:100D00008303A2EB43039AF80C260492D9B2B14AAA
:100D1000059102EB830B134602F53872A3F2CC580F
:100D20001E460192049B994500F02681D8F81830A0
:100D3000D8F80470D3F8F810D3F8FC50029106F0FC
:100D4000DBFCA04B382D039093F8704140F26E818C
:100D50000122A1480299542C02FA07F2284493F880
:100D6000717101EB4000009201EB470300F04C81F0
:100D7000009A984240F25581B3F800C01CEA020F75
:100D800000F04781B3F802C01CEA020F00F057815F
:100D9000B3F804C01CEA020F00F05481B3F806C097
:100DA00008331CEA020FE4D10092591A98424FEA24
:100DB000610E40F23681A5EB0E00452828BF452084
:100DC00003EB4000834280F0318100251F46009AEA
:100DD000AC462946CDF80890CDF800E0B3F800E025
:100DE0000EEA020E8E451CD1B3F802E00EEA020EA6
:100DF000714540F0E380B3F804E00EEA020E71455D
:100E000040F0DE80B3F80690083309EA020949454C
:100E100008D1984209D9B3F800E00EEA020E8E45D7
:100E2000E2D00233984200F2AE80BCF1110FDDF83F
:100E30000890DDF800E040F2F980DCF1150200F1E5
:100E4000F5806649039F4B689E455E4BD3F884014D
:100E500038BFC1F804E03B1A002B14DB604B03449D
:100E60009F4201D93B4605335648C0F884314B6850
:100E7000052B40F2EA80053BDBB2524880F8713125
:100E80004FF0FF334B603AB105FA02F2CCF1140C8B
:100E9000012505FA0CF51543524BC5F3C43203EB9B
:100EA0008202906A05F01F0203EB8202916AC5F389
:100EB0004412C5F3842503EB820241EA0031926AB1
:100EC00003EB850341EA02119B6A41EA0321DAF848
:100ED000F83C81EA1122013382EA121202F00F0279
:100EE0000F2A40F08580B1F5803F80F08180542C3E
:100EF0004FEA111100F0AB80B1F5606FCAF8F83C11
:100F000000F0AC80019B998196F858300598834297
:100F100010D0DBF8082033689B1A33607368DBF865
:100F200030209B1A73600023CBF80830CBF83030A8
:100F300086F85800336801333360DBF8083001333A
:100F4000CBF808304FF6FF73994207D1736801332D
:100F50007360DBF830300133CBF83030019B09F19E
:100F600001095C360BF15C0B1433B9F1080F08F181
:100F7000200801937FF4D6AE012301208AF8F43DC6
:100F800007B0BDE8F08FA3EB070E174F33F8021C34
:100F90004FEA6E0E11400EF1010E87FB0E97A7EB84
:100FA000EE774FF0010E012FB8BF0127BD40BC44C2
:100FB000013F0EFA07F73D431F460FE7043331E7C1
:100FC00006332FE78028002400ED00E01F85EB5159
:100FD000CDCCCCCC140A0020C7FFFF7FA403002493
:100FE00020A1070068BB090856555555040000208C
:100FF000542C44D0CAF8F83C4FF6FF71DAF8F43CB0
:101000000133CAF8F43C7FE7204AA2F87A71009ACB
:10101000AFE602330092591A98424FEA610E3FF64A
:10102000CAAE1FB1013F194B83F87171542C95D191
:10103000164AB2F876310133A2F876318EE70433DE
:101040000092B2E606330092AFE6002315E70F48A0
:10105000B0F874210132A0F874214DE70B4A92F8E0
:10106000C13003EB430302EBC3034B4493F8D1308D
:101070000D2B7FF447AF8023019A937744E7034910
:10108000B1F874210132A1F87421B3E7802800245B
:1010900010B5044659F0E8FA0146204689B2BDE889
:1010A0001040FFF7A3B900BF38B50B4D00EB40006F
:1010B00005F24C53C40003EBC003254493ED027AC0
:1010C000D3ED037AE7EE007AB0EE670A59F0CCFA76
:1010D000D5F84C35186038BD0400002038B5002024
:1010E0000E4C4EF071FE0E49A4FB00400D4DD1F8A0
:1010F000FC20800C0C4B42F08072C1F8FC204FF0B9
:1011000060420A49C5F88801C2F8B01F00225A603F
:101110001A6842F001021A6038BD00BF83DE1B432B
:1011200000ED00E080280024001000E055CEACC5A2
:10113000F8B5A0F668042379DB0725D5657994F81E
:101140004C3805F001073D46FBB1D4F848341A6825
:10115000D36A5B08536294F8503823B1B4F85A3814
:101160000133A4F85A3885F00101606C54F064FA38
:10117000012384F84F38002384F84D3884F84E3822
:10118000A4F8563884F84C38F8BD94F84F68012E0E
:1011900003D194F84D3884F84E382046FFF7B6FB5B
:1011A0004EB9012385EA030184F84F38606CBDE82D
:1011B000F84054F041BA0023394684F84F38F5E737
:1011C00038B5A0F668040022344D606C03685A629A
:1011D000A1F12903302B31D895F88C3195F88D1178
:1011E0000133DBB2012B85F88C3109D9B4F85638BC
:1011F00085F88C215B08A4F856384B1C85F88D3196
:1012000095F88D210023082AA4F8583815D185F8BF
:101210008D31B5F88E3101339BB2032BA5F88E3199
:1012200008D92379DB0705D5E36A94F8560843B358
:10123000216B98470023A4F8563838BD5B396C29D8
:101240000CD8B4F8563885F88C215B0843F080033D
:10125000A4F8563895F88D310133CFE794F851381A
:10126000002BCDD1012185F88C31A5F88E3180235A
:1012700084F85118A4F8563885F88D1154F0DCF92B
:10128000BEE7E3696269D054E369E2680133B3FB06
:10129000F2F102FB1133E361CCE700BF80280024A8
:1012A0001A4B4FF48452002170B5054618465AF087
:1012B000EFF9034616492846C5F8883456F004F974
:1012C0001449284656F000F9D5F88864124B0020DE
:1012D00006F58052D3F89031A2F801001B689847B8
:1012E00010232A6913611369DB06FCD460231361A0
:1012F000146914F02004FBD141F2080228461F2390
:101300000121324456F072F8204670BD803200242C
:1013100022BC090829BC09088028002410B504460D
:1013200000F5827155F066FF204604F5317155F0E5
:1013300061FFD4F88834002003F58053587010BD45
:1013400070B54C780546FE2C3ED0FF2C24D0012CE5
:101350003CD1D0F88864898806F580529378022BB6
:101360004BD0012B16D00B0614D5324B812182F8BD
:10137000344093620023537041F228020D2332441B
:1013800055F098FF41F208021F23214632442846B7
:1013900056F02CF8002070BD4B88BBB9CB88ABB998
:1013A00091F90030002B11DBD0F888144FF48075D0
:1013B00041F208021F2301F580540A440121A4F8D8
:1013C000015056F013F8E5E74B880BB1022070BDD1
:1013D000CC88012CFAD191F90030002BF6DA164EA8
:1013E000D6F890319B69984706F5CA73C5F8FC405A
:1013F00086F89401C5F8F030CCE790F8043190F904
:10140000041103F00F0380F80641002900EB830369
:1014100007DBD96B0B68002043F400130B6090705E
:10142000B8E7D9690B68002BF4DA0B6843F0804306
:101430000B60EFE7555342538028002470B5D0F875
:101440008854044605F580514B78022B19D0033B94
:10145000012B14D81D4B41F228028B6200232A4431
:1014600081F834304B700D23812155F023FF41F278
:1014700008021F2301212A44204655F0B7FF00200F
:1014800070BD41F21702497D2A444FF045FD002806
:10149000F5DAD4F88854002201260C4905F580536A
:1014A00020465A7041F22802996281212A4483F829
:1014B00034600D2355F0FEFE41F208021F23314631
:1014C0002A44204655F092FFD9E700BF55534253B6
:1014D0002DE9F041D0F88874044607F580567578F8
:1014E0003DB3012D02D00020BDE8F08141F217028A
:1014F000717D3A444FF010FD0028F4DAD4F8886486
:1015000000224449204606F580535A7041F22802D1
:1015100099628121324483F834500D2355F0CAFE7C
:1015200041F208021F2329463244204655F05EFF4F
:10153000D9E733693363F368F362B0F8D482B8F162
:101540001F0F06D1344BB2689A4202D1717D012936
:101550001DD996F83930204641F25001052403EB9D
:101560004302013307EB8202DBB2545441F25801CB
:10157000042B4FF0200408BF00235454022286F8A5
:101580003930B2704FF076FC0020BDE8F081B37DB9
:10159000013B0F2BDDD841F217023A444FF0BCFC5F
:1015A00000281ADB7378013B022B9CD97368D4F8AE
:1015B0008864B3B106F5805120463A460C6981F83B
:1015C00034500425A3424D7028BF23460C6BE41A07
:1015D0000C63812155F06EFE85E720464FF04AFCF2
:1015E00081E706F580520B49204682F8343053706B
:1015F0000D23916241F228028121324455F05AFEB6
:1016000041F20802434601212046324455F0EEFEE5
:1016100069E700BF555342535553424310B1036825
:1016200082889A61704700BF084B02460220996881
:10163000B2EB910F4FEA910307D25B0840009A4248
:1016400080B202D2FF28F8D970477047A403002463
:1016500038B50409013C052C1AD80F4D00F00F03D2
:1016600005EB4402B2F8C80040FA03F212F001029E
:1016700010D00122254402FA03F3013B18405AF02E
:101680009BF895F8D430054A034402EBC30038BDFB
:10169000002038BD104638BD68BB0908182A002450
:1016A00070B586B00024054600F5847E0DF1040C6B
:1016B000C0F8044144F23B360594C0E93D44C0E91A
:1016C0003F44CDE90144CDE90344BCE80F00AEE856
:1016D0000F00CEF8004095F82131A5F84C610BB908
:1016E00006B070BD1C0903F00F03013C052C33D874
:1016F0001B4E06EB4402B2F8C80040FA03F2D207D0
:101700002AD50122264402FA03F3013B18405AF07D
:1017100053F896F8D430134A034402EBC30452F84A
:101720003320A38812691340DAD1294626200E4AB5
:10173000E080204641F80C2F1A4654F023FDA28881
:101740004FF0B0414FF00043B2FA82F20868D34044
:1017500003430B6006B070BD034BEB60C0E700BFF6
:1017600068BB0908182A0024391A040850B1828875
:101770004FF0B0414FF00043B2FA82F20868D34014
:1017800003430B60704700BF30B1036882881B6958
:101790001A4214BF01200020704708B516F030FB34
:1017A000072807D8044BD3F898340344187DBDE8C4
:1017B00008404DE7002008BD80280024704700BF86
:1017C0000020FFF705BA00BF0020FEF72DBC00BFC8
:1017D0000120FFF7FDB900BF0120FEF725BC00BFC7
:1017E0000220FFF7F5B900BF0220FEF71DBC00BFC5
:1017F0000320FFF7EDB900BF0320FEF715BC00BFC3
:1018000010B1036882889A62704700BFF0B506681D
:1018100000238C68B5690A682B703369DB686B60DC
:10182000002A63D0344B96469A4202D2334B9A42F6
:101830001CD202F01F0C04F11F0322F01F029C4473
:101840002CF01F0CBFF34F8FBCF1000F0ADD944446
:1018500002F120032A4F9C45C7F868221A4603F17B
:101860002003F8D1BFF34F8FBFF36F8F0023C5E97B
:1018700004E303686C625B697BB3F06900224B6828
:1018800002707269D268426043B31B4A1E4693429B
:1018900002D21A4A93421AD203F01F0223F01F0108
:1018A0001F32224422F01F02BFF34F8F002A0ADDAD
:1018B0000A4401F12003124D9342C5F870121946F3
:1018C00003F12003F8D1BFF34F8FBFF36F8F0022D6
:1018D000002344628361C0E90462F0BD094E012225
:1018E00000234462C0E904628361F0BD064BFF221D
:1018F0009E461A700123BAE7405E012400150124B8
:1019000000ED00E020150124001501242DE9F04F21
:101910000668012281888346736890F888A034891C
:1019200086F824201A688C4222F001021A6012D034
:10193000B1F5807F0A469C68A8BF4FF48072022AE6
:10194000B8BF022292FAA2F2B2FA82F2013A62F32C
:101950001E749C6031819BF80C20B17A914208D0B2
:10196000D96821F04071D960D968002A52D0D96075
:10197000B2721A6896F80C9042F001021A60326A4C
:101980009368002B49D04FF0000C1432274C284F9D
:10199000E646DFF8A08052F8101C9E440CF1010CC2
:1019A00001EA04050B4351B1706970B3B5F1005FF2
:1019B0002BD0B94201D2414501D2DB0625D152F8E4
:1019C000143C143203EA040113B1B1F1005F1CD0DE
:1019D00052F80C3C002BDED1B9F1000F15D0BAF152
:1019E000000F12D0BCF1010F0AD8BEF1070F07D8C3
:1019F0000CEB8C0C4FEA8C0C336A63441B7B23B9D1
:101A00005846BDE8F04F5AF09BB85846BDE8F04F35
:101A10005AF08EB841F04071A9E7B9F1000FF4D047
:101A2000BAF1000FF1D09C46E6E700BF0000FEFFD0
:101A3000405E01240015012438B5294B0446D0F836
:101A4000D8105A68D0F8E030501A834200DC23B92D
:101A5000D4F8E4300B44C4F8DC3094F8D030C4F847
:101A6000D820012B05D0D4F8D4300133C4F8D430B9
:101A700038BD201D04F1E8056168EFF3118C1023D7
:101A800083F3128863681B6A0BB3D4F8F0302A46DC
:101A90001BB1D3691432002BFBD10B6A6BB199686F
:101AA00039B99A4209D0196829B15B689968002947
:101AB000F7D01433F3E7C3E900055FFA8CFC8CF32D
:101AC0001188D4F8D4300133C4F8D43038BD5FFA6B
:101AD0008CFC0D628CF31188FFF718FFC3E700BF81
:101AE000001000E082692DE9F04192F8DC308AB004
:101AF0000546012B4CD0023B012B54D892F84C31B7
:101B0000EC46D2F89C2063F07F032D4C137087695C
:101B1000D7F8A03007F11006D7F8108003F1010EB6
:101B20000FCCACE80F00D7F89C30CDE9003E0FCCCD
:101B3000ACE80F0094E803008CE80300EFF3118099
:101B4000102383F312883B691B6A002B2FD0029B62
:101B50006A461BB1D3691432002BFBD1D8F8203070
:101B600073B1996839B99A420AD0196829B15B688A
:101B700099680029F7D01433F3E71E60C3F804D046
:101B8000C0B280F31188AA6911690B6A002BFCD1DD
:101B9000D2F8A0305A8852BAEA819A8852BA2A8278
:101BA000DB885BBA6B8201200AB0BDE8F081C0B26D
:101BB000C8F820D080F311883046FFF7A7FEE2E78F
:101BC00044BC09082DE9F04190F8DC308AB00446A5
:101BD000D0F8A050012B73D041D9023B012B6BD818
:101BE00090F84D31EC46D0F89C2000F1100763F0DE
:101BF0007F035C4E1370D0F8A030D0F8108003F152
:101C0000010E0FCEACE80F00D4F89C30CDE9003EB9
:101C10000FCEACE80F0096E803008CE80300EFF36A
:101C20001180102383F3128823691B6A002B00F0B4
:101C30008F80029B6A461BB1D3691432002BFBD103
:101C4000D8F820302BB3996839B9934221D019685C
:101C5000E1B15B6899680029F7D01433F3E7D0F855
:101C60009C304FF0FF3205211A605A609A60DA60AA
:101C7000D0F8E030C0F8F010B3F57A7F3BD80323FA
:101C800080F8DC3001200AB0BDE8F0811F60C3F8A5
:101C900004D0C0B280F311882269136A002BFCD1F2
:101CA0006B885BBAA4F8D030AB885BBAA4F8D230AA
:101CB000EB885BBAA4F8D43001200AB0BDE8F0810B
:101CC00090F84C2190F84D319B1A5B100133DBB238
:101CD00035F8132005EB430553BAA0F8D0306B88D4
:101CE0005BBAA0F8D230AB885BBAA0F8D430012040
:101CF0000AB0BDE8F08103691A7B2AB35B691BB3A4
:101D000090F8983003B390F84C310122D0F89C0041
:101D100063F07F03C4F8A4401349037094F84D3175
:101D200094F84C0184F800211B1A84F8DC20D4F8C4
:101D3000A0200733C4F804110132D4F89C10C4E980
:101D40003E23C4F8F410B7E7022384F8DC30B3E78D
:101D5000C0B2C8F820D080F311883846FFF7D6FD0E
:101D60009AE700BF44BC09080100040808B51D201B
:101D7000FFF76EFC10B190F9063053B11E20FFF74B
:101D800067FC10B190F9063003B108BD5523C3803C
:101D900008BD5523C380F1E70D4B01380D494FF0C5
:101DA0002C0CD3F830240CFB00110B4842F4000239
:101DB000C968C3F83024814214BF4FF480014FF446
:101DC0000011D3F830240A43C3F83024704700BF11
:101DD00000400258A4030024000002402DE9F04313
:101DE000451E2B4C2C2798462A4B83B007FB0547F2
:101DF00089461646F868984214BF3620352054F0BC
:101E000067FA694601AA3869C7F81C90C7F82880A4
:101E1000FEF726FA9DF804300099032B22D803EB35
:101E200043005A0820234700C00007EB820251F804
:101E3000107B934042583B4002F01002002B18BF29
:101E4000002A4FF02C02C6F3871102FB054414BF91
:101E500001230023B4F92400236303B0BDE8F04359
:101E600054F012B9181F03EB4303DA00C0F3400724
:101E7000C3B203EB43035800202300EB87008340E9
:101E800001F11000496812580B4002F01002D5E72A
:101E9000A40300240000024003464A4A4A4870B4A2
:101EA0004A4CA34298BF10460A461B1A702B00F0FA
:101EB00082800FD8402B7CD0582B5DD0A3F1280115
:101EC000B1FA81F149091378012B0ED0043270BCAC
:101ED0004DF034B8A02B6AD0B82B4BD0882B137898
:101EE0000CBF05210021012BF0D101EB4103956AC4
:101EF00000EBC3035C6A2C4344F004045C62946806
:101F00009C615469DC61546B5C61D56894691E699D
:101F10002C43956B2C43156B2C43156A2C43556A47
:101F20002C432B4D35402C431C61146934BB1C6978
:101F300044F400741C61D469002C2CD11C6944F455
:101F400080641C61D46A002C2CD11C6944F4807418
:101F50001C611C4B98420CBF1E4B1F4B0B449B003B
:101F6000196821F0FF01196019685268114370BCAB
:101F7000196070470721A6E70321A4E7012C1C691B
:101F80001BD044F400741C611C6944F400441C61BF
:101F9000D469002CD2D01C6924F480641C61D46AFA
:101FA000002CD2D01C6924F480741C61D1E7062176
:101FB00089E7022187E7042185E724F400741C6186
:101FC000B9E700BF0000024000040240FF030240E6
:101FD0003F871CFE00820010088200102DE9F04FA0
:101FE000056883B03D226C68D5E90486D8E9007B9A
:101FF000F061384698F80810D6F804904DF004F8CF
:10200000D6F800A03D22317A103750460AF1100A66
:102010004CF0FAFF002301AA6946CBF8003048468D
:10202000C9F80030FEF71CF99DF80430009A5846B4
:1020300003EB4303A9691032DB0053F802C04CF0F4
:10204000100C43F802C0FFF727FF4846E969FFF785
:1020500023FF236823F0010323602B6A9B686268D7
:102060006FF30F0213436360236843F0010323609F
:102070001823327A13FB02AADAF8002042F0010298
:10208000CAF8002098F8082013FB02773B6843F059
:1020900001033B60A36843F48043A360A36843F457
:1020A0000043A360236843F40073236003B0BDE8DA
:1020B000F08F00BF10B582B06A4601A9FEF7D0F8D4
:1020C0009DF80020019C02EB4200032A04EBC003B0
:1020D000196921F0010119614FF00001196159617D
:1020E0009961D961196259620AD852083D234000AA
:1020F000A16800EB820083400B43A36002B010BDD7
:10210000043AE168D3B2C2F3400203EB43035B003D
:1021100003EB82033D2202FA03F30B43E36002B0B8
:1021200010BD00BF70B5264D264AA842264C05F1C9
:10213000010598BF1446A2F1100298BF1546431B33
:10214000702B39D00ED8402B2ED0582B26D0282BD0
:102150002DD118340123012910D0236823F0010365
:10216000236070BDA02B24D0B82B1AD0882B1ED191
:10217000012904F178044FF00503EED1DEB22022EC
:10218000284631464CF040FF1022314628464CF09C
:102190003BFF236843F00103236070BD48340323F1
:1021A000D9E7A8340723D6E730340223D3E7002346
:1021B000D1E790340623CEE760340423CBE700BF99
:1021C000FF0302401000024010040240F8B5264B05
:1021D00093F8C02093F8C1309A4240D1234F3B6816
:1021E000002B21DD3D1D0026214CD5F8B030BFF37A
:1021F0004F8F03F1E002C4F8683220339342FAD1E2
:10220000BFF34F8FBFF36F8F97F8443513B12B7E19
:10221000012B1DD028690121FFF784FF01363B689F
:1022200005F58875B342E0DC05F066FAD7F8F84D9D
:10223000002C0CDD0F4B03EBC4041968083333F892
:10224000042CC8689C4242EA0002CA60F5D1F8BD7D
:102250000023284685F80031FEF7ACF9DAE759F09B
:102260007BFC0028BAD1F8BD80280024040000209F
:1022700000ED00E0000E002038B5037D044605683F
:102280001F2B07D9203B2022696802FA03F30B4277
:1022900006D138BD2022296802FA03F30B42F8D098
:1022A0000A4B0021606883F89C14FFF73BFF237DF5
:1022B0001F2B05D9203B202202FA03F3EB6038BD27
:1022C000202202FA03F3AB6038BD00BF802800244F
:1022D000354B2DE9F04793F8C02082B093F8C13018
:1022E0009A425AD1314C94F81C5EA5B394F8E00E92
:1022F00004F5626490B34FF000082D4F40F20D36A4
:10230000D4F808A001AA6946B4F80C90504608F128
:102310000108FDF7A5FF9DF80430009A504603EB35
:1023200043030121143242F83390FFF7FBFE54F8C7
:10233000183BA845D3F8E02002EA0702C3F8E020E2
:10234000D3F8E02042EA0602C3F8E020DA6842F45B
:102350008072DA60D4D102B0BDE8F0870646236807
:102360000130A78818341968A84234F8042C21F0E9
:1023700080011960DF62196841F0800119605969B4
:1023800041F001015961D96842EA0102DA6024F89A
:10239000046CE4D102B0BDE8F08759F0DDFB002801
:1023A000A0D102B0BDE8F0878028002404000020FE
:1023B000C0C0FFFF38B5037D044605681F2B07D951
:1023C000203B2022696802FA03F30B4206D138BD94
:1023D0002022296802FA03F30B42F8D00A4B0021AD
:1023E000606883F89D14FFF79DFE237D1F2B05D9A0
:1023F000203B202202FA03F3EB6038BD202202FAD0
:1024000003F3AB6038BD00BF80280024D3B20F2B8C
:1024100022D8124B00B503F1930E02E0033373454B
:1024200017D093F800C08445F8D193F801C08C45CB
:10243000F4D102EB42020A48997800EB820300F5DE
:102440003370C3F8D41200EB820083F8CC125DF82D
:1024500004FB00205DF804FB002070476CBC0908F9
:10246000A403002410B40C4C002304F5946C01E088
:10247000152B0CD003EB430201331CF802108142F0
:10248000F6D1144494F9A2045DF8044B70474FF060
:10249000FF305DF8044B70478028002430B5134DA1
:1024A000002305F5CC7C02E00133362B1BD05CF811
:1024B00033408442F8D10CEBC30EDC009EF804E0FC
:1024C0008E45F1D102EB42020948254400EB82031C
:1024D00000F5337095F89D1100EB8200C3F8D4121B
:1024E00083F8CC1230BD002030BD00BF68BB0908A6
:1024F000A4030024F0B1002310B504460E4894F85C
:1025000004E000F5946C01E0152B11D003EB4302BD
:1025100001331CF802107145F6D1831861792068E7
:1025200093F9A224D3B20F2B02D8BDE81040B5E72F
:10253000002010BD002070478028002428B10368C7
:10254000828809B19A6170479A6270470B4A0C4BB6
:1025500090429B6810D002F5806290420CD00949ED
:1025600002F58042904218BF884205D002F5806291
:10257000904201D098087047580870470000014009
:10258000A4030024004001400A4840220021D0F862
:102590004C3410B543F00103074CC0F84C3404F53B
:1025A000967059F075F84FF0FF33C4F8E034C4F872
:1025B000E33410BD00400258802800240120FEF7BB
:1025C00065BA00BF0220FEF761BA00BF0420FEF723
:1025D0005DBA00BF0820FEF759BA00BF1020FEF711
:1025E00055BA00BF4FF47870FEF750BA4FF47C40F4
:1025F000FEF74CBA70B505460C4640B101680F4B6A
:102600000F4A0B449B0A02EB4303B3F8480353F011
:102610005FFE2E68AD88C4F3411204F0030130461A
:102620002B464CF013FD2B46C4F38102C4F300117A
:102630003046BDE870404CF031BD00BF0000FEA741
:1026400068BB090800B1D5E7704700BFCA780AB96E
:10265000002070472DE9F0478B780F46013B052B92
:1026600000F2A7805B4D0446012103EB830005F5D2
:102670009D6684F8981005EBC00106EBC00001F5DB
:102680009D66206191F8E804022800F09480DBB296
:1026900005EB0313D3F8D835C1F8EC34002B00F068
:1026A0008880022381F8E8344FF48073B38104F109
:1026B000200304F11006C1F8003504F15C03C1F8F1
:1026C00004354FEA121802F00F0208F1FF38B8F192
:1026D000050F5AD8DFF8109109EB4803B3F8C8008A
:1026E00040FA02F3DB0750D50123DFF800A1934045
:1026F000013B184059F060F809EB0803222205213C
:1027000093F8D49081440AEBC908C4F81880404675
:102710003B7888F80620013388F80730FFF76AFF16
:102720005AF83930B8F804209A61D5F86C31632B27
:10273000FBD9294B29499B68B1EB930F4FEA9302D0
:102740004FF0020306D252085B008A429BB201D9C5
:10275000FF2BF8D9A382224F224B02E057F8043F07
:10276000B3B1304698470028F8D0236984F8D800E0
:102770001B78012B27D0022B04D195F83836013372
:1027800085F838360120BDE8F0870023A361CCE747
:10279000A46974B1D5F83C3641222021204601338A
:1027A000A271E371C5F83C36FFF724FF2368A288C5
:1027B0009A610020E7E791F8F53404F1100601333F
:1027C00081F8F5347DE795F83936013385F83936E7
:1027D000D8E700BF80280024A403002440420F0053
:1027E000BCBE0908CDAD080868BB0908182A00243A
:1027F00070B50D4C94F80C66A6B104F24444002563
:1028000003E001352034B5420CD0237F002BF8D0F3
:10281000E0680028F5D00135217DFFF7EBFE20347C
:10282000B542F2D1012070BD040000202DE9F04135
:102830000C460546174640B10168114B114A0B443E
:102840009B0A02EB4303B3F8480353F041FD2E68A3
:10285000AD88394630462A464CF040FC2B46C4F33E
:10286000411204F0030130464CF0F0FB2B46C4F358
:102870008102C4F300113046BDE8F0414CF00EBCBB
:102880000000FEA768BB090800B1CFE7704700BF92
:102890002DE9F047A34D05EB0013D3F8D845002CE4
:1028A00000F09980B3F8E27506464FEA0018384602
:1028B00053F00EFD01227B0907F01F07013BBA40D0
:1028C000072B15D8DFE813F0C7000801D400BA00C1
:1028D000EE00FB000800E100934BD3F828141143ED
:1028E000C3F82814D3F8281421EA0202C3F82824D4
:1028F00005EB0803013693F8DC05F6B2FEF7A8FEF7
:10290000824610B11223C671837105EB080393F858
:10291000DD05FEF79DFE814610B11323C67183715C
:1029200005EB080393F8DE05FEF792FE074610B1AB
:102930001423C671837145445046462195F8DF251E
:10294000FFF7A2FF95F8E02548462621FFF79CFFF8
:10295000062195F8E1253846FFF796FF734B9C4218
:1029600000F0C78039D9724B9C425BD003F5C0534D
:102970009C420AD140F614104CF036FC6A4AD2F858
:10298000243423F48013C2F82434A368694A23F45E
:102990000043A360A36823F48043A360A168E368B5
:1029A00021F01F0143F0E8630A43A260E360236D56
:1029B00023F400632365A36843F40003A360236842
:1029C00043F480532360A36823F48003A360236847
:1029D00043F001032360BDE8F087A3F578439C42F0
:1029E00000F0938003F574439C420FD0A3F5784325
:1029F0009C42CAD140F60E004CF0F6FB4A4AD2F88F
:102A0000203423F48043C2F82034BEE740F60C1093
:102A10004CF0EAFB444AD2F8243423F48053C2F841
:102A20002434B2E740F615104CF0DEFB3E4AD2F8F3
:102A3000243423F40013C2F82434A6E73A4BD3F825
:102A40001C141143C3F81C14D3F81C1421EA02020D
:102A5000C3F81C244CE7344BD3F810141143C3F8CB
:102A60001014D3F8101421EA0202C3F810243FE72F
:102A70002D4BD3F818141143C3F81814D3F81814B5
:102A800021EA0202C3F8182432E7274BD3F82C14AA
:102A90001143C3F82C14D3F82C1421EA0202C3F812
:102AA0002C2425E7204BD3F820141143C3F820141D
:102AB000D3F8201421EA0202C3F8202418E71A4BA5
:102AC000D3F824141143C3F82414D3F8241421EAAE
:102AD0000202C3F824240BE7134BD3F81414114358
:102AE000C3F81414D3F8141421EA0202C3F814240E
:102AF000FEE640F60D104CF077FB0B4AD2F824347A
:102B000023F40053C2F824343FE740F60F004CF0A2
:102B10006BFB054AD2F8203423F40043C2F820347A
:102B200033E700BF802800240040025800340140F1
:102B30000038014007000020421C00F051812DE9BF
:102B4000F84F2C23DFF8A493064600FB03F359F853
:102B500003B009EB0302BBF1000F06D09468002C10
:102B600000F01F8194F9061009B1BDE8F88FD2F882
:102B70000CA0BAF1000F00F041819AF90630002B49
:102B8000F3D12C2109EB860206FB01F182F8B0306B
:102B900082F8B13082F8B23082F8B33001F1180215
:102BA0004944D1F8048049F802304A44C2E901336B
:102BB000C2E90333731CDBB2002C00F06D811522D7
:102BC000E371A2711622BBF828008AF807308AF850
:102BD000062053F07DFB2368A288112120469A61CC
:102BE000DAF80030BAF804209A61FFF703FD1121EA
:102BF0005046FFF7FFFC0927332524B9C9E0013D02
:102C000007D004F0EFFD23680A20A28819690A4260
:102C1000F5D09A62052004F0E5FD2368A2889A6148
:102C2000052004F0DFFD013FE6D1002C00F00A8111
:102C3000332503E0013D07D004F0D4FD23680A20CA
:102C4000A28819690A42F5D005209A6204F0CAFDEB
:102C5000BAF1000F00F02F81DAF800300520BAF841
:102C600004209A6204F0BEFD2368A28805209A61C0
:102C700004F0B8FDDAF80030BAF8042005209A61B3
:102C800004F0B0FD2368A2881B691A4240F0A980B5
:102C90002C2303FB06939A7C002A1A7C14BF36214E
:102CA00016212046FFF7C2FD2C2303FB06939B7CD5
:102CB000002B14BF36211621BAF1000F06D02C23A9
:102CC000504603FB06935A7CFFF7B0FD40460024B4
:102CD0004CF03AFAD8F81010834A42F6E05321F04B
:102CE0007041C8F81010D8F8101021F47001C8F81D
:102CF0001010D8F8101021F47021C8F81010D8F86E
:102D000010100A432146C8F81020D8F8102022F4E9
:102D10007F42C8F81020D8F8102022F0FF02C8F82F
:102D20001020D8F810201343C8F81030C8F8084015
:102D3000D8F8083043F40043C8F80830D8F8003019
:102D400023F40033C8F80030D8F8003023F480535F
:102D5000C8F80030D8F8003023F47063C8F80030A9
:102D6000D8F8003043F47063C8F80030D8F8003069
:102D700043F00103C8F800309BF82B0053F084F9AE
:102D800021469BF82A00BDE8F84F53F07DB904F0C6
:102D900029FD013D4FF00A00F9D1052004F022FD84
:102DA0003EE7D2F80CA0BAF1000F7FF4E6AE18337C
:102DB000D2F8048049F803A04B44C3E901AAC3E94F
:102DC00003AA09EB8603BBF8280083F8B0A083F8B8
:102DD000B1A083F8B2A083F8B3A053F079FA0AE760
:102DE00070472C23DAF8002003FB069312699A7CC3
:102DF000002A1A7C0CBF1621362152E71833D2F86C
:102E0000048049F803A04B44C3E901AAC3E903AA1B
:102E100009EB800383F8B0A083F8B1A083F8B2A0D7
:102E200083F8B3A01523A371431CE371BBF82800FA
:102E300053F04EFA2368A288112120469A61FFF7C9
:102E4000D9FBD8E6332401E004F0CCFC013C4FF080
:102E50000A00F9D1052004F0C5FCBAF1000F39D001
:102E6000DAF800300520BAF804209A6204F0BAFCBF
:102E7000052004F0B7FCDAF80030BAF80420052089
:102E80009A6104F0AFFC2C2303FB06939B7C002B80
:102E900014BF3621162112E78AF8073016238AF864
:102EA0000630BBF8280053F013FADAF80030BAF80D
:102EB00004209A619BE6052004F094FC2368A28814
:102EC00005209A6104F08EFC052004F08BFC236839
:102ED0001B69DDE6052004F085FC052004F082FC7A
:102EE000052004F07FFCF1E6000042408028002429
:102EF00070B590F8723004461D09013D052D11D8BA
:102F00001D4E03F00F0306EB4502B2F8C81041FA5C
:102F100003F2D20706D590F87520012AD0B205D069
:102F2000012070BD94F875300120FAE7984001380F
:102F3000084058F041FC7319104A93F8D430034408
:102F400002EBC30552F83320AB8810691840E8D073
:102F5000002394F873200221284684F87530FFF787
:102F600065FC236E1A6822F008021A601A6842F0A3
:102F700008021A60D4E700BF68BB0908182A0024B9
:102F8000F8B50E4C94F80C7697B104F5C2640025A0
:102F900001E0082D0ED0A6683079FEF759FB217D9F
:102FA000F27908B1FFF742FC01358034BD42F0D11F
:102FB0000120F8BD00239B68FFDE00BF0400002055
:102FC0002DE9F04FDFF8E0829BB098F840A6BAF107
:102FD000000F03D100201BB0BDE8F08F00222F218D
:102FE00050460DF019FE06460028F3D00568C8F8D3
:102FF0004456FFF77FFA0028ECD0D0E90149C8F821
:103000004846002CE6D09E4F00233A4601E0102BA4
:10301000E0D0516818462C3201338C42F7D1DFF8EA
:103020008CB22C2303FB00B393F92C20002AD1D1BE
:1030300050464FF02F0AA3F82CA0FEF709FBC8F862
:103040004C0628B1A0F806A02621F279FFF7EEFB86
:10305000DFF85CA200230AF55A7151F8332095423B
:1030600000F0F18001330E2BF7D1002053F030F93E
:103070002B6823F001032B60824B9D4200F0E88017
:1030800003F580639D4200F0E38003F57053DBF8A5
:1030900008109D4200F0E6807B4AAA1AB2FA82F23A
:1030A0005209002A40F0DE8003F5006377489D4214
:1030B00000F0DE80B0EB910F4FEA91030AD8744A1A
:1030C00074491A44A1FB0212920D013A92B2511CAA
:1030D000B3FBF1F31B0AADF810206F4A4FF0000B61
:1030E0006E492846A2FB0332ADF812B01309ADF8C1
:1030F00014B01209ADF820B0A1FB031304A9069285
:103100005B08CDF824B0CDF81CB0A8F852365B00AF
:10311000A8F850364DF066FA602271792846CDF84D
:103120000CB0CDE901BB4DF0DBFBB3799A077BD541
:103130000423ADF806300022717928464DF026FCB4
:1031400001AA717928464DF0C9FA602271792846A2
:103150004DF0C6FB7179284608224DF035FC6B6CAA
:10316000284643F400436B642B6843F080032B60D4
:10317000B37971799B075FD552F0BCFD2B680020B5
:1031800043F001032B603B4601E0102857D05A68FA
:1031900001302C339442F8D1FEF7FEFD002001E00F
:1031A00010284ED07B6801302C379C42F8D1002388
:1031B00060223B490027FEF711FE2046FEF77AFF0A
:1031C00000212046FEF7AEFF2046FEF773FF354B89
:1031D00072790BA90F9340232046CDF830901393BA
:1031E0004FF48053109711934FF44033159305F12A
:1031F000340303EB82030D9301230E93129340F2E9
:103200002A431493FEF748FE7379032B03D80AEB85
:103210004303B3F8D873EB68204610213B43EB60BF
:1032200053F062FB0120D6E60123ADF804304FF4E1
:103230008073ADF80C307EE752F086FD9EE70020EB
:10324000AAE70020B3E70AEBC303B3F86C030DE76A
:10325000DBF808200D495308B1EB520F7FF62FAF72
:10326000002237E7094A4B08B2EB510FF8D826E79E
:10327000B0EB510F4FEA51033FF62CAF1FE700BFF1
:10328000B00300240000014000440140006CDC0257
:1032900000366E01819F5E16598B4F01ABAAAAAA18
:1032A000792204084066012480280024A403002415
:1032B00068BB090830B5184B83B0BFF34F8F17496F
:1032C00003F58652C1F8683220339342FAD1BFF336
:1032D0004F8FBFF36F8F124C01AA6946D4F848563E
:1032E0002846FCF7BDFF9DF80430009A40F22A41C1
:1032F00003EB4303D4F844461432DB0020469950D4
:1033000052F0DEFC2368012128460B43236003B002
:10331000BDE83040FEF706BF4066012400ED00E046
:1033200080280024C74BD3F85416D3F8582670B51C
:103330008C0F93F82851100EC2F3072C83F888469F
:10334000C1F383640001012D83F88946C1F3016450
:1033500083F88A46C1F3074483F88B46C1F30724F8
:10336000C9B283F88C46C2F3035483F88D16A3F8D0
:103370008E06C2F3C030B3F88E1689B241EA04015A
:10338000C2F30344A3F88E16C2F3403183F890468B
:10339000C2F3803483F891064FF0000083F8924620
:1033A00083F89316C2F3003183F89416D3F85C16B1
:1033B00083F8950640F2EF80022D00F0C3802A20AA
:1033C0004FEA4C0C83F8A146C1F3C01201F07F0113
:1033D0000CF07E0C83F8A2C64FF0010C93F8A246C5
:1033E0001443D3F8602683F8A246D40F83F8A316BB
:1033F000910D83F8A446C2F3417401F00C01C2F3AD
:10340000815583F8A546C2F3826483F8A64683F803
:10341000A71693F8A716D3F86446294383F8A7168E
:10342000C2F3405183F8A816002183F8A916C2F30D
:10343000004183F8AA16C2F3C03183F8AB16C2F379
:10344000803183F8AC16C2F3403183F8AD16C2F375
:10345000003183F8AE16C2F3812183F8AF16C2F3B0
:103460000121C2F3460283F8B016C4F3074183F882
:10347000B126220E090283F8B2C683F8B426C4F33B
:103480000722A3F8B6162406B3F8B61689B211437C
:10349000A3F8B616D3F86816C3F8B8460C0ED3F8DE
:1034A000B82642EA0442C3F8B8260A0AD3F8B84656
:1034B00002F47F422243C1F30724C9B2C3F8B826FD
:1034C000D3F8B856D3F86C262C43C3F8B84683F823
:1034D000BC16110E83F8BD16110C0906C3F8C016F0
:1034E0001102D3F8C0460A4601F47F01214392B28B
:1034F000D3F87046C3F8C016D3F8C0160A43C3F811
:10350000C026C4F30352D3F8C01641EA1461C3F8CD
:10351000C01693F8C4161143C4F3072283F8C416E7
:10352000210A01F47061A3F8C616B3F8C61689B271
:103530001143C4F34602A3F8C61683F8C82683F8DD
:10354000C9C670BD1204C1F3072C0D0E02F47C1223
:10355000C3F89826C1F30742D3F8984644EA0524F5
:10356000C3F89846D3F8984622434FF40074C3F842
:103570009826D3F89826C3F8D846013240F10004C3
:10358000A40244EA92549202C3F8D446C1F38034B0
:10359000C3F8D02614E74FEA8C2CC1F3C26594001F
:1035A0000CF44062C1F3072C04F47F74C3F898262E
:1035B000D3F898261443CA0BC3F8984602F00602C3
:1035C000D3F8984644EA9174C3F89846C1F302646C
:1035D00083F89C56012583F89D46C1F3425483F835
:1035E0009E46C1F3824483F89F46C1F3C03483F8FA
:1035F000A02693F8A026224383F8A026D3F8984665
:1036000093F8A02693F89066023205FA02F2B540CC
:10361000D617A2FB052EC3F8D85605FB06EE04FB11
:103620000EEE0134A2FB0424A644520AC1F38034F6
:1036300042EACE52C3F8D0264FEA5E22C3F8D4261F
:10364000BEE600BF802800240B4801230B4A40F24D
:103650000D1110B50468D2F824212046FCF7CCFFE8
:1036600040B96069C0F34320A0F10400B0FA80F0D3
:10367000400910BD002010BDA403002480280024B0
:103680002DE9F047754D95F8E0462CB1744B93F851
:103690008C432046BDE8F087714E0321714A4FF0FC
:1036A0000108336885F8E08658680240022042F03D
:1036B000F4025A603368196004F032F9376823461F
:1036C000224621463846FCF797FF0446A0BB072355
:1036D0004FF4D5724FF484713846FCF78DFF80B3F8
:1036E000A2460123002240F237113846FCF784FF3E
:1036F000044608BBDFF8749180464AEA09090FE0E6
:1037000040F229113846FCF777FF08F101084FF61F
:10371000FE72044680B97B69002B17DB904515D8F3
:103720000123002240F237113846FCF765FF0323DE
:103730004A4604460028E3D0204686F88C43BDE87C
:10374000F0874FF0804A85F82881CAE74FF6FF726C
:10375000904500F08180590064D53B684FF0020825
:103760009A0785F8288166D00223002240F20231B0
:103770003846FCF741FF04460028DDD17B69B8F1EB
:10378000020FC5F86436BB69C5F86836FB69C5F831
:103790006C363B6AC5F870364FD9B8F1060F4CD07D
:1037A0000223D5F8242140F209313846FCF724FFE2
:1037B00004460028C0D17B69C5F85436BB69C5F8FA
:1037C0005836FB69C5F85C363B6AC5F86036FFF7CA
:1037D000A9FD04460028AFD10123D5F8242140F2E9
:1037E00007113846FCF708FF7A681E4B0446134061
:1037F00043F008037B6000289ED195F8E6363BB382
:103800004FF48040FCF7AAFF04463268164B51681B
:103810000B4043F0080353603268536843F40033AD
:10382000536089E73B689B0705D095F82881B8F17C
:10383000040FCCD098E726247EE70623002240F22E
:1038400003113846FCF7D8FE04460028A8D073E7D9
:10385000FCF784FF0446D8E71B246DE7802800248A
:10386000A4030024002CFEFF00ECFEFF00001080EB
:1038700038B5444D2868436BDA0525D54FF480727E
:10388000414B424C8263026D22F001020265C26B21
:103890001340C363036D23F040030365D4F884260B
:1038A00012F002024DD00022C4F88026D4F88436EB
:1038B000DB074CD429680122354800238863C4F80B
:1038C0007426C4F8783638BD426B436B12F03A0266
:1038D00029D09B0741D4436B1C0743D52B4B0422B3
:1038E000C3F878262A4A012327498263C26B114014
:1038F0000022C163016D21F040010165C16A41F4FC
:103900000051C162C16A21F40051C1624FF4867155
:10391000FCF772FE2B684FF400629A631A6D22F076
:1039200001021A6538BD1B01CDD54FF00061174B60
:1039300081632C21C3F878161349C36B1940012306
:10394000D7E7C4F87C26D4F88436D907B2D501234A
:103950004FF48671FCF750FEACE70C4B0222C3F823
:103960007826BFE7436B990607D4436BDA06B9D5CF
:10397000064B0522C3F87826B4E7044B0622C3F8A9
:103980007826AFE7A4030024C53EFFFF802800246B
:103990003A0F0018FFF76CBF2DE9F0471D4612F0F3
:1039A0001F0372D13E4F1446DFF800912946C7F835
:1039B0007436064697F8283100224FEA452840F22F
:1039C000111A022B18BF4602204652F039F9D9F8D5
:1039D0000000344B4FF400724FF488714362C0F81A
:1039E0002880C36A43F09303C3620123FCF704FEFB
:1039F000022DD9F800904FF00A0528BF4FF4897ABC
:103A00000123324651464846FCF7F6FD50BBD7F835
:103A10006C0141F28831D7F8742642B9D7F86C317D
:103A20001B1A8B4234D8D7F87426002AF6D000230C
:103A300024F01F04C7F87836BFF34F8FB8F1000F9A
:103A400009D0A8F12008184AA044A045C2F85C4259
:103A500004F12004F9D1BFF34F8FBFF36F8F002023
:103A6000BDE8F087013D0123002240F237114846AE
:103A7000EDB2FCF7C1FD08B1002DC1D10028C6D0C0
:103A80000023C7F87C36BDE8F0870920BDE8F08741
:103A90000420C7F87806C7F87C26BDE8F08700BF89
:103AA0008028002400E1F50500ED00E0A4030024D7
:103AB000D1066AD12DE9F84F354D9A46834640F23A
:103AC000191895F82831914614460A26022B314BD5
:103AD00018BF4FEA402BBAF1020F1F6838BF4FF4EE
:103AE0008C7801235A4641463846FCF785FD90BB49
:103AF0004FEA4A26BFF34F8F3EB109EB0602264B31
:103B0000C3F8684220349442FAD1BFF34F8FBFF319
:103B10006F8F01225146484652F092F81D4B1F4AC2
:103B200041F288301B685A629E62DA6A42F0910262
:103B3000DA62D5F86C1104E0D5F86C315B1A834277
:103B40001CD8D5F87426002AF6D000231846C5F8EC
:103B50007836BDE8F88F013E0123002240F237118C
:103B60003846F6B2FCF748FD08B1002EB9D100285E
:103B7000BED00023C5F88036BDE8F88F0420C5F814
:103B80007806C5F88026BDE8F88F0920704700BF89
:103B900080280024A403002400ED00E000E1F505E6
:103BA000F0B5AE4B8DB0046E05469C4200F0BA8174
:103BB0002BD8A3F530539C4200F0C68100F29D81C2
:103BC000A3F500639C4200F0378103F580639C42BB
:103BD00040F0CC81A24B1220D3F8202442F4802262
:103BE000C3F82024D3F8202422F48022C3F8202410
:103BF000AE684CF0E9F822687308170428D403442F
:103C0000B3FBF6F39BB2E3602DE0964B9C4200F0D1
:103C1000B08103F580639C4200F02E81A3F5184328
:103C20009C4240F0A3818E4B0220D3F8202442F026
:103C30000042C3F82024D3F8202422F00042C3F825
:103C40002024AE684CF0C0F8226873081704D6D55B
:103C500003EB40034FF6F071B3FBF6F3C3F34202FC
:103C60000B401343E36021686B7921F0010113F0ED
:103C700004022160216821F010212160216818BF11
:103C800041F4805113F0020F2160236823F00103F7
:103C90002360636823F440536360636818BF43F490
:103CA00000536360236823F001032360236823F437
:103CB000C06323602368002A00F0F08043F480632F
:103CC0002360236823F001032360A36823F4807337
:103CD000A360A368A360236823F001032360A368A3
:103CE00023F40073A360A368A3602B79DE0700F1BF
:103CF000E080980700F1D48095F938006E79FDF7DF
:103D00004CFD20B106F00101FEF718FC6E79236826
:103D1000310723F001032360A3684CBF43F008037D
:103D200023F00803A360236843F0010323602B7989
:103D3000DA0748D5EE6B002E00F0CD800023012776
:103D40003046029307930993069308934FF4803308
:103D500004970B93EB6D03936B690593EB680A93E0
:103D6000FEF7A8F9304601AA6946FCF779FA02AADB
:103D70009DF8041000984BF0E1F839463046FEF704
:103D8000D1F9394BA2689E4238493B4442F0400287
:103D900098BF0B46A260A6EB0306354A354B98BF89
:103DA0001346702E00F0FE8000F28C80402E00F052
:103DB000F780582E00F0EE80282E00D118331A68B4
:103DC0002B7992B26A659B0734D52E6C002E00F0D9
:103DD0008F8000240123AA6D304604930392AA69C0
:103DE0000294CDE907432B69CDE905240A934022CB
:103DF0004FF4803309920B93FEF75CF901AA6946F0
:103E00003046FCF72DFA02AA9DF8041000984BF0FA
:103E100095F89621304652F067FD2146286CFCF754
:103E20005DFA2C6EA36843F08003A360236843F01F
:103E3000400323600DB0F0BD094B1120D3F82024BE
:103E400042F40032C3F82024D3F8202422F40032B4
:103E5000C3F82024AE684BF0B7FFF5E600780040C9
:103E60000040025800100140FF03024000000240E1
:103E700014000240140402404B4B1320D3F82424B6
:103E800042F02002C3F82424D3F8242422F0200294
:103E9000C3F82424AE684BF097FFD5E6236010E703
:103EA000236823F008032360236843F0080323609A
:103EB00022E7226822F004022260226842F0040213
:103EC000226016E7A02E69D0B82E65D0882E7FF428
:103ED00076AF783373E7226A42F0200222622268CA
:103EE00042F020022260226842F0100222606AE75B
:103EF000236843F08003236098E72C4B9C4235D124
:103F0000294B0220D3F8202442F48012C3F8202445
:103F1000D3F8202422F48012C3F82024AE684BF09A
:103F200053FF91E6204B0220D3F8202442F0804238
:103F3000C3F82024D3F8202422F08042C3F82024A0
:103F4000AE684BF041FF7FE6174B0220D3F82024E8
:103F500042F40022C3F82024D3F8202422F40022C3
:103F6000C3F82024AE684BF02FFF6DE6AE6800204A
:103F70006AE60D4B1020D3F824240243C3F824240E
:103F8000D3F8242422F01002C3F82424AE684BF0A6
:103F90001BFF59E6483312E7A83310E790330EE7CA
:103FA00030330CE760330AE700400258005000400D
:103FB0002DE9F041044682B0EFF31185502383F3DD
:103FC0001288066C01AA69463046FCF749F9019B44
:103FD000009803EB43031030DB00C358DB0705D523
:103FE000EDB285F3118802B0BDE8F0813046FCF7F0
:103FF00037F99DF80430009803EB43031430DB00DD
:104000001F58BFB207BBD4E90903984228D0A06962
:1040100000EB03083046FCF723F99DF80430009AC2
:1040200003EB43031C32DB0043F80280D4E909317F
:104030008B4213D822693B46511AA36200233046B3
:1040400084F86430FCF74AF901213046FEF76AF83B
:10405000EDB285F3118802B0BDE8F081591AECE7A2
:10406000012384F86430BBE7F8B5044600681822E1
:10407000217A00F1100C12FB01C2032900F2978093
:104080004B0806259B0015FB01352023AB40056836
:104090002B40156805F01005002B37D0B5B3202252
:1040A000E5694AF0B1FF217A206810224AF0ACFF9E
:1040B000217A2068032900F29D804B0802460626DB
:1040C0009B0052F8247B16FB0136182313FB0123B7
:1040D0001A680123B34002F080023B401BB112B1C9
:1040E00001224AF091FF2846FFF762FF95F86430FD
:1040F00043B195F87530022B04D095F87530002B3C
:1041000000F08E802068217A00F1100C182203291B
:1041100012FB01C22CD84B08062506689B001768C5
:1041200015FB01350823AB40334212D07B0710D575
:1041300008224AF069FF217A206803294AD84B08EF
:10414000062500F1100418229B0012FB014215FB0A
:104150000135042306681468AB4004F002043340C0
:104160002BB124B10422BDE8F8404AF04DBFF8BDA0
:104170000D1F4FF0080C4768061DEBB2C5F3400554
:1041800003EB43035B0003EB85030CFA03F5D2F862
:1041900000C03D4202D01CF0040FC9D1356814683C
:1041A000042202FA03F304F002042B40D8E7A1F141
:1041B000040E4668156820235FFA8EF2CEF3400E97
:1041C00005F0100502EB4202520002EB8E02934012
:1041D000334061E70A1F00F11004061DD3B2C2F399
:1041E000400203EB43035B0003EB8203182212FB44
:1041F0000142D3E70A1F00F124031827C2F3400647
:1042000017FB0137D3B203EB43035A00012302EB40
:1042100086029340426813403A6802F080025DE7EC
:1042200095F87200FDF714FA2B6E01211A6822F03E
:1042300008021A601A681A6085F8751000283FF4A1
:1042400061AF2021FEF7D6F95CE700BFBFF34F8FC7
:104250000549064BCA6802F4E0621343CB60BFF322
:104260004F8F00BFFDE700BF00ED00E00400FA053E
:1042700008B572B6FFF7EAFF70B541F2043082B0BC
:104280004AF0B2FF7A4A41F60F40D2F8003843F4C0
:104290008073C2F800384AF0A7FF4FF40043754915
:1042A00001938B689C0613D45323CA224A624B6243
:1042B000CB6823F02003CB6000E033B1CA68019BD8
:1042C000900603F1FF330193F7D56A4BFF225A6240
:1042D000684BFF24CA205321674A5C6258625962C6
:1042E000D2F87424D20003D51A6D644B9A4212D0CE
:1042F000634ACA245F4B53200026FF21614D5C6254
:10430000586242F8046BAA425962F8D15B4A5C6277
:1043100058621A655962574BDA6D012A5AD0564ACB
:10432000D2F80834C3F38103022B00F09380032BEF
:104330006CD0012B63D1544A4F4B40F60D7053495A
:10434000534D544CE160D3F87414AA60D3F8302470
:1043500022F48042C3F83024D3F8742442F08072EF
:10436000C3F874244C4BC3F8EC164AF03DFF40F6FA
:1043700015404AF039FF40F616404AF035FF40F646
:1043800017404AF031FF4FF498504AF02DFF40F6A5
:1043900005604AF029FF40F606604AF025FF4FF419
:1043A00060604AF021FFFCF799FE3C4AAB68A2FB33
:1043B00003239B09013BB3F1807F09D24FF0E02238
:1043C000F02000215361072384F8230091611361D9
:1043D00002B070BDCA2153220024FF2059625A62E4
:1043E0002C492F4ADC6558628A60BFF34F8FBFF3B8
:1043F0004F8F136883F3088853689847FEE7D2F815
:10440000C434284AC3F30143DA4095E7D2F80444A0
:10441000D2F80414D2F8043404F03F04D2F898041B
:10442000C1F38811C3F3064310F4403F01F10101C9
:1044300003F10103C0F301450ED1D2F8C404194AB7
:10444000C0F30140C240B2FBF4F201FB02F2B2FB46
:10445000F3F271E7144A6FE7012D0CBF124A0A4AC2
:10446000B2FBF4F201FB02F2B2FBF3F264E700BF2D
:104470000050005800400058004002583166654224
:10448000544000586C40005800127A000005FA05AC
:10449000A403002400ED00E080280024D34D621026
:1044A0000000F01F0090D00300093D00704700BFDE
:1044B000154A830AB2EB902F0CD3B3F5801F1ED39D
:1044C0006FF480121A44042A1BD8DFE802F00E10A1
:1044D00012140C000D4A93420FD00D48834214BFB2
:1044E000FE200720704706207047022070470320F7
:1044F0007047042070470520704700207047FE2059
:1045000070470120704700BF0500100040001000F8
:10451000410010002DE9F04FDFF8FC828FB04FF022
:10452000000CDFF8F892B64DA8F5A966DFF8F0A206
:10453000CDF808C008E0013B012B00F21C810AF114
:104540001C0AC24500F00C81DAF800703846FFF70B
:10455000AFFF072899F82237EDD83044012B90F8A7
:10456000604404F1010464B200F0F280022B01D136
:10457000082CE4D14FF0000B1FFA8BF120460CF011
:104580006BFA0CF0F3FA90F90030002B18BF542BA3
:1045900014BF0123002340F0F0800BF1010BBBF1AD
:1045A000040FE9D1029A22B395499B4601970AE08C
:1045B000304490F86024013252B2A2420CD001F58E
:1045C0008871A94211D08F683868FFF771FF0728FA
:1045D000EED90022A242F2D17B799AF805209A42C4
:1045E000ADD001F58871A942EDD15B46019F002B4A
:1045F000A5D1DAF808000022824B03E001320C3327
:10460000102A9CD059688842F8D152B29AF8051005
:104610003846FDF743FF002891D0446800237A4ACA
:1046200003E0102B02F12C0289D0516818460133A7
:104630008C42F6D12C23754A03FB002090F92C30D4
:10464000002B7FF47CAFDDF808C0C5F808A005F5A5
:1046500088750CF1010CBCF1040F7FF467AF6C4A54
:104660004FF0010B92F80C3602F2444A01330493E6
:10467000049B5B4569D099F83637DAF80C600593EE
:104680009AF810300293002E5FD0614B34681D6899
:1046900060482746B388002D204401934FEA9020BC
:1046A00073DD574A002304E0013302F58872AB4200
:1046B00068D011688142F7D103EB0313504A019D82
:1046C00002EB0314029B4FF00302CAF80C604FF098
:1046D000030E8AF81030019BCAF81840B3FA83FC25
:1046E000CCF11F03CAF80430B271012286F807B07A
:1046F0005E00E16C02FA03F30EFA06FE02FA06F619
:10470000606C314340EA0E00D4F850E0E164404967
:10471000606491F8446599B2D4F8B000002E00F0BE
:10472000DE8043EA0E032365BD61FBF71DFE0BF13E
:10473000010B2046FBF73EFF0AF1200A40F201136D
:10474000BBF1090F2AF8043C92D10FB0BDE8F08FFD
:10475000012C3FF40FAF0AF11C0AC2457FF4F4AEFE
:10476000DDF808C005F588750CF1010CBCF1040FEB
:104770007FF4DCAE73E70024FCE6029A002A7FF4A3
:1047800013AFDCE6042B00F00482214A05EB05138D
:1047900002EB03132A010692DA680392002A00F062
:1047A000158258604FF05402013083F81021C2B2D4
:1047B00083F811216B1C0892154A13600022039B99
:1047C000597918689F688C460E4B04E001320C330F
:1047D000102A00F0078259688F42F7D1614652B221
:1047E000FDF75CFE069B0A4A2B44DFF81C8002EBB7
:1047F00003134146D0E90172C3E90572002215E0B6
:104800000800002070060024B0030024A403002444
:10481000040000200000FEA7B0C009088028002482
:10482000D0BF0908102A01F12C018ED04868134628
:1048300001328742F6D12C21734A079701FB0323EB
:1048400093F92C10002980D1D2F808E04FF0540CD5
:10485000069A08992A4483F82CC083F82D106B49D6
:1048600042F31B036A4801FB03F36A4900F5607CCD
:1048700001EB02118C60C3EBC30403EBC30300EB39
:1048800044100CEB4313C1F8B4001001C1F8FC3024
:1048900033230990C1F8B8308C235F48C1F8003148
:1048A000039900EB02145D4B09689942089122D0EC
:1048B00003F5806399421ED0594A03F5804399421B
:1048C00018BF914217D003F58063994213D0059B1E
:1048D0004FEA9E02062B13D15249534B19E0CCF1FB
:1048E0002F0C02FA0CF3324643EA0E032365BD6235
:1048F000FBF73AFD1BE7059B4FEA5E02062BEBD068
:10490000072B4A484A4B4B4918BF19464A4B18BF18
:1049100003464048089FB2FBF3F3B2FBF1F206995D
:10492000013A013B29449BB200EB01110430A1F88C
:10493000BC20099AA1F8743002F158010022A4F8B1
:1049400068204250014423663846A4F85C20626621
:10495000E2664BF047FE3B683846602243F0800336
:104960003B60039B59794BF0BBFF012302210A22D4
:104970003846CDE90B314FF480730D93039B597981
:104980004CF004F83B6838460BAA23F001033B6067
:10499000039B59794BF0A2FE039B3846602259795C
:1049A0004BF09EFF039B1879002840F0FD80089A89
:1049B0000020079F136843F00103136004E01028F0
:1049C00008F12C0800F0ED80D8F8043001309F4247
:1049D000F5D107970590FDF7DFF9039B05985B7903
:1049E000032B00F2DC80154A02EB4303B3F8D81323
:1049F000069B084A2B4402F6FC5C02EB0313DDE93C
:104A0000077E1982002322E0A4030024F1F0F0F0D5
:104A1000405E012404000020080000200000014046
:104A200000400140882A1100A0BB0D00D0DD060027
:104A3000449508001055220040771B0068BB090808
:104A4000964500F0C9800133042B00F0C8805CF863
:104A50003320002AF4D1654A07971746D2F8F82D7B
:104A60000132C7F8F82D07EBC302089FDB00C2F83C
:104A7000FC7D9C44902223460027BCF804E04FF0C4
:104A8000010841EA0E01ACF804105949FDF7A6F9F6
:104A90000798102151F028FF069B84F874804FF48A
:104AA00000322B44C4F88480C4F8A0801D464F4BCC
:104AB00003EB0515C4E92577AB69C4F8AC204FF4C6
:104AC0008052A3674023C4F89070C4F89C70C4F867
:104AD000A430D5F8B830C4F8A830AB68C4F880204A
:104AE00003F118020593099BE2674FF48042D5F861
:104AF000B410C4E9221203F174013E4A68691144FA
:104B00000390FDF7C9F9099B3A4A03F11C01039888
:104B10001144FBF717FD059B84F8BC804FF400613E
:104B2000C4F8CC8003F11000C4F8E8804FF4804250
:104B3000C4F8EC70DDF80C80C4E93777AB69C4F8D1
:104B4000D870C4F8C0304FF44033C4F8E470C4F8EF
:104B5000F430D5F80031C4E93101C4F8F0304046F2
:104B6000D5F8FC30099DC4E9343205F1BC01214A75
:104B700011441746FDF790F905F1300140463944DC
:104B8000FBF7E0FC4046102151F0AEFE3768B588D7
:104B900098E5032389F837370FB0BDE8F08F00217F
:104BA00026E70020079715E7FCF752FD059038B17E
:104BB000039B0221DA79FDF739FE5422059BDA8046
:104BC000089A536C43F400435364F0E6022389F8D7
:104BD00037370FB0BDE8F08FDB00079749E70023B8
:104BE0009B88FFDE00235B68FFDE00BF040000201F
:104BF00019030000080000201E4B93F88D13B9BB69
:104C00002DE9F047DFF8748098F8483573B308F25F
:104C10004C545027184E2C25894608E0013198F84D
:104C2000483554F8182B9942C2F800901EDA237CBC
:104C3000002BF3D0D4F804A05046FFF739FC072826
:104C4000ECD8EFF3118387F31288DAF8242005FB00
:104C50000060DBB20132C0F86027DAF8142042F0BD
:104C60000102CAF8142083F31188D7E7BDE8F08762
:104C7000704700BFA4030024802800240400002003
:104C800010B5002386B001390068144C89B2CDF804
:104C90000230ADF81030A04205930393104B0291FF
:104CA0009B6810D00F4988420DD004F5804401F56F
:104CB0008041884218BFA04205D001F5806188423A
:104CC00001D09B0800E05B086946B3FBF2F2013AB1
:104CD000ADF800204BF086FC06B010BD000001408E
:104CE000A4030024000401402DE9F04385B00D46E3
:104CF000804619469DF834602846BDF83090FFF78D
:104D0000BFFF2C686F79002E3FD0AE7986F0010688
:104D100000236022394620460393CDE901334BF04E
:104D2000DFFDB30733D5F600042306F00806ADF81F
:104D30000630ADF80A604A46394620464BF026FE5A
:104D400001AA394620464BF0C9FC3946204660226C
:104D50004BF0C6FD3946082220464BF035FE626C0A
:104D6000234642F400426264226842F0010243F8A2
:104D7000342B00226979C8F8044003EB8103C8F89A
:104D800000301A6005B0BDE8F083AE79C0E70123BA
:104D90007600ADF8043006F002064FF48073ADF8EB
:104DA0000860ADF80C30C6E710B50446FFF768FFA1
:104DB00000232168164C0A6804F55A7042F001027B
:104DC0000A6050F83320914208D001330E2BF8D1FD
:104DD00001210020BDE8104051F056B904EBC30496
:104DE000012194F86E43204651F04EF91B2C07D058
:104DF0002E2C0BD101212C20BDE8104051F044B9DC
:104E000001211920BDE8104051F03EB910BD00BF8E
:104E100068BB090870B50468054616462046FFF7CA
:104E200047FB072845D86A790223844603FA02F52E
:104E300000EB800300EB43031344002945D0E268F4
:104E400028482A4300EB8305C5F83C17C5F84C6792
:104E5000E260EFF31186502383F312882C2303FBC7
:104E60000C02D2F8381729B3C2F85C1704311E4B74
:104E70000FFA8CF21D4D02EB820E02EB4E029200F5
:104E800015441032134453F8042F0AB10A60111D5F
:104E90009D42F8D10023F6B20B6086F311882C23D3
:104EA00003FB0C00D0F85C3753B1E36843F0010317
:104EB000E36070BD242213FB0C220B4B9918D7E73B
:104EC000E36823F00103E36070BDE268054822EA6D
:104ED0000502E26000EB8302C2F83C17C2F84C679F
:104EE000B7E700BF80280024B82F0024D82F002463
:104EF00001490248FBF7E6BDB82F0024000001403D
:104F000002494FF08040FBF7DDBD00BFE42F0024D5
:104F100001490248FBF7D6BD1030002400040040D0
:104F200001490248FBF7CEBD3C3000240008004098
:104F300001490248FBF7C6BD68300024000C004060
:104F4000F8B5184D184ED5F81024D5F80C341A4081
:104F50004FF00040B2FA82F3F2B120FA03F3012AD3
:104F60006FEA030302EA0301C5F810340A46F1D1DF
:104F7000D6F868788FB1013F0023BFB2C6F8683811
:104F8000D6F8644834B123682046394698476468A7
:104F9000002CF8D10022DBE7F8BDD5F82C74BFB2A5
:104FA000EEE700BF001000408028002401490248BD
:104FB000FBF788BDEC300024000401402DE9F041EE
:104FC000134D4FF0000840F222264FF4B072A5F5C1
:104FD000A967A5F5F07400210E4856F059FB55F865
:104FE0002810002354F8332091420BD001330E2BAC
:104FF000F8D1002008F1070851F06AF9B045EED168
:10500000BDE8F08107EBC303B3F86C03F2E700BF20
:10501000B0C00908B82F0024F0B5144C83B094F840
:105020009D34002BFBD1D4F898580126104B6946CB
:1050300001AA28461F6984F89D64FBF711F99DF8C1
:105040000430009A03EB4303D4F89C481432DB008D
:1050500020469F5050F034FE2368314628463343A3
:10506000236003B0BDE8F040FDF75CB88028002461
:105070002017012437B590F85F380446032B2FD151
:105080000023204D8DF807309DF8073094F86028F4
:105090009A4201D803B030BD9DF8073005EBC30339
:1050A00093F8A4388BB181F0010383B19DF80730E8
:1050B00005EBC303D3F8A008FCF7B0FA9DF807305E
:1050C0000133DBB28DF80730DEE70B46EDE79DF8E4
:1050D000073005EBC303D3F8A008FCF791FBEDE71D
:1050E000D0E910039B7903F00103994204D003B087
:1050F000BDE83040FCF792BA03B0BDE83040FCF7A1
:105100007FBB00BF8028002438B5044600790D46D7
:1051100050B1FCF79DFA08B10323C380E279294618
:10512000BDE83840FDF7B0BB38BD10B504462221BC
:10513000FFF7EAFF02236279216803FA02F2D24301
:105140000A616079CA6883401343CB6010BD10B513
:1051500004460121FFF7D8FF022221686079CB685D
:10516000824023EA0203CB6010BD10B510F8133C57
:10517000A0F664041BBB94F850388BBBD4E9092318
:105180009A421CD05A1CA169A262CB5C21695B00C7
:105190008A4228BF002243F40073A262A4F8543864
:1051A0000A2384F85238012384F8503894F85F3881
:1051B000012B01D0042B02D1606CFFF7C8FF94F8DB
:1051C0004C38002B6FD194F84D380133DBB2092BEA
:1051D00084F84D3827D12046BDE81040FBF796BB38
:1051E00094F952387BB1B4F8541820464B0801F0BA
:1051F0000101A4F85438FFF73DFF94F85238013B01
:1052000084F85238DBE784F85038D4E909239A420D
:10521000D5D194F85F38012B01D0042BCFD1606C2D
:10522000FFF783FFCBE70A2B3DD194F84F382BB91A
:10523000B4F8563843F00103A4F856382379D90757
:105240000AD5B4F85608820501D4C30718D4B4F8B7
:105250005C380133A4F85C380122002384F84C2820
:1052600094F84F2884F84D38012A1CD16179606C7C
:1052700084F84F3801F00101BDE8104050F0DCB96E
:10528000E36AC0F3470013B1216B9847E4E7E36991
:105290006269D054E369E2680133B3FBF2F102FBC7
:1052A0001133E361D8E710BD2DE9F04110F8133C4C
:1052B000A0F664049BB9424E96F8E0781FB901212C
:1052C0002046FFF7D7FE94F85038002B3DD1D4E9A3
:1052D00009239A4219D1002386F8E03813E0B4F884
:1052E000583801339BB2082BA4F858380BD9002149
:1052F000606C84F85118A4F8581850F09DF994F88F
:105300005138002BD7D0BDE8F081022F12D807F119
:10531000010714BFFF237F2386F8E078A4F85438F0
:105320000823606C84F85238012384F85038BDE8B3
:10533000F0410CE75A1CA169A262CB5C2169DBB287
:105340008A42EBD30022A262E8E794F952386BB3A9
:10535000B4F8548896F8E15818F001010BD0012DEB
:1053600001D8012103E0AB1E012B09D80021204602
:10537000FFF780FE04E015F0FD03F2D0012BF6D01C
:105380000135EDB2032D86F8E158BCD994F85238B6
:105390004FEA58080022013BA4F8548886F8E12817
:1053A0005BB284F85238002B91D0ACE7D4E90912F3
:1053B0009142A8D1606C84F85038BDE8F041B4E661
:1053C00080280024F8B5BFF34F8FBFF36F8FCC4C0C
:1053D0000020CC49626A034622F480326262D4F82B
:1053E000942022F00102C4F894200246C4F89C00E4
:1053F000C4F8A000C4F898300133C4F89C20102BE6
:10540000C4F8A010F6D1BFF34F8FBFF36F8F052301
:10541000BD48BE4AC4F89430636A121ABC4943F4CA
:105420008033636256F0DCF8BA48BB4ABB49121AB3
:1054300056F0D6F8D4F88820B94B42F47002C4F87C
:105440008820D3F8002442F08042C3F80024D3F827
:105450000024002AFBDAD3F84C244FF0B044B148C2
:1054600042F00102B049B14DC3F84C24D4F868248D
:10547000AF4E22F00102C4F86824D3F80824AD4CE2
:1054800022F00302C3F80824D3F800241040AA4AEB
:10549000C3F80004D3F8C4040140A848C3F8C414F6
:1054A000D3F808142140A64CC3F80814D3F88C1480
:1054B0000A40A449C3F88C24D3F890242A40A24D72
:1054C000C3F89024D3F8942414400022C3F89444E1
:1054D000D3F8D0442040C3F8D004D3F8F0040140FE
:1054E0009A48C3F8F0144FF4E001C3F80C64C3F811
:1054F000CC149749C3F804044FF6FF70C3F88454E2
:10550000C3F88854C3F89824C3F88014C3F8D82487
:10551000C3F89C24C3F8A024C3F8A424D3F80044FF
:105520007F4944F48034C3F80044D1F80034013298
:105530009C0301D48242F8D1794BD3F80024900324
:1055400040F1DB80D3F84C244FF0B040814942F069
:105550000102814CC3F84C24D0F8682442F00102C7
:10556000C0F86824D3F808047C4A40F08000C3F8EF
:105570000804D3F8080440F08060C3F80804D3F8A6
:10558000080440F00050C3F80804D3F80804C3F836
:105590000804D3F8080440F48050C3F80804D3F892
:1055A00098040140C3F89814D3F8981441F00211FC
:1055B000C3F89814D3F804142140C3F80414D3F8A2
:1055C00004140A43C3F80424D3F8802422F07F0291
:1055D000C3F88024D3F8802442F00102C3F8802469
:1055E000D3F8802442F06072C3F88024D3F80024FA
:1055F00042F08072C3F80024D3F800249101FBD557
:10560000D3F80814464A21F00301C3F80814D3F86C
:10561000081441F00301C3F80814D2F8083403F069
:105620000C030C2BF9D14E4B354CA360BFF34F8FBD
:105630004C4800214C4A121A56F02AF84B484C4A62
:105640004C49121A55F0CCFFBFF34F8FBFF36F8F49
:10565000616A0023484A4FF0010C21F4803118465A
:105660006162D4F8941021F00101C4F89410C4F8D8
:105670009C30C4F8A03026E000293FD01568537A4A
:10568000103212F806EC1B0612F8057C12F8046CB6
:1056900043EA0E7312F803EC43EA8743C4F8980018
:1056A000C4F89C50013043EA4643032843EA0E43C2
:1056B00043EA4103C4F8A030D4F8A03043F001031A
:1056C000C4F8A0305AD05368117A002BD4D0156892
:1056D0000029D4D125F01F015B1A202B38BF2023CD
:1056E000B3FA83F6C6F11F010CFA01F7BB4288BF7B
:1056F000C6F120010139C9B2C1E7FEE7FEE700BFEC
:1057000000ED00E00800001000000000A0DE000036
:1057100048E80A08000000200400002003F80B08F5
:1057200000400258FFFFF2EAFEFFFFAF808088884A
:105730000000FF140C03C000CC3F007EFEFCFFFF06
:10574000C0EFFFC3888888FF2020010120200001CE
:1057500001010100F8FFFCFF0080800042250001EC
:1057600000000008E0160124201701240015012480
:10577000E016012407F80B0834070024BFF34F8F0D
:10578000BFF36F8F0523C4F89430636A43F480330A
:105790006362BFF34F8FBFF36F8F0022C4F85022B4
:1057A000BFF34F8FBFF36F8F636943F400336361BF
:1057B000BFF34F8FBFF36F8FC4F88420BFF34F8FB9
:1057C000D4F8805043F6E0760F48C5F34E34C5F365
:1057D000C905640104EA06012B4641EA8372013BD4
:1057E000C0F860225A1CF8D1203C14F1200FF1D1EE
:1057F000BFF34F8F436943F480334361BFF34F8F4F
:10580000BFF36F8FF8BD00BF00ED00E02DE9F04F52
:10581000012385B0DFF8ECA24FF000090193B44BEF
:105820000AF57F7BB34FA3F533780CE0019B09F1B8
:1058300001090AF1280A0BF1050B0133B9F1060F32
:10584000019300F0F2809AF80030022BEED19BF920
:105850000320561C00F0EC80D2B2944602EB4204C6
:10586000A34B5FFA89F14FF02C0E03EB84040F2A4F
:105870005ED8A14802E00330B84259D00378002B2B
:10588000F9D145788D42F6D18678D8F81050606805
:10589000A660A842267000F03781D8F83C50A84294
:1058A00000F05081D8F86850A84200F05581D8F82F
:1058B0009450A84200F05681D8F8C050A84200F099
:1058C0006181D8F8EC50A84200F07981D8F81851DD
:1058D000A84200F06D81D8F84451A84200F07B81C5
:1058E000D8F87051A84200F07081D8F89C319842E5
:1058F00000F09381D8F8C831984200F08081D8F840
:10590000F431984200F08281D8F82032984200F0B9
:105910009F81D8F84C32984200F0A181D8F87832B3
:10592000984200F0BF81D8F8A432984200F0AC81D0
:1059300001320C34D2B2624599D9002303939BF90A
:105940000420531C78D0D2B2964602EB4204684B36
:105950005FFA89F103EB84040F2A5DD8664802E000
:105960000330B84258D00378012BF9D145788D42E5
:10597000F6D18678D8F810506068A660A8422670E4
:105980005ED0D8F83C50A84200F0E280D8F86850C9
:10599000A84200F0ED80D8F89450854200F0ED80E8
:1059A000D8F8C050A84200F0F380D8F8EC50A842D4
:1059B00000F0F980D8F81851A84200F0EE80D8F82D
:1059C0004451A84200F01581D8F87051A84200F067
:1059D0000981D8F89C51A84200F03481D8F8C83128
:1059E000984200F02881D8F8F431984200F01C81E8
:1059F000D8F82032984200F03981D8F84C329842D9
:105A000000F03B81D8F87832984200F04481D8F811
:105A1000A432984200F04D8101320C34D2B2964546
:105A20009AD20023CAE9043300E705B0BDE8F08F3D
:105A30004FF00F0C002211E74FF00F0E002284E709
:105A400000239C4602932C2000FB0C8090F92C50E4
:105A5000002DE1D103750CF10104019B029A80F83D
:105A60002D30264B86611344CAF81430132380F876
:105A70002C302046FCF790F9039B002BD1D0DAF8AC
:105A800014603046FAF7C4FBDAF810000290FAF717
:105A9000BFFBDAF818300298DAF804101D70C268FB
:105AA00040201D615A600122186201F120009D61B1
:105AB000DA605A61DA619860C3E9095576B1DAF8BB
:105AC0001C3030311D70F0685A619D62C3E90101DC
:105AD000C3E90325C3E90652C3E90855002320465C
:105AE00007491A46FCF77AF901238AF80C309DE63B
:105AF00070060024FFBC09086CBC0908B003002430
:105B00009D010000682D00241846CDE902330EFBEC
:105B1000008595F92C0000287FF40AAF2B75019BB6
:105B2000039A85F82D30664B02981344AE6101301C
:105B3000CAF81030142385F82C30FCF72DF9012316
:105B40000393FCE601232C20CDE902301846DEE762
:105B50002C209C46029076E702235820CDE90230A3
:105B60001846D4E703238420CDE902301846CEE757
:105B7000022358209C46029065E7032384209C461C
:105B8000029060E70423B020CDE902301846BEE75A
:105B90000423B0209C46029055E706234FF48470FE
:105BA0009C4602904FE70523DC209C4602904AE782
:105BB00006234FF48470CDE902301846A7E7052389
:105BC000DC20CDE902301846A1E708204FF4B0757B
:105BD000CDE902059BE707234FF49A70CDE9023027
:105BE000184694E74FF4B0734FF0080C029300236B
:105BF00029E707234FF49A709C46029023E70A2076
:105C00004FF4DC750223CDE9020580E74FF4F2730F
:105C10000B2003930323029079E74FF4C673092006
:105C200003930123029072E74FF4F2734FF00B0CD1
:105C30000293032307E74FF4DC7002234FF00A0CB2
:105C4000029000E74FF4C6704FF0090C0290FAE69C
:105C50004FF404730C2003930423029057E74FF48E
:105C60000F730D2003930523029050E74FF4047344
:105C70004FF00C0C02930423E5E64FF40F734FF042
:105C80000D0C02930523DEE64FF425730F200393DA
:105C9000072302903BE74FF41A734FF00E0C029368
:105CA0000623D0E64FF41A730E20039306230290C6
:105CB0002DE74FF425734FF00F0C02930723C2E634
:105CC000B00300242DE9F04F4C484FF0010A4C4935
:105CD0004FF002094B4B4FF00408082710262025EF
:105CE00040244FF0800EDFF820C130F8022B12F074
:105CF000010F03D01960083323F804AC12F0020F2F
:105D000003D01960083323F8049C12F0040F03D069
:105D10001960083323F8048C12F0080F03D01960BF
:105D2000083323F8047C12F0100F03D019600833F5
:105D300023F8046C12F0200F03D01960083323F805
:105D4000045C12F0400F03D01960083323F8044CB0
:105D500012F0800F03D01960083323F804EC12F41A
:105D6000807F05D04FF4807B1960083323F804BC92
:105D700012F4007F05D04FF4007B1960083323F83C
:105D800004BC12F4806F05D04FF4806B19600833A7
:105D900023F804BC12F4006F05D04FF4006B1960B7
:105DA000083323F804BC12F4805F05D04FF4805B05
:105DB0001960083323F804BC12F4005F05D04FF4D7
:105DC000005B1960083323F804BC12F4804F05D03F
:105DD0004FF4804B1960083323F804BCD20B05D074
:105DE0004FF400421960083323F8042C01F5806158
:105DF00061457FF47AAFBDE8F08F00BF30BC090881
:105E000000000258182A00240018025810B4294C27
:105E100094F81C3E6BB3D4F8202E904236D0012B60
:105E200027D0D4F8382E824238D0022B21D0D4F893
:105E3000502E904234D0032B1BD0D4F8682E9042C1
:105E400030D0042B15D0D4F8802E90422CD0052BC6
:105E50000FD0D4F8982E904228D0062B09D0D4F831
:105E6000B02E904224D0072B03D0D4F8C82E824203
:105E700012D003EB4302591C04EBC20284F81C1E2F
:105E80005DF8044BC2F8200E184670470023DBB2C1
:105E90005DF8044B184670470723F8E70123F6E73F
:105EA0000223F4E70323F2E70423F0E70523EEE7F8
:105EB0000623ECE70400002010B4EFF31182102356
:105EC00083F312880A4B4FF0E0200024D2B2D3F8BB
:105ED0006C110131C3F86C118169C3F80419C3F85E
:105EE0000849036982F311885DF8044B704700BFCD
:105EF0008028002410B4EFF31181102383F312885B
:105F00004FF0E0229469136913F4803F0D4B03D0E6
:105F10000120C3F808099469D3F86C01C9B2D3F819
:105F2000082981F311880244D3F888114FF47A705C
:105F300000FB01F31B1B5DF8044BB3FBF1F300FB0B
:105F400002307047802800242DE9F0410746DFF831
:105F500048802C24FFF7CEFF42F20F76054604FB63
:105F6000078404E0FFF7C6FF401BB04207DC637EF6
:105F7000002BF7D1207E80F00100BDE8F081B8F859
:105F80000C39384601339BB2A8F80C39FCF7D4FD24
:105F90000020BDE8F08100BF8028002410B582B049
:105FA00004468DF807300DF107034FF023FF08B9C1
:105FB00002B010BD2046FFF7C7FF02B010BD00BF02
:105FC000B0F1FF3F00F0BE8003282DE9F04F0446FA
:105FD00083B015DC4FF02C0ADFF870911F460AFBE6
:105FE00000FA09EB0A03D3F804B0BBF1000F07D0A5
:105FF0008846597E1646019301F0FF02009219B1BE
:10600000002003B0BDE8F08F4FEA48080AF1200AEB
:10601000FFF770FF019B5FFA88F8009A012105469F
:106020000C9883F81A800BF11808DE765A77997766
:1060300049F80A00CA44CAF8040042F20F7A1F77EE
:1060400059761A7604E0FFF755FF401B50454ADCAD
:10605000D8F800301B04F6D40BF1040842F20F7A92
:1060600004E0FFF747FF401B50453CDCD8F8003008
:1060700013F48043F5D1DBF80020FF2E43F638718E
:1060800022F0F602CBF8002009EB8402CBF81C10BA
:1060900082F8B0300CBF0123002382F8B1304FF0FA
:1060A000010382F8B2302DD082F8B3302C22DBF815
:1060B000183002FB049943F00103CBF8183099F82B
:1060C0001A3043F49033BFF34F8FCBF80430BFF353
:1060D0004F8FBFF36F8FDBF8003043F0F203CBF844
:1060E000003001208DE72C230022204603FB04937F
:1060F0005A76B9F80C3901339BB2A9F80C39FCF780
:106100001BFD7DE7022382F8B3302C22DBF8183028
:1061100002FB049243F00103CBF81830927E0A4B45
:1061200042EA07421343BFF34F8FCBF80430BFF36B
:106130004F8FBFF36F8FDBF8003043F0B403CBF821
:106140000030CEE7002070470024000280280024A1
:106150002DE9F843DFF8908001F0CEFA204E0021BF
:106160000546D8F80070002F2FDD00231C4603EBF6
:106170000312013308EB0212BB4292F8052144EAF4
:106180000204F4D121435FFA81F97368C3F3080371
:10619000C3B9EFF31183ABB901F002FB401BB0F5BB
:1061A000FA6FCCBF002104F001010029DBD1B9F165
:1061B000000F04D00B4B93F87021542A08D04846A6
:1061C000BDE8F883FFF796FEE8E789460024DCE7A0
:1061D000B3F8782148460132A3F87821BDE8F88366
:1061E00000ED00E08028002404000020002070471B
:1061F00000207047034B93F82400003818BF01209B
:10620000704700BF00430024034B93F82400032889
:1062100094BF0020012070470043002400487047CD
:1062200028430024184B002030B49C7B14B11D6817
:106230008D4205D0013010330B28F6D130BC7047A9
:10624000C2B1124B03EB40218A4201D1022C18D07B
:106250000F4B93F8E42712B9012283F8E4270D4B82
:1062600001225A7000F5B170012203EB00139A71FC
:1062700030BC7047074B00F5B17003EB00139A7107
:10628000DCE7183BEEE700BFE8800024E86A002462
:10629000D07A0024D06A002430B400231C4C04F5CA
:1062A000C36084F8D03603E0013310300B2B15D0D7
:1062B00005688D42F8D190F80EC0BCF1030FF3D100
:1062C000C2B1144901EB4320824209D1A1F1180265
:1062D00003F5B173012102EB0312917130BC7047D9
:1062E00094F8E42712B9012284F8E4270A4A01212C
:1062F0005170EDE7D4F8CC1603F5B173064A0420CB
:10630000013102EB0313C4F8CC169871E6E700BF25
:10631000D07A0024E86A0024D06A0024A0B18368FF
:106320001BB10D4B07229A7070470B4A042110785D
:10633000137503289170C2E9033314BF4FF48073BF
:106340008023C2E901337047034A012302F58051DB
:10635000537081F8E4377047D06A0024704700BF5B
:106360002DE9F047002BDDF820A0884607460CBF3A
:106370004FF020094FF030095646002A144616F80F
:10638000011B23DD11B3334601E0002C05DD13F8BA
:10639000012B2546013C002AF7D1023D3CB149467C
:1063A0003846C047013DFAD29AF8001059B1384634
:1063B000C047334616F8011B0029F8D1A4EB0A04A4
:1063C0001819BDE8F0872046BDE8F087002C04F1DD
:1063D000FF35E4DC00240029E9D1F4E703685A1C06
:1063E00002601970704700BF10B56FF0004402469C
:1063F000044404E0B3EB0E0015D1A24214D012F80D
:10640000013BA3F14100192811F8010BA0F1410C47
:1064100098BF203300F1200EBCF1190FEAD91B1AE6
:1064200004D10028E9D110BD002010BD184610BDD0
:10643000884230B54FF001043AD301FB04F4B0FBBD
:10644000F4FC8C45F9D2BCB102BB06E0A14203F8D2
:10645000015B11D81446B0FBF2FCBCF1090F0CF142
:1064600057050CF1300E04FB1C00B4FBF1F2EDDC1F
:10647000A14203F801EBEDD900221A7030BDA14210
:1064800003F8015BF8D81446B0FBF2FCBCF1090F2D
:106490000CF137050CF1300E04FB1C00B4FBF1F2DB
:1064A000EDDCA14203F801EBEDD900221A7030BDFA
:1064B0008446002AEAD1D0E7002870B503DA2D23FC
:1064C000404201F8013B092886464FF0010307DDF1
:1064D00003EB83035B00B0FBF3F2092AF8D89BB10E
:1064E0000F4CA4FB030CBEFBF3F2092A4FEADC0CB1
:1064F00002F1570602F1300503FB12EE07DD092B0E
:1065000001F8016B6346ECD800230B7070BD092BBA
:1065100001F8015B6346E4D800230B7070BD00BF37
:10652000CDCCCCCC0378202B03D110F8013F202B0D
:10653000FBD0092BF9D02D2B00F0A9802B2B75D087
:10654000B7EE000AA3F13002D1B2092977D8F2EEF2
:10655000046ADFED5F7A07EE102A10F8013FB8EE0B
:10656000C77AA3F13002D1B2A7EEA67A0929F0EEDC
:10657000477AF0D92E2B66D003F0DF03452B40F08D
:10658000838010B442782D2A00F096802B2A00F0E8
:106590008380A2F130030130092B00F284800024B3
:1065A000002303EB830302EB430310F8012FA2F156
:1065B0003001303B0929F4D9B3F59A7F1A46B7EE7A
:1065C000007A28BF4FF49A72072B09D91346DFEDE2
:1065D000416A083B27EE267A072BFAD802F0070219
:1065E000DAB1F2EE046A012A27EE267A15D0022AE1
:1065F00027EE267A11D0032A27EE267A0DD0042A18
:1066000027EE267A09D0052A27EE267A05D027EE2E
:10661000267A062A18BF27EE267A002C45D0C7EE28
:10662000877A5DF8044B20EE270A70474378B7EE6F
:10663000000A0130A3F13002D1B2092987D92E2BEB
:10664000DFED237A98D143780130A3F13002D1B243
:10665000092991D8B2EE047AF0EE475A06EE902A54
:1066600010F8013FB8EEE66AA3F13002D1B2C6EEEF
:10667000076A092927EE257A77EEA67AEED903F084
:10668000DF03452B3FF47DAF20EE270A70474378A8
:10669000BFEE000A013055E782780230A2F13003E4
:1066A000092B7FF67CAFB7EE007A67EE877A5DF84C
:1066B000044B20EE270A704782780230A2F13003A3
:1066C000092B01D801246BE7B7EE007AA7E700BFDA
:1066D0000000000020BCBE4C032870B518D80E4B3B
:1066E000C943C60003EBC00001F0010190F86450FB
:1066F00090F8652081EA0504A24209D0026E22B119
:10670000A9421068928804D08261334483F86540BE
:1067100070BD8262F9E700BF004300242DE9F04F0D
:1067200001F1FF3985B0AF4C0746DFF8C8B2DFF89A
:10673000C882AD4DCDF80C904EF0B0F84FF4FA7A17
:10674000DFF8ACC24FF010094FF0E0223946DCF818
:106750000430C3F30803002B40F07081EFF3118382
:10676000002B40F06B812368966920688342FAD140
:1067700028688642F7D8DBF800704FF47A7000FB87
:1067800007FEAEEB0606B6FBF7F600FB03664FF41A
:106790007A77CDF804A0DCF80430C3F30803002BAB
:1067A00040F02C81EFF31183002B40F02781236808
:1067B000D2F818E020688342F9D128688645F6D8D7
:1067C000DBF800A0704607FB0AFEAEEB0000B0FB52
:1067D000FAF007FB03039B1BB3F57A7FDBD3DDF8ED
:1067E00004A0BAF1010AB2D1804B0F46D3F8882039
:1067F00093F88060D3F8843032B116F0020F11683C
:10680000908800F03D8188612BB1F607196898885F
:1068100000F18B828861BA46754E12B19188126878
:10682000D16213B19A881B68DA62704B1A46B3F8CA
:106830009030002B40F0C781134692F89820D3F88F
:106840009430002A40F0B88113B11A689B88936293
:10685000FA214FF0E022B94608467368C3F30803F3
:10686000002B40F06C81EFF31183002B40F0678127
:106870002368976921688B42FAD129688F42F7D83B
:10688000DBF800C04FF47A7101FB0CFEAEEB070E93
:10689000BEFBFCFE01FB03EE4FF47A7C0121CDE947
:1068A00001A07368C3F30803002B40F00881EFF3E5
:1068B0001183002B40F003812768906923689F4271
:1068C000FAD12B689842F7D8DBF800A00CFB0AF34A
:1068D0001B1AB3FBFAF30CFB0733A3EB0E03B3F560
:1068E0007A7FDED3DDE901A00138B6D13F4B4F46B8
:1068F000D3F8883013B19A881B68DA623B4BD3F81F
:10690000843013B19A881B68DA62384B1A46B3F8A0
:106910009030002B40F03681134692F89820D3F83F
:106920009430002A40F0418113B11A689B8893612A
:10693000FA214FF0E022B94608467368C3F3080312
:10694000002B40F0D980EFF31183002B40F0D4806E
:106950002368976921688B42FAD129688F42F7D85A
:10696000DBF800C04FF47A7101FB0CFEAEEB070EB2
:10697000BEFBFCFE01FB03EE4FF47A7C0121CDE966
:1069800001A07368C3F30803002B7BD1EFF31183DD
:10699000002B77D12768906923689F42FAD12B6832
:1069A0009842F7D8DBF800A00CFB0AF31B1AB3FBE4
:1069B000FAF30CFB0733A3EB0E03B3F57A7FE0D3B6
:1069C000DDE901A00138B8D10AF1FF3A4F465FFA7C
:1069D0008AFABAF1FF0F00F00C81044BD3E921329F
:1069E0001BE700BFEC29002484310024004300246D
:1069F00000ED00E0082A002488310024EFF3118321
:106A000089F31288D2F818E01069C00304D5012078
:106A1000C8F80000D2F818E02068DBB2D8F800A06F
:106A200083F311885044DBF800A007FB0AF3A3EBC3
:106A30000E03B3FBFAF307FB0033CCE6EFF3118050
:106A400089F31288D2F818E01369DE0304D5012314
:106A5000C8F80030D2F818E02668C0B2D8F8003084
:106A600080F311884FF47A70DBF80070334400FB38
:106A700007F6A6EB0E06B6FBF7F600FB036686E606
:106A80008862C1E6EFF31183102080F312889769C2
:106A90001069C00302D5C8F8001097692068DBB2FE
:106AA000D8F800A083F311885044DBF800A00CFB59
:106AB0000AF3DB1BB3FBFAF30CFB00337BE7EFF3CA
:106AC0001183102080F3128897691069C00302D5E2
:106AD000C8F8001097692068DBB2D8F800A083F3EB
:106AE00011885044DBF800A00CFB0AF3DB1BB3FB5E
:106AF000FAF30CFB0033F0E6EFF31181102383F37C
:106B00001288D2F818C01369DF0304D50123C8F82E
:106B10000030D2F818C02768C9B2D8F8003081F325
:106B200011884FF47A713B44DBF8007001FB07FEDB
:106B3000AEEB0C0EBEFBF7FE01FB03EE1CE7EFF322
:106B40001181102383F31288D2F818C01369DF0370
:106B500004D50123C8F80030D2F818C02768C9B29C
:106B6000D8F8003081F311884FF47A713B44DBF898
:106B7000007001FB07FEAEEB0C0EBEFBF7FE01FB47
:106B800003EE89E66A4AD2F8B030002B3FF4D0AE6B
:106B9000B2F8B430002B3FF4CBAE00231146D2F84C
:106BA0009C20136081F8AD30C2E6002B3FF4C0AEEC
:106BB0001A689B889362BBE6002B3FF449AE1A68C3
:106BC0009B88936144E65A48D0F8B030002B3FF4DC
:106BD0003FAEB0F8B41000293FF43AAE554BD0F8B0
:106BE0009C20B3FBF1F301210B41136080F8AD1041
:106BF0002EE64FF47A7ADFF840C14FF010094FF0DB
:106C0000E0223946DCF80430C3F30803002B6AD1D4
:106C1000EFF31183002B66D12368966920688342C5
:106C2000FAD128688642F7D8DBF800704FF47A7002
:106C300000FB07FEAEEB0606B6FBF7F600FB0366AD
:106C40004FF47A77CDF804A0DCF80430C3F30803DE
:106C50004BBBEFF3118333BB2368D2F818E02068F5
:106C60008342F9D128688645F6D8DBF800A0704643
:106C700007FB0AFEAEEB0000B0FBFAF007FB0303D4
:106C80009B1BB3F57A7FDFD3DDF804A0BAF1010ACC
:106C9000B8D1039B0F46013B039301337FF44CAD06
:106CA00005B0BDE8F08FEFF3118389F31288D2F8B5
:106CB00018E01069C00304D50120C8F80000D2F81C
:106CC00018E02068DBB2D8F800A083F311885044A4
:106CD000DBF800A007FB0AF3A3EB0E03B3FBFAF308
:106CE00007FB0033CCE7EFF3118089F31288D2F869
:106CF00018E01369DE0304D50123C8F80030D2F888
:106D000018E02668C0B2D8F8003080F311884FF43C
:106D10007A70DBF80070334400FB07F6A6EB0E0632
:106D2000B6FBF7F600FB03668AE7886273E500BFEF
:106D30000043002440420F0000ED00E02DE9F04741
:106D4000144CDFF85490DFF8548004F5407702E0EB
:106D50000834BC421CD094F90650002DF8D12668A6
:106D6000083406EB08039B0A39F813004FF0B0FA19
:106D700034F804AC012229465346304648F066F9FF
:106D800053462A462946304648F088F9BC42E2D1AB
:106D9000BDE8F087182A0024B0BE09080000FEA74D
:106DA00070B54BF039FA1B20FAF752FC08B12923D1
:106DB000C3801C20FAF74CFC08B12923C380234C64
:106DC00094F8BD30022B01D0012070BD94F8C4307E
:106DD000022BF9D11E4D0026D5E901122B68C4F80B
:106DE000EC60C4F8C8301B4BC4F8F060C4E933123F
:106DF00004F1C8021A60EB68C4F8D4302B69C4F8F7
:106E0000D8306B69C4F8DC30D5E90623C4F8E0203B
:106E1000C4F8E8304BF05EF90F4B05F150000F4A13
:106E200005F12001C4F8F5304FF48073C4F8002157
:106E3000A4F8F93084F8FB604DF0C6FA4BF0AEF9D7
:106E4000074B304683F8236070BD00BF0043002429
:106E500064070024102A00240210080000000440E7
:106E600000ED00E008B5FCF70BFC48B10F4A137EBB
:106E70000133DBB2072B137603D9002382F82430C9
:106E800008BD536D43B1186892F851109B88006992
:106E9000034041B1002BF0D1054B01211B6882F862
:106EA0002410536108BD002BE7D0F5E70043002410
:106EB000EC29002410B503791A4C002B14BF0123D0
:106EC000002384F8503009D0174B5B78003B18BF83
:106ED000012384F85C3051F093FB18B9002384F847
:106EE000243010BD636D83B1196894F851209B88DC
:106EF00009690B403AB943B9237E0022013384F873
:106F00002420237610BD002BF6D1FCF7B9FB002816
:106F1000F2D1064B012220761B6884F8242063619D
:106F200010BD00BF00430024642F0024EC2900247E
:106F300010B51D4C94F8C100FAF78AFB20B11F224E
:106F40002021C280FBF756FBD4F8843033B194F88B
:106F500080101A68C9079B8819D49361134B0021CC
:106F6000032093F90320FBF751FA70B1436863B132
:106F700051F046FB48B1636D6BB1196894F851202C
:106F80009B8809690B4022B12BB1012010BD93628F
:106F9000E4E7002BF9D0FCF773FB0028F5D1044B94
:106FA0001B68C4F8943510BD00430024642F0024EE
:106FB000EC2900240E4838B5436D0D4614463BB10C
:106FC000196890F851209B8809690B4052B15BB950
:106FD000FCF7A8F9074A4FF400730020926C2A606E
:106FE000236038BD002BF3D14FF0FF3038BD00BF18
:106FF00000430024082F002408B5FCF725FB98B1B6
:107000000B4B586D58B1026893F851308088126963
:1070100010402BB9003818BF0120013840B208BD1C
:10702000B0FA80F04009F8E74FF0FF3008BD00BF2C
:1070300000430024F8B5894C94F85060002E00F00D
:10704000C28094F824506B1E082B0ED8DFE803F0A2
:10705000AE056E0D2758400D1900FCF7F5FA002813
:1070600040F0B58094F824506B1EDBB2022B40F246
:10707000A180082D18BF042D0CBF01260026304624
:10708000F8BDFCF7E1FA002840F0D180744A63694A
:107090001268FA339342E5D2FFF7E4FED1E7714B71
:1070A0009F6A002F40F0BB80FCF7CEFA0028C8D0C2
:1070B0000423E568277684F82430002DDFD0236987
:1070C000384622686168A84794F824506B1ECCE7C4
:1070D000FCF7BAFA0028D9D0226A0023012A2376C5
:1070E00040F2A980E169013A0131C4E9071294F83C
:1070F0005C200AB1C4F89835082384F82430BEE730
:10710000584BDB6A002B5BD1554B0722E5681B68A7
:1071100084F824206361002D52D023690120D4E932
:107120000021A84794F824506B1E9EE7FCF7FAF85C
:1071300000283FD14C4B206293F82C10DA8D84F854
:107140002E10A285196B1A6B090E120C84F82F10E1
:1071500084F830201A6B196B120A84F8321093F8F5
:10716000341084F8312084F8331093F8351093F8F4
:107170003520090902F00F0284F8381084F839200C
:107180009A6BD88F6263DA8FD98FC2F30B1301F039
:107190000F02042143EA102384F83C2003F00F037C
:1071A00084F8241003F5FA6363874AE7022384F81E
:1071B000243046E72A4B62691B689B1AC82B23D8E8
:1071C00000263046F8BD304684F82460F8BDFCF750
:1071D000A9F800287FF446AF244B1B78002BA3F1BD
:1071E0000203B3FA83F308BF01255B096576A37632
:1071F000FCF798F800287FF44FAF1B4B03229B6CE1
:1072000084F82420A3621CE7FFF72CFE94F8246086
:10721000042E18BF082E0CBF012600262FE7104AA7
:107220006369126864339342FFF40BAF21E70423D0
:1072300084F8243023E7FAD194F85C2023620AB161
:10724000C4F89835FCF700FA0028F0D1044B092265
:107250001B6884F824206361B2E700BF0043002468
:10726000EC290024D42E0024082F0024A82900246F
:1072700070B5124C05460E4694F82430042B0ED0FF
:10728000082B19D1E36983420ED0002394F85C20C7
:1072900023620AB1C4F89835FCF7D6F930B1082357
:1072A000C4E9075684F82430022070BD044B09223B
:1072B0001B6884F824206361012070BD0043002412
:1072C000EC29002470B5134D10460A466C6D3CB194
:1072D0002668A1883469214095F85140A4B1A9B924
:1072E00001210D4CA1620021FCF756FB70B9A36A85
:1072F000002BFCD1FCF7A8F90028FBD0074B00209D
:107300001B68C5F8943570BD0029E9D14FF0FF30F6
:1073100070BD00BF00430024D42E0024EC290024BB
:107320002DE9F843224C05468946904694F82400FE
:107330001F46042811D0082802D00020BDE8F88399
:10734000002394F85C2023620AB1C4F89835FCF756
:107350007BF928B3042384F824300126154B4A46D0
:1073600028469E6200213346FCF716FB50B1FFF71A
:1073700079FDE568002DE0D00022236961681046A0
:10738000A847DAE70C4B05223046C4F800901B688A
:10739000656084F824206361C4E90387BDE8F8834D
:1073A000054B09221B6884F824206361C5E700BFF0
:1073B00000430024D42E0024EC29002470B5134D82
:1073C00010460A466C6D3CB12668A188346921409C
:1073D00095F85140A4B1A9B901210D4CE1620021F9
:1073E000FCF766FB70B9E36A002BFCD1FCF72CF9C3
:1073F0000028FBD0074B00201B68C5F8943570BDF2
:107400000029E9D14FF0FF3070BD00BF00430024D8
:10741000D42E0024EC2900242DE9F047394C1F46D6
:1074200005460E4694F824309046042B11D0082BC4
:107430003DD1E36983420CD0002394F85C202362A1
:107440000AB1C4F89835FCF7FFF850B3042384F868
:107450002430D4F89895C9F34F230F2BC4E9006565
:1074600028D8D4F820A0BAF1000F23D094F85C30CB
:1074700003B325484FF400723146484454F0B0F845
:1074800009F50073C3F34F22C4F898355B0A102A3C
:1074900002D0BAF1010F2AD19BB21B4E5A1EAD1A6F
:1074A00009E01A4B09221B6884F82420636101203B
:1074B000BDE8F0870123062128460125324684F8DD
:1074C00024101349C4F80C80CD6200212761257275
:1074D000FCF7EEFA0028EBD0FFF7C4FCE66826B113
:1074E0002369002261682846B0470320E0E7E2698B
:1074F0000AF1FF33042102200132236284F82410B0
:10750000E261D5E70043002424830024EC29002411
:10751000D42E0024092917D0B1FA81F35B0999B15F
:10752000013903604A0001F0030102F00802C1EBD7
:1075300001119300C1EB0111A3EB92038900C3EB8E
:10754000031381809B004380704700BFB5EEC00AE3
:10755000DFED357A0023F1EE10FA30B5C8BF30EE1A
:10756000270A87B0D8BF30EE670ADFED307A0546CC
:1075700003A9029320EE270ACDE90033FDEEC07A7D
:1075800017EE904A84EAE470A0EBE4704BF0D6FA70
:10759000002C03A8B4BF2D2320238DF8003051F018
:1075A00095F901282AD0022834D003281ED003A937
:1075B000684654F075F8684651F088F90446694603
:1075C0002846033CE4B2224654F00AF80023284639
:1075D0002B5551F07BF92E22431C0DEB04012A544C
:1075E000E81854F08AF8284607B030BD302303A9C4
:1075F00068468DF8013054F053F8DCE743F230026E
:10760000302303A96846ADF801208DF8033054F00B
:1076100047F8D0E743F2300303A96846ADF80130DC
:1076200054F03EF8C7E700BF6F12033A00007A44F7
:1076300008F07ABD38B5054658B14C1E14F8011F44
:10764000284619B9BDE8384008F082BD08F06CFD45
:10765000F4E738BD08B5202154F031F80346184648
:107660001BB102780133202AF9D008BD08B5CB0739
:1076700001D4FCF7FDFD08BD2DE9F3410023134DB6
:10768000044600EB810685F89C3505F29C55104FA9
:10769000B44203D10F4802B0BDE8F0813946284614
:1076A0004FF0000853F0FCFF2146684654F025F8DF
:1076B0002021684654F003F828B969462846043466
:1076C00053F0EEFFE4E780F80080F1E70043002488
:1076D000B6520A089C48002408B5CA24054B53201A
:1076E0000021FF225C625862D9655A6272B6FCF7CB
:1076F000ADFD00BF00400058244B5B68C3F3080396
:1077000010B4EBB9EFF31183D3B9214A4FF0E02C59
:10771000204C1368DCF8180011688B42F9D12168FD
:107720008842F6D81C4A4FF47A71146801FB04F2BF
:10773000101AB0FBF4F05DF8044B01FB0300704736
:10774000EFF31182102383F312884FF0E0239C693A
:10775000196911F4803F114902D0012008609C6929
:107760000B4BD2B218680B6882F311880A494FF4A8
:107770007A720344096802FB01F0001B5DF8044BB8
:10778000B0FBF1F002FB0300704700BF00ED00E02A
:10779000EC29002484310024082A002488310024A4
:1077A00010B40D4A4FF0E02C0C4C1368DCF81800B4
:1077B00011688B42F9D121688842F6D8084A4FF403
:1077C0007A71146801FB04F2121AB2FBF4F25DF84C
:1077D000044B01FB03207047EC2900248431002472
:1077E000082A0024494B5B68C3F308032DE9F04FD6
:1077F0000646002B66D1EFF31183002B62D1444B78
:107800004FF0E024434D1A68A06919688A42FAD102
:1078100029688842F7D8404F4FF47A713C6801FBE1
:1078200004F52D1AB5FBF4F501FB0255DFF8DC80F9
:107830004FF0100A4FF0E02CDFF8E0903548D8F810
:107840000420C2F30802DAB9EFF31182C2B91A6850
:10785000DCF8184019688A42F9D101688C42F6D8E0
:10786000D7F800E04FF47A7B0BFB0EF1091BB1FB5C
:10787000FEF10BFB0212521BB242E0D3BDE8F08FC7
:10788000EFF311828AF31288DCF81840DCF810104C
:10789000C90304D50121C9F80010DCF818401968A3
:1078A000D2B2D9F800E082F311884FF47A7B7144A8
:1078B000D7F800E00BFB0EF2121BB2FBFEF20BFB43
:1078C0000122D8E7EFF31181102383F312884FF0E0
:1078D000E0239C691A6912F4803F104A02D001200B
:1078E00010609C690A4BC9B21868126881F311884C
:1078F000094F02444FF47A71386801FB00F52D1BE3
:10790000B5FBF0F501FB025590E700BF00ED00E08C
:10791000EC29002484310024082A00248831002422
:107920000138424B4FF0E0212DE9F04F404F4FF02E
:107930001009DFF804810446DFF800E13D4A52688F
:10794000C2F30802002A5DD1EFF31182002A59D157
:107950001A688D6918688242FAD1DEF80000854203
:10796000F6D83E684FF47A70A24600FB06FCACEBFA
:10797000050CBCFBF6FC4FF47A7600FB02CC012030
:107980002C4A5268C2F30802F2B9EFF31182DAB955
:107990001A688C691D68AA42FAD1DEF80050AC4220
:1079A000F6D83D6806FB05FBABEB0404B4FBF5F42D
:1079B00006FB0242A2EB0C02B2F57A7FE0D3BAF1E9
:1079C0000104BBD2BDE8F08FEFF3118289F3128876
:1079D000D1F818B00C69E40303D5C8F80000D1F859
:1079E00018B01D68D2B2D8F8004082F311882C4438
:1079F0003D6806FB05F2A2EB0B02B2FBF5F206FBBB
:107A00000422D7E7EFF3118089F312888D690A69A0
:107A1000D60303D50122C8F800208D691E68C0B2C4
:107A2000D8F8002080F3118832449AE7EC2900242A
:107A3000082A002400ED00E088310024843100246D
:107A4000284C08B5D4F8C03594F8C605002B39D1B8
:107A500014200025FFF764FF234800BFD4F8C03589
:107A60005BB1196894F8C6259B8809690B4012B967
:107A70001BB1FFF731FE002BFBD00268D4F8943520
:107A8000D31A322B0EDCD4F8C835D31A002BE4DD20
:107A9000D4F8843013B199881B68D9623232C4F8A3
:107AA000C825DAE794F88030D4F8842003F0010385
:107AB0001AB1918812681BB99161C4F8C855CCE716
:107AC0009162FAE719689A880B69134020B1002B7C
:107AD000BED10B691340FAE7002BB9D00B691340F4
:107AE000FAE700BF00430024EC29002409F09CBE03
:107AF000094A536D73B11968988892F851300A6930
:107B000010401BB1B0FA80F040097047003818BF30
:107B1000012070470120704700430024034BD3F835
:107B2000CC0508B183691847704700BF00430024A3
:107B3000024BD3F8CC351B6A184700BF0043002422
:107B40000378022B12D00F4943680269D1F8480824
:107B5000023A184010B4400AD1F84048D1F83C1815
:107B600004FB02005DF8044B08447047054B426873
:107B7000D3F83418D3F8300800EB410000EB522062
:107B8000704700BFD07A00242DE9F04F9B4683B0A8
:107B900002F0020E8B4E10B9BEF1000F50D1D6F894
:107BA0003858002D37D14FF0FF3C874C0023874FCA
:107BB000E146E046CDF804C000922268A57B9042E1
:107BC0004AD015B303F5B17A012D07EB0A150DD193
:107BD000ED79EA070AD415F07E0F07D1ED0940F0E0
:107BE000A580A568A84584BFA846994601331034EE
:107BF0000B2BE2D1BCF1000F009A80F2C080019BF8
:107C0000002BC0F2A280019B2AE09C460133103475
:107C10000B2BD2D1EEE7D6F84048D6F83C3804FB1F
:107C200005339842BFD396F8E43713B9012386F899
:107C3000E437664B01225A70002003B0BDE8F08F94
:107C400096F8E437A6F58054002B7AD00123022061
:107C5000637003B0BDE8F08F009A002D40F0918072
:107C60005A4C41F21868D6F8C85603F5B17704EBC0
:107C7000031C01354CF8080041F21C68C6F8C856D0
:107C80004CF808504FEA071C44F80C5004EB071559
:107C90004FF0000CC5F804C004EB0715AD79042DB6
:107CA0004BD80FF2080C5CF825F000BFC17C04082B
:107CB000F17C0408397C0408F17C0408F77C040892
:107CC00012F001056CD104EB0710BBF1030F4FEA72
:107CD000E20C90F807806CF3C71880F807805DD934
:107CE0004FF6FF70584528BF584604EB0715A8808B
:107CF000BEF1000F2FD1500705D504EB0715E87929
:107D000040F00100E871D20608D504EB0717FA79B4
:107D1000C2F34500013060F34602FA712C4A01209B
:107D200002EB43220A6003B0BDE8F08F01930133F8
:107D300010340B2B7FF441AF5CE796F8E437002B4F
:107D400084D1012386F8E43780E7B9F1000FFFF60C
:107D500073AF4B4684E7D6F8C806D6F8CC56013048
:107D60000135C6F8C806C6F8CC5604EB031541F237
:107D70001C66A85104EB071004258571BBE7634618
:107D80006EE7D6F8C85603F5B177104C01354FEAC7
:107D9000071CC6F8C85644F80C507DE72846A4E7EF
:107DA0000B490C4A01EB43210B4BD3F8CC359D68B2
:107DB0000023A84700283FF43FAF04EB0717022336
:107DC000BB7139E7D07A0024E8800024D06A00240F
:107DD000E86A0024256204080043002470B5114EAF
:107DE00082B00D463378022B16D1020AC4B20E4B74
:107DF00001A9D3F83008002310440322FFF7C4FE82
:107E0000012807D13378019A022B0CBF22F81450B5
:107E100042F8245002B070BDC0F3D41200F07F04C9
:107E2000E5E700BFD06A0024D07A00242DE9F04FA6
:107E3000DFF820910D4685B0164699F800102B68A2
:107E4000032940D0022966D14FEA132A4FF4807BE0
:107E50005FFA83F8421E012A24D801249E421CD9CD
:107E600001283B4F8CBF002201220192D7F8A8279E
:107E70001AB1D7F8C417994250D0D7F83008002368
:107E8000092203A95044FFF77FFE012824D00228CD
:107E900015D020B12B689E42E8D803202E6005B093
:107EA000BDE8F08FB8F1000F14D0294B93F8E42708
:107EB00012B9012283F8E427012389F80130022056
:107EC00005B0BDE8F08F4FF0800BC3F3D41A03F078
:107ED0007F08BFE75C46C1E799F80010022916D079
:107EE0000329ECD1039B53F8282022F07042B2FA08
:107EF00082F2019BD5F800C052099A4220D0A044DA
:107F00000CEB0403D8452B601DD20229EAD1039B58
:107F100033F81820EBE74FF4807BD6E7D7F840180A
:107F2000013A02EB41224902B2FBF1F21344B3FBE6
:107F3000F4F204FB12320AB123449B1A2B60AAE725
:107F40006645ACD8A9E70AF1010A4FF00008A2E79C
:107F5000D07A0024D06A00242DE9F04FDFF8889110
:107F60008B4685B0174699F800C009F5805309681B
:107F7000BCF1020FD3F8305840F08280CEB24FF4FB
:107F8000807305EB1125A6EB010890449844B94293
:107F900008F1FF38B8FBF3F84AD200F00103A84417
:107FA0006FF0404A0193BCF1030F07EB0604A8EB06
:107FB0000503284614BF4FF480728022641A03A977
:107FC000944228BF1446944228BF002E14BF0122B9
:107FD00000220A32FFF7D8FD01282AD199F800C003
:107FE000DBF800E0BCF1020F0EF1010324D0B44233
:107FF00055D9039806EB0A02011F00EB820201EB40
:10800000840142F8043F8A4203F10103F9D1DBF80D
:108010000030A11B19448F42CBF8001002D1019B04
:10802000002B48D18F4205F101054FF00006BAD868
:10803000012005B0BDE8F08FB44246D903986FF037
:108040000042811E324401EB440100EB420222F85F
:10805000023F914203F10103F9D1A11B71448F4208
:10806000CBF80010DED1019B002BDBD086466FF0F1
:1080700000434FF6FF72012023442EF81320D8E767
:1080800001F07F06C1F3D413BCF1030FA6EB010886
:108090001D4414BF4FF480738023904476E7AEEB09
:1080A000060E0EEB04018F42CBF80010BAD1019BF3
:1080B000002BB7D003986FF040434FF0FF322344BA
:1080C00040F82320DBF80010ACE7AEEB060E0EEB19
:1080D00004018F42CBF80010A4D1019B002BA1D04A
:1080E000DDF80CE0C3E700BFD06A002430B50446D9
:1080F000C06983B010B9012003B030BD0D46002324
:10810000032201A9FFF740FD0128F5D1B4F9202091
:10811000002A19DB019B012D4FEA421103EB4212A9
:1081200003D0022D1BD1E5205854A368D3612378D6
:10813000032B04D10023137753779377D377636AA4
:10814000190C53839182D6E7064A92F8E41709B9CD
:1081500082F8E407044B012202205A70CCE7E3685E
:10816000E4E700BFD07A0024D06A00242DE9F04370
:10817000022383B004460F4694F83C20042A78D8A2
:10818000DFE802F02F036C5040003F4E4FF6F778C7
:10819000DFF8FC9006F5805518E0C4455CD84CF03B
:1081A000E3F801284FF00001034637D1206BFFF7B9
:1081B00015FE0128034631D10199D5F844084A1E1D
:1081C0002163824228BF0246C5F84428307801A9BD
:1081D000226B03281FFA82FC1046DED14A45DED905
:1081E0003AE07900204601F0FE01FFF77FFF012809
:1081F00003463ED1626B002A14BF0222012284F89A
:108200003C20B9E794F82830042B02D1002384F8ED
:108210002830A36B0BB1204698470123184603B0C2
:10822000BDE8F08319480021E26AD0F8C43700F5B0
:10823000F46042629B1AD0F8A02002FB03F382682C
:1082400002EB43228260C26802EB4322C260FFF766
:108250004DFF012803460CD10422D0E7626B04F1E4
:1082600030010020FFF778FE0128034601D10322E8
:10827000C5E7022BD2D194F82820042ACED10022BF
:1082800084F82820CAE700BFD06A0024D07A0024EE
:10829000F7FFFF0F38B5044694F83430052B60D84B
:1082A000DFE803F031251D130D0394F82830082B67
:1082B0003FD02D4B0122022083F8E52738BD94F8EA
:1082C0002830082B30D0012038BD00212046FFF790
:1082D0000DFF012845D1042084F83400DCE7D4E9FF
:1082E0000B01FFF77BFD01283BD10320F4E74FF0A2
:1082F000FF31206BFFF772FD012832D1E36A002BBA
:10830000F3D00220E8E7184D04F130010120D5F840
:1083100038280232FFF78AFD012813D00238C0B294
:1083200001281ED80520D7E70023012084F8283033
:10833000CAE700230122022084F828300A4B83F880
:10834000E527BBE7E368D5F84018226B03EB412330
:10835000C5F84428C4E90332E36A002BBCD1626249
:10836000BAE7002038BD00BFD07A0024F8B5044633
:10837000022094F83830032B07D8DFE803F02118E7
:108380000B0200212046FFF7B1FE431EDBB2012B9A
:1083900041D9F8BD0120626B04F13001FFF7DCFD2B
:1083A00001284FF00303F0D184F83830E1E70021D1
:1083B0001E48FFF79BFE01284FF00203F4D0E4E7CC
:1083C0001B4AE66802F580531278032AD3F8401856
:1083D000D3F8C45714BF4FF480728022256102FB8A
:1083E00001F1AF1A2A4406EB4126E660D3F8A867EC
:1083F000C3F8C427A6EB4126C3F8A867D3F8AC6737
:10840000A6EB4121C3F8AC17E36A2563626353B955
:1084100065620123C8E794F82830062BB9D1002300
:1084200084F82830F8BD2763F3E700BF708200248A
:10843000D06A00244368C3F308020A44B2F5007FFF
:108440002DE9F043054683B00C4605D223446B600A
:10845000012003B0BDE8F08390F91A20501C0AD027
:10846000444902F5B17201EB0212D17921F0010108
:10847000D171FF22AA7695F91B20511C0FD002F56D
:10848000B1723C48FF2600EB0210C279C2F34501ED
:10849000013921EAE17161F34602C271EE762A7870
:1084A000022AD3D0DFF8CC8008F58057D7F84028CF
:1084B000B4EB422F4FEA42292CDCD7F848681E4023
:1084C0007242A24226DCA21928694A4513D32A7EA9
:1084D00012072BD5D7F8C427411C8A421CD300D1E0
:1084E00000214B44A4EB0909686108469B1B09EB7A
:1084F000060429616B600028AAD098F80020032A9E
:1085000033D080B24FF6F7729042A1D81A46144485
:108510006C609DE700209CE797F8E4270ABB0123E5
:1085200087F8E43788F801306B68DAE701A94BF087
:108530001BFF0128EED16B68A4EB0904286999445C
:10854000297868613444A9EB0603019802291A4688
:108550006B602861CFD1D7F85018B3EB412FD6D339
:1085600076E7012288F80120BBE7034A90423FF6F4
:108570006FAFCBE7D06A0024F7FFFF0F2DE9F0477C
:10858000044682B094F83830032B00F2A680DFE86E
:1085900003F057170C020020236C84F8280003B165
:1085A0009847022002B0BDE8F0870022236C84F8CF
:1085B00028200BB120469847012002B0BDE8F08783
:1085C00023786668022B03D0454BD3F848381E4009
:1085D000C6F34F262046FFF7B3FA414F361A054639
:1085E000A7F58058B6B206EB050C022201A90023BC
:1085F00028461FFA8CF9FFF7C7FA01284FF40072DA
:108600004FF00001CED1019853F042F8E3694FF4E6
:10861000007120460BB16368EBB1D7F84038013BDD
:10862000994547D2FFF706FF01231D440028DAD100
:1086300097F8E4270AB987F8E43788F80130D2E7D9
:108640002046FFF727FE012802D0022845D103204B
:1086500084F8380096E7019B4FF020324FF0100E5F
:108660004FF02E0C42F62E6AC3F80120C3F8052005
:10867000A3F8092083F800C0D4F824C0A3F820A0F0
:1086800083F80BE0C3F82220C3F8262083F82A20C1
:10869000E26BA3F81AC02CFA0EFC5A8722FA0EF2EB
:1086A00083F82BE0A3F814C09A86D7F84038013B32
:1086B0009945B7D3C3EBC35320465902FFF7BAFE1F
:1086C00028B997F8E43723B1064B01225A700220EB
:1086D000BEE7012387F8E437F6E7002062E700BF32
:1086E000D07A0024D06A0024B1F904300F2B2DE990
:1086F000F0410E4682B00446174632D02046FFF7BE
:108700001FFA94F91B80B8F1FF3F3BD05C4B41F25C
:10871000186203EB08118A58904211D1183303EB09
:108720004825B388204601331BB205EB4315B380BF
:108730003D60FFF705FA3060012002B0BDE8F0812E
:1087400003F5805292F8E41700295CD001225A7098
:108750002378022B4CD02269002A60D100233B6091
:10876000EAE74FF40071FFF765FE002847D04FF6A7
:10877000FF732046B380FFF7E3F994F91B80B8F14B
:10878000FF3FC3D12378022B41D02269002AE5D0D4
:108790003B4B1B78032B69D093B24FF6F7718B429A
:1087A00094BF00230123002BD6D138B9354B93F861
:1087B000E427002A4DD0324B01225A7000231122A7
:1087C00001A9FFF7E1F9012810D1019D2E4BEB1A09
:1087D00048BF03F2FF13B3F5B05F4FEA63222DD217
:1087E0004FFA82F884F81B80002D9AD12378B0E7E5
:1087F000244A6368D2F85028B3EB422FAED200204F
:1088000002B0BDE8F081012182F8E4179EE71D4B1C
:10881000D3F850286368B3EB422FC6D39EE7184BBA
:108820001B78032B19D093B24FF6F772934294BF83
:1088300000230123002B91D10020E1E7114B93F895
:10884000E42712B9012283F8E4270D4B01225A7064
:10885000C8E7012283F8E427ADE70C4B9A4294BFA6
:1088600000230123002B7FF479AFE5E7074B9A4201
:1088700094BF00230123002B7FF46EAF95E700BF68
:10888000D06A0024D07A0024E86A0024F7FFFF0FA2
:1088900070B503780446017E023B012B02D911F02A
:1088A000060F5BD18D063BD494F91A30581C0AD0C0
:1088B000304A03F5B173FF2002EB0313DA7922F09B
:1088C0000102DA71A07694F91B305A1C0FD003F51F
:1088D000B173284800EB0310C379C3F34502013A92
:1088E00022EAE27262F34603FF22C371E2760B07CB
:1088F0000DD5214B93F8C827072A05D093F8E42714
:108900009AB31C4A01215170002283F8C827002322
:10891000E26A237084F82830FAB1BDE8704010474D
:1089200000231648E5691A018258954206D00133A2
:108930000B2BB9D01A0182589542F8D103F5B173C7
:108940000C4800EB0310C379C3F34502013A22EA55
:10895000E27262F34603C371A6E770BD0121FFF71F
:10896000C5FB0128F9D1217E9CE7012283F8E42789
:10897000C7E700BFD06A0024D07A0024E880002432
:1089800038B5184D014605F5805494F8100820B903
:1089900061B191F8283013B138BD002038BD4422B0
:1089A00004F5FD6052F01CFE012038BD44220E4843
:1089B00052F06EFE2B7803224FF6FF70022BD4F894
:1089C0004C1884F8002818BF13461022A4F8020897
:1089D0000548C4F80C1884F8E83784F801284EF0EC
:1089E000D9F8E1E7D06A0024B88200244FF0FF3CB8
:1089F000334A002333482DE9F041644603E0013354
:108A000010320B2B15D011780429F8D103F5B17170
:108A100000EB0111C979CE07F1D4651C52F80A1C8C
:108A200001D08C45EBD91C4601338C4610320B2B00
:108A3000E9D1002C02DA0120BDE8F081214D04F5D6
:108A4000B1772601DFF8888005EB07139988E9B92B
:108A5000D8F8CC25AB191C4ED2F8108041F2186220
:108A600006EB442198580023184AC047C0B1022899
:108A70000AD106F6E87605EB07150122D6F8CC36C2
:108A8000AA71013BC6F8CC360020D5E705EB0413EC
:108A900041F218629858D8F8CC35DB689847D7E788
:108AA00006F6E87605EB071503210122D6F8CC3649
:108AB000A971013B86F8D026C6F8CC36E4E700BFA2
:108AC000F6800024D06A0024E86A00249962040831
:108AD00000430024704700BF10B58C18A14215D088
:108AE00001F1FF3E013C41F2210C1EF8012F082349
:108AF00080EA022002B24000002A8CEA420180B2E1
:108B0000B8BF88B2013BF5D17445EED110BDF8B5C0
:108B1000164D6B78BE2B26D1AC1C154F0222294670
:108B20004FF6FF70FFF7D8FF22884AB1A618BE4261
:108B300019D2052A17D921463446FFF7CDFFF3E7AE
:108B400021460222FFF7C8FF0222A1180634FFF7D0
:108B5000C3FF084B641BA3F8D04541F60F53C31A5B
:108B600058425841F8BD0020FCE700BF0000020851
:108B700000000408004300240823484041B240009C
:108B80000029C0B2B8BF5040013BF7D1704700BFC9
:108B900030B5056804468D4218D901F1FF3E681EC4
:108BA00000231EF801CF082183EA0C034FFA83FC4F
:108BB0005B00BCF1000FDBB2B8BF53400139F5D107
:108BC0007045EED16A1C22602B7030BD00236A1CF8
:108BD00022602B7030BD00BF07EE901A9FED3B7AEC
:108BE0009FED3B3AF8EE677ADFED3A4ADFED3A3A2D
:108BF0009FED3A5A27EE800ADFED395A9FED396A28
:108C0000F7EE007A20EE070AB8FE404A30EE447ACA
:108C1000FDEEC46A16EE903A67EE076A03F00202B0
:108C2000DB07E6EE834AA6EEA35AE6EEA45AA6EECA
:108C3000856AE6EEA57A27EE067A39D5002A3ED077
:108C4000F1EE676AF0EE477AB0EE667AB7EE006A48
:108C5000DFED254AF6EE006A0023F8EE003AB0EEAA
:108C6000464A80ED096A76EE675A8361B0EE465A4D
:108C70004361A7EE244A036267EEA37AC361A7EEBD
:108C8000645A25EEA67AC6EE046A27EE267A65EEC9
:108C9000A65A67EEA67A65EE266A80ED007AC0EDE8
:108CA000015A80ED027AC0ED037AC0ED046A704784
:108CB000002ACBD0B1EE477AF1EE677AC6E734EE00
:108CC000404AB0EE677A64EE067ABFE7BD37863673
:108CD000762FA7BC00D8813E4AD99E3DA04B25BF28
:108CE000CEE99DBF8E0FC93FF304353FDFED197A02
:108CF00020EE270AF8FE407ABDEEE77A30EE670AEA
:108D000017EE103A60EE007A03F00202DB070DD591
:108D10009FED116ADFED116A9FED117AE7EE866A29
:108D2000A7EEA67A20EE070A82B170479FED0D6A82
:108D3000B7EE000ADFED0C6A9FED0C7AE7EE866A6B
:108D4000A7EEA67AA7EE870A002AEED0B1EE400A77
:108D5000704700BF83F9223F4AD99E3DA04B25BFF3
:108D60008E0FC93F762FA7BC00D8813ECEE99DBFAC
:108D7000B0EEC07AF0EEE06AF0EE407AC6FE875AB6
:108D8000F5EE405AF1EE10FA3BD086FEC75A85EE5A
:108D9000256A9FED1D2A9FED1D3A9FED1D4ADFEDCF
:108DA0001D4ADFED1D2AF7EE005ADFED1C3A9FED5C
:108DB0001C5AA6EE423AE6EE223AA6EE034AE6EE48
:108DC000235AE6EE044AA6EE245A85EE250AF4EE6E
:108DD000C76AF1EE10FA03D59FED127A37EE400A1A
:108DE000F5EEC00AF1EE10FA03D59FED0F7A37EEDB
:108DF000400AF5EEC07AF1EE10FA48BFB1EE400A33
:108E000070479FED070AE2E739094E3DE3B59E3E04
:108E100088FA163E45FE7F3F99FB243F69A2163E25
:108E2000A7DFA834DB0FC93FDB0F49402DE9F04F26
:108E3000884689B01E461178531C0393002900F020
:108E40001681002514460746A94609E03846013533
:108E5000C047039C621C21780392002900F08F8098
:108E60002529F3D16078A31C3028CDE9033923D01C
:108E7000A0F130034FF0000ADBB2092B26D96C2891
:108E80002AD078287FD8572878D9A0F15803202BEA
:108E900079D8DFE803F0BD787878787878787878D2
:108EA0007882AF787878787878787878AA787878CF
:108EB000789E788A7878BD00E31CA0784FF0010A8C
:108EC0000393A0F13003DBB2092BD8D804AA03A97D
:108ED00049F050FF6C28D4D1039B1A785C1C782A87
:108EE0000394B7D8572A40F28E80A2F15803202B62
:108EF000B0D801A151F823F02F900408558E040832
:108F0000558E0408558E0408558E0408558E0408A5
:108F1000558E0408558E0408558E0408558E040895
:108F2000558E04089D8F04084B900408558E040844
:108F3000558E0408558E0408558E0408558E040875
:108F4000558E0408558E0408558E0408558E040865
:108F5000ED8F0408558E0408558E0408558E0408BC
:108F6000558E0408D58F0408558E04085B900408BC
:108F7000558E0408558E04082F90040828B92846F9
:108F800009B0BDE8F08F039C64E72528FBD1039C62
:108F9000252138460135C0475CE7039C56F8041B81
:108FA00038460135C9B2C04754E70DF1140B002211
:108FB0000A2156F8040B5B46039CFDF739FA534629
:108FC000049A41463846CDF800B0FDF7C9F905448A
:108FD00040E7039C56F8040B0023049A4146009096
:108FE0003846FDF7BDF9054434E7039C56F8043BC9
:108FF0001D602FE70DF1140B56F8040B039C594626
:10900000FDF75AFADBE7002AB9D0252AC0D021E7BC
:10901000A0F158020DF1140B102156F8040BB2FA0E
:1090200082F25B465209FDF703FA039CC7E7A2F1FF
:1090300058020DF1140B102156F8040BB2FA82F20B
:109040005B465209FDF7F4F9B9E70DF1140B56F838
:10905000040B5946FDF730FAB1E70DF1140B00226D
:109060000A2156F8040B5B46FDF7E2F9A7E70D4627
:1090700085E7F8B5134C07460D461646D4F8D405D7
:10908000C0B11149FEF7D6FA3946D4F8D405FEF737
:10909000D1FA0E49D4F8D405FEF7CCFA0C49334680
:1090A0002A46D4F8D405FFF7C1FE0A49D4F8D405FE
:1090B000FEF7C0FA94F8D83513B1012384F8D935F6
:1090C000F8BD00BF00430024684D0A0838680A084C
:1090D00031760408754D0A080EB400B584B008490D
:1090E00005AB019001A853F8042B0393FFF79EFEF4
:1090F0000022019B1A7004B05DF804EB03B07047C6
:10910000DD630408F7B50023114E0C46154686F8BA
:10911000DA35104904EB45050F4B104F002818BFF6
:10912000194606F2DA5006F2DA5652F0B9FAAC42B3
:1091300002D10B4803B0F0BD394634F8022B684623
:10914000FFF7CAFF6946304652F0AAFAEFE700BFC0
:1091500000430024824D0A08794D0A088B4D0A0805
:10916000DA480024F7B50D4D0022044600EB410615
:1091700085F80B2605F20B65094FB44202D1094868
:1091800003B0F0BD394634F8022B6846FFF7A4FF60
:109190006946284652F084FAEFE700BF00430024F6
:1091A000586F0A080B49002403685A1C02601970A2
:1091B000090A03685A1C0260197070470268134656
:1091C000511C016013F802CB0360D31C517803607B
:1091D00093781B0443EA0123111D43EA0C03016049
:1091E000D07843EA00607047A0F13003092B07D91B
:1091F00020F02000413819288CBF00200120704742
:1092000001207047303809288CBF002001207047AA
:10921000413819288CBF0020012070476138192877
:109220008CBF00200120704720280BD0092809D0CE
:109230000A2807D00D2805D00B3801288CBF002044
:109240000120704701207047A0F14103192B98BFFE
:1092500020307047A0F16103192B98BF2038704768
:1092600002B3844610B5841803E0981A15D1A445BA
:1092700014D01CF8013BA3F14100192811F8010B8F
:10928000A0F1410E98BF203300F12002BEF1190F6A
:10929000EBD91B1A04D10028E9D110BD002010BD64
:1092A000184610BD1046704770B5044608460D4676
:1092B0004FF00CFB064602E014F8013F43B1324682
:1092C00029462046FFF7CCFF0028F5D1204670BD87
:1092D0001C46204670BD00BF2DE9F0430646864679
:1092E0009EF800C074460EF1010EBCF1200FF7D0BD
:1092F000BCF1090FF4D0BCF10A0FACF10B00EFD0B8
:10930000ACF10D05B5FA85F56D09002DE8D1012800
:10931000E6D9BCF12B0F3DD0BCF12D0F39D0102A6E
:109320003ED04FF0FF3E9046BEFBF2FE02FB0EF732
:10933000FF43FFB2002014F801CBBCF1390F4CF011
:109340002009ACF1300C0DD85FFA8CFC944510DA92
:109350007045264602D819D1674517D21D404FF0F7
:10936000FF30E8E7A9F1570CB9F1600F5FFA8CFC08
:10937000ECD801B10E6003F00103D5B9002803DA7F
:10938000002B18BF6FF00040BDE8F08300FB08C061
:10939000D1E70125102A94F801C004F10104C0D1DD
:1093A000BCF1300F10D06FF0704E0F274FF0100847
:1093B000C0E7B0F1004F04D91BB14FF00040BDE849
:1093C000F0834042BDE8F08360786FF0704E0F2765
:1093D0004FF01008A0F14106192E04F1010698BFC4
:1093E000203078280CBF02343446A3E701230A2238
:1093F000002171E770B50D461446FEF72BF90646BD
:10940000A0B1FFF7F3FF40F6340319229842A8BF3A
:109410001846B0F5617FB8BF4FF46170A0F5617375
:10942000B3FBF2F32B702378013323703046FEF741
:1094300011F90646A0B1FFF7D9FF40F6340319220F
:109440009842A8BF1846B0F5617FB8BF4FF461706D
:10945000A0F56173B3FBF2F36B70237801332370D3
:10946000304670BD03880021184AA3F5FA6C70B528
:1094700003F0030490F802E0154E40F2B5550EF1EA
:10948000FF3E04EB44044FEA9C0C0EEB8403C478CB
:1094900036F81330013C05FB0C3390F804C023442C
:1094A000847903EB430322444FF47A740CEBC30C2E
:1094B00043790089CCEB0C1C03EB8C03C3EB031347
:1094C00002EB8302C2FB040170BD00BF80436D3814
:1094D0003CC909082DE9F04116461F46404D044697
:1094E000394630464FF47A7200234FF04DFE3D4B23
:1094F00005443D4F3D4E83FB0510E9172844C1EB61
:10950000601183FB0103C8170B44C0EB631087FB9A
:10951000003CC317C3EBAC0386FB03764FEAE37E44
:10952000CEEBE61EC1EB0116A5EB860CC0EB0015D9
:109530004FEA8E0684F806C0A1EB8501617103EB4A
:109540004301A0EBC10040F2B55101FB1E33207175
:10955000B3F5896F33DA40F2DA218B4237DCB3F5A9
:10956000B77F234FB4BF4FF0000E4FF0010E0EEB4C
:109570004E0175464FEA4E0807EBC101C88A08EB59
:109580000E0C0B2107EBCC0C0CF1160C01E03CF897
:10959000020D984210DD0139F9D1F044012137F86C
:1095A000380006F5FA6E0133A17075441B1A22814A
:1095B0002580E370BDE8F0810131C9B2F1E70325F0
:1095C00040F296500A4F4FF00608AE46D7E7022504
:1095D00040F22940064F4FF00408AE46CFE700BFE7
:1095E00080BC92C789888888ABAAAA2A73B06D16F6
:1095F0003CC909080D4B10B553E9024354EA030274
:109600000AD10146002340F2011218460B80C1F82E
:1096100002208B710B8110BD054A1268121943F1AB
:109620000003FFF757FF012010BD00BF4049002491
:10963000EC2900242DE9F043044689B094F8303039
:10964000042B11D8DFE803F04B135C035500237E95
:109650009A0640F1E3800023112205A9E069FEF794
:1096600093FA012800F0DA8009B0BDE8F08301AE7A
:1096700004F11C07C74D324639462846FFF734F837
:10968000012800F0E4800228EED1C34A02F580559B
:1096900095F902385F1C0AD003F5B17302EB03138E
:1096A000D97921F00101D971FF2385F8023895F9A4
:1096B00003385E1C0FD003F5B17302EB0313DA79A4
:1096C000C2F34501013921EAE17161F34602FF214C
:1096D000DA7185F80318042384F83030AEE7AD481A
:1096E0004DF058FA4FF6FF720123228484F830308F
:1096F000A4E70020E36A207009B0BDE8F0431847F2
:10970000A64D95F81038002BAED104F11C0701AE20
:1097100005F5FD68324639464046FEF7E5FF01286B
:1097200040F0EC80DDF80490B9F1000F00F0C38048
:1097300099F800300BB1E52BECD1994AB9EB020254
:1097400048BF02F2FF12B2F5B05F4FEA622380F029
:1097500014811B01904A93490B44997B04290CD036
:10976000D5F8C8160131C5F8C81659600421997397
:10977000D5F8CC360133C5F8CC3695F90238581CEB
:109780000AD003F5B173FF2102EB031385F8021829
:10979000D97921F00101D97195F90338591C0FD0FD
:1097A00003F5B173FF2102EB0312D37985F8031897
:1097B000C3F34501013921EAE17161F34603D37135
:1097C00020220021484651F063FFD4F83120D4F81C
:1097D000353005A8C9F80020C9F8043094F83B30AA
:1097E000B4F8392089F80A30A9F80820637E89F88E
:1097F0000B30FFF7FFFEBDF81430002B40F008815E
:1098000044F281720321A9F81020A9F80E30A9F8BA
:109810001820A9F8163084F830100FE720464DF0D4
:10982000B9F92369002B70D0237E03F0F70213F0FF
:109830000403227676D1122A00F08B800022E36A9C
:10984000204684F8282009B0BDE8F0431847DDF829
:109850000480B8F1000F00F0A78098F80030002BCA
:1098600000F0A28098F80B9019F0080F7FF403AF76
:109870000B2204F13101404651F047FF00287FF4EC
:10988000FAAE637E89EA0303DF0640F1F880424ABC
:1098900002F5805595F902385E1C3FF408AF03F5D8
:1098A000B173FF2102EB031385F80218D97960F335
:1098B0000001D971FBE695F8E8370922022B3FF445
:1098C0000AAF95F81038002B7FF405AF85F82038E3
:1098D000C5F82438C5F8283885F81C38D5F8FC3781
:1098E0002C48C5F81438D5F8443885F81028C5F840
:1098F0001838FEF743FE01283FF40CAF02287FF42E
:10990000B3AE042384F8303098E6237E1B0795D548
:10991000224B93F8C827002A7FF4A6AE072283F8CB
:10992000C8278BE70023A5682046E66A294684F805
:109930002830FEF77FFD002840F09B8094F8283007
:10994000002B7FF491AE0223C4E90B6584F8283024
:109950008AE6E06A0421626AA063204684F83C300B
:1099600084F8281063636362C4E90B22C4E90233FC
:1099700009B0BDE8F0434DF00DB995F8E43713B9DF
:10998000012385F8E4370123034A53706FF00F0376
:10999000E1E600BFB8820024D06A0024D07A002417
:1099A000E86A0024E8800024554A02F5805595F9BC
:1099B0000238581C0AD003F5B17302EB0313D979AE
:1099C00021F00101D971FF2385F8023895F9033898
:1099D000591C0FD003F5B17302EB0313DA79C2F30C
:1099E0004501013921EAE17161F34602FF21DA7193
:1099F00085F80318237EDB067FF56DAE41484DF0F8
:109A0000C9F84FF6FF720223228484F8303015E63D
:109A10003D4B05A8B3F94056FFF724FD4FF47A7289
:109A200000234FF0B1FB3C2392B205FB03014FF43E
:109A30007A700023C1FB002302A8FFF74BFD9DF8BD
:109A40000A309DF80B209DF80E1042EA4312BDF833
:109A50000830A3F2BC7342EA43229DF80D305B014B
:109A600092B243EA51039DF80C1043EAC1239BB222
:109A7000C8E6002E3FF4F8AD204633463CE6B8F881
:109A80001420B8F81A30214D43EA0243D5F8402893
:109A900063625202D8F81C30B3FBF2F102FB1131C1
:109AA000A36009B113445B1AE36084F8199095F937
:109AB0000238134A581C0AD003F5B17302EB0313A2
:109AC000D97921F00101D971FF2385F8023895F980
:109AD0000338591C0FD003F5B17302EB0313DA7985
:109AE000C2F34501013921EAE17161F34602FF2128
:109AF000DA7185F80318032384F830309EE500BF3F
:109B0000D06A0024B882002400430024D07A0024C4
:109B10002DE9F04390F8283083B00446013B082B30
:109B20000BD8DFE803F0393D1F24052A0A2F340043
:109B30000121FEF71BFB012802D003B0BDE8F08332
:109B400000222378216C84F82820002BF5D00322F2
:109B5000E162D4E9010384F82820834238BF034638
:109B60002046A36003B0BDE8F043FEF791BE00219C
:109B700003B0BDE8F043FEF7F9BA03B0BDE8F04327
:109B8000FEF7F4BB03B0BDE8F043FEF783BB03B0C0
:109B9000BDE8F043FEF7F2BC03B0BDE8F04349E591
:109BA000524F4268D7F84858036B1540D7F8401811
:109BB00090F800E0E8184E02B0EB412F43D3A7F530
:109BC00080594FF6F778BEF1020F14D0216908468C
:109BD000002963D16068A3680021E26A834284F8A7
:109BE000281038BF0346A360002AA6D0204603B041
:109BF000BDE8F0431047D7F850186068B0EB412F2C
:109C000034D22069217E09073AD5D7F8C41700F16C
:109C1000010C614530D297F8E41700294FD1012398
:109C200087F8E43789F80130626894F800E0236B24
:109C30009B1B32442B44521B00259E4262602363CF
:109C4000C4E904C0BFD9BEF1020F0ED021690029BA
:109C5000C0D027480078032843D089B24FF6F77068
:109C60008142B7D898186060B5E76068D7F8501897
:109C7000B0EB412FF6D3AEE7DAD14FF0000CD7E7C7
:109C800001A94AF071FB01287FF457AF2069DDF884
:109C900004C094F800E06268236BC9E799F800C03B
:109CA000BCF1030F11D01FFA81FCC44594BF4FF0E3
:109CB000000C4FF0010CBCF1000FC8D1A2E701214C
:109CC00089F8011094F800E0B2E7DFF828C0614598
:109CD00094BF4FF0000C4FF0010CBCF1000FB6D157
:109CE00090E7044881423FF675AFBBE7D07A002485
:109CF000D06A0024F7FFFF0F2DE9F0410446154616
:109D000008469442B4FBF2F607D205FB1644134B07
:109D10001B5D00F8013BBDE8F0819642B6FBF2F70F
:109D20000CD20E4B05FB176705FB1644DA5D1B5D75
:109D300000F8012B00F8013BBDE8F081BA42B7FB07
:109D4000F2F807D905FB1878044B13F8082000F83F
:109D5000012BE7E74046FFF7CFFFF3E7D0700A0893
:109D600030B56F4C83B0B4F8703AB3F57A7F03D94D
:109D70004FF47A73A4F8703AB4F8723AB3F57A7F74
:109D800003D94FF47A73A4F8723AB4F8741AB1F59F
:109D90007A7F04D94FF47A731946A4F8743AB4F868
:109DA000760AB0F57A7F03D900231846A4F8763AEC
:109DB000B4F8783AB3F57A7F4CD94FF47A73B4F8A3
:109DC0007A2A9A42A4F8783A49D900238842A4F81A
:109DD0007A3A80F08F80B4F8862AB4F8883A9A42AA
:109DE00002D90023A4F8863A4E4B1B88EBB14E4DA6
:109DF000AA78062A52D9297900297ED19FED4B7A7B
:109E000094F8902A07EE903AAB7906EE902AF8EE95
:109E1000E77AB8EEE66AC6EE276A0BB137EE077A44
:109E2000B4EEE67AF1EE10FA46DC94F8992A032AA9
:109E300025D83F4B03EB421394F8982AC4F8A83A6C
:109E4000032A14D8EA213B4B02FB0133C4F8AC3A95
:109E500003B030BDB4F87A2AB2F57A7F18D88842B8
:109E600012D29A42B7D30023A4F8783AB3E700227B
:109E7000304B84F8982AC4F8AC3A03B030BD0022C5
:109E80002B4B84F8992AD7E70021A4F8741AE8E745
:109E900000228842A4F87A2AE3D3F5E7264901EBA9
:109EA000820191ED187A29790029A9D0531F032B3B
:109EB000BBD9002AB9D025E067EE877ABCEEE77AF5
:109EC0008DED017A9DF8043007EE103AB8EEC77AAE
:109ED000F4EEC77AF1EE10FA01DD0133DBB2EBB13B
:109EE000102BA8BF1023DBB2934238BF134684F86F
:109EF000903A9AE7A4F8743A6DE7053A032A94D9A0
:109F00009FED0A7AB7EE000A80EE070A50F0ACFB2C
:109F10002B88834228BF03462B8086E70123E2E794
:109F200000430024F80E0020902F00246F12033805
:109F300044490024C44900243CC909082DE9F04FD4
:109F4000AF4E83B096F8B03A00AFA3F11702022AE1
:109F500000F2D482AB4B7B6096F8C83A00243B6099
:109F6000A94B03F1840998461AE0BAF1140F4FD0B7
:109F7000584651F021FC1BF4003F40D0012847D047
:109F8000082845DC1DB1A14B1BEA030F04D1396839
:109F900058464DF011FBD8B308F10C08C84534D031
:109FA00098F904A050460DF0C5FB03281AD198F883
:109FB0000620D8F80000022A20F04100A8BF0222A3
:109FC000C8F8000098F8070088F80620022898F8DA
:109FD0000820A8BF0220022AA8BF022288F8070092
:109FE00088F80820D8F800B01BF00105BDD058460D
:109FF000013451F0E1FB1BF4003FE4B2BED1012873
:10A00000BEDC08F10C08C845CAD1013C022C03D9BA
:10A010007D497F4844F02EFF0023022086F87C3BD8
:10A020000DF03AFE96F8843BD6F8809B022B00F0A8
:10A030000A83002800F05683764B4FF47A7C96F81A
:10A04000E1AB002503F56A7E4FF0640B33F8082C72
:10A05000B2F57A7FB3F8462088BF23F808CCB2F572
:10A060007A7F33F8062C88BFA3F846C0B2F57A7F12
:10A0700033F8042C88BF23F806CCB2F57A7F02D9D6
:10A08000002223F8045C33F8061C9142B3F85A10FE
:10A09000B3F85C2098BF23F8065C914293F86B20DC
:10A0A00003F1650102F1FF3288BFA3F85A50632A19
:10A0B00093F86C2002F1010288BF83F86BB0D2B232
:10A0C000092A4FF0000288BF83F86C5013F8320061
:10A0D000013211F8014F844238BF0D70032AF5D1C7
:10A0E000BAF1010F03F1EA0318BF03F8645C9E455F
:10A0F000ACD1DFF834A19AF80230042B00F0C6820C
:10A100002BB9BAF80030B3F5F07F00F21582FFF7F3
:10A1100027FE414896F8F41BFDF7FCF9103096F83D
:10A12000131CFDF7F7F9103096F8231CFDF7F2F930
:10A13000B6F8322CB6F8303C1343B6F8342C13433F
:10A140001BB213B10123A6F8363C344B09EA0303D2
:10A15000002B00F0D48219F0010F40F08C8219F42A
:10A16000804F40F0EE8119F0080F00F058822C4A21
:10A17000D6F8D43B09EA02091340C6F8809BC6F81A
:10A18000D43B19F4004F00F02D82002386F8CF3A1B
:10A1900086F8DF3A19F4805F00F02F8296F8433C8E
:10A1A000022B02D1012386F8433CDFF878904B461E
:10A1B00009F1780402E006339C420CD01A780A2A8E
:10A1C000F9D19978DA78914202D35A79002AF2D0FB
:10A1D0000A201DF069FC00234FF4806086F87C3B68
:10A1E0000DF05AFD002800F06A820E4DAB469BF838
:10A1F000051031B39BF8000008B34B4619E000BFCF
:10A20000004300243CC90908F44D0024BC020200AC
:10A210007CC70B08CE490024044F002409600002CB
:10A22000FE9FFFFD484F0024902F002406339C42E0
:10A2300007D01A788A42F9D15A79002AF6D01DF04F
:10A2400033FC0BF1060B5C45D1D19AF80290B9F1C1
:10A25000080F00F0EA8196F8E13B96F86D2AA3F129
:10A260000103032AB3FA83F34FEA531386F8C03C81
:10A2700096F8E23BA3F10103B3FA83F34FEA5313D9
:10A2800086F8C63CD6F8D43BC3F3C03186F8C31C6D
:10A2900002D9002286F86D2AB949D6F8802B0B40E6
:10A2A0000A4096F8A61AC6F8D43BC6F8802BC1B966
:10A2B000B448DFF8F8B290F808C090F812E0B2495C
:10A2C0004CEA0E0E90F809C0C07C4EEA0C0C5CEA19
:10A2D000000018BF59460A431943C6F8802BC6F838
:10A2E000D41BB6F8DC3C002B40F0BB81D6F8E03C38
:10A2F000B3F5000F02D30023C6F8E03CD6F8E83CE3
:10A30000A24A1A401AB140F20223C6F8E83C96F875
:10A31000E43C013B042B02D9012386F8E43CA9F17B
:10A3200005099B4BB9F1030F93F8908540F25081DA
:10A33000B8F1000F1CD000233B60DFF8749206E0F8
:10A34000ABF1060BABEB0A0BD84540F2FC80CB46D9
:10A3500019F8010F0028F3D006F048FB0028EFD0D1
:10A3600081798B07ECD53B680122002B40F0F0800F
:10A370009AF8063013B100238AF80630B6F8F23C9A
:10A3800003F00F02042A03D8C3F30313022B03D9EB
:10A390004FF42063A6F8F23CB6F8F43C03F00F0249
:10A3A000042A03D8C3F30313022B03D940F6012375
:10A3B000A6F8F43C96F8651D96F8712D96F8643D64
:10A3C000914205D9002286F8652D53B1A6F8682D73
:10A3D00096F8702D9A4204D2002386F8643DA6F8C0
:10A3E000683D96F8662D96F85A3E9A4202D90023A7
:10A3F00086F8663DDFF8BCC10CF1800B63467968D6
:10A4000013F8032D02EB42020A4492F834A292F8A8
:10A41000359292F836E213F8010F99795045DA78BF
:10A42000A8BF50464945A8BF494672451870A8BF05
:10A43000724663459971DA70EDD103F1200CDC4569
:10A44000DCD1D6F8EC2A002A00F017810020012187
:10A4500002E00635AC420ED02B782B2BF9D16B786D
:10A46000043301FA03F31342F3D0063522EA030260
:10A470000120AC42F0D108B1C6F8EC2A454C6D463B
:10A4800004F10808234601E043456FD013F8012F7B
:10A49000072AF9D9002304F8013F0133082BFAD128
:10A4A000B6F8DA2BAD46B6F8D83B9A4202D33A4B0F
:10A4B000C6F8D83B394BFF22394C03F1840086F8AB
:10A4C0008C2E13F9082C142A05D053F80C1C34EAEE
:10A4D000010100F0D8800C338342F2D196F8BD30F0
:10A4E000012B04D0022B05D196F8C43013B90023F8
:10A4F00086F8BD300C37BD46BDE8F08F294A1146BD
:10A500007A60DA0001EBC30393F87C1021B1D3F831
:10A510008030002B00F0CF807B68134493F87D20BF
:10A52000002A3FF419AD93F85C31002B7FF414AD91
:10A53000182386F8B03A0FE54FF4F073AAF800300C
:10A54000E5E5194A14E63B680022002B3FF410AF02
:10A550009AF81130002B7FF411AF9AF80530012BD7
:10A560003FF406AF002A7FF403AF07E788B020224C
:10A57000FF21E946484651F08BF8064A21E000BF2A
:10A58000FDD77718D431002400040500FDFDFFFF3E
:10A59000F80E0020A22F0024AE014A01004E002434
:10A5A000010002003CC90908F6DFFFFD4004050078
:10A5B000972F002449490024424549F823303FF4AD
:10A5C0006FAF12F8013F59F823100131F4D061E761
:10A5D00000238AF80430B8F1000F00F08E800123C8
:10A5E0003B60AAE696F8CF3A002B75D0002319F409
:10A5F000805F86F8DF3A7FF4D1AD19F0800F3FF429
:10A60000CDAD96F8B02A182A04D8414BD340DA07CA
:10A610003FF5C4ADDFF8049109F17804DBE519F4E6
:10A62000005F3FF4AEAD3B4AA2E59AF80630002B3E
:10A630003FF411AE9AF81130012B7FF40CAE0223D7
:10A640008AF8113007E600283FF4F6AC90F9044090
:10A65000FF2500E0057220460DF00EFB0028F9D121
:10A66000EAE496F8D80C06F0C1F900287FF43EAE73
:10A67000A6F8DC0C3AE6284A7AE52B201DF014FAFD
:10A68000D6F8EC2AE2E686F88C2E27E7D6F8D43BFB
:10A6900029F4805923F48053C6F8809BC6F8D43B34
:10A6A000BAF82030B3F57A7FBFF431AD4FF47A7346
:10A6B000AAF820302BE5172386F8B03A2CE7D6F815
:10A6C000803B23F00063C6F8803BD6F8D43B23F0F0
:10A6D0000063C6F8D43B88E542F2010319EA030F90
:10A6E00084D157E5D6F8D43B29F0800923F08003C4
:10A6F000C6F8809BC6F8D43B9EE4424628E7D6F8CD
:10A70000D43B49F0080943F00803C6F8D43B2EE5D2
:10A7100000410001F6BFFFFDF79FFFFD484F0024F9
:10A720002DE9F04F844E83B096F8903E013B012B0B
:10A7300040F2EC80D6F8C02E804BDFF8208202F287
:10A74000DC524345C6F8C02E80F0F280DFF810924C
:10A7500001229B467A4D09F102070192B9F80210D5
:10A76000002900F0BD80052907EB010240F2B88006
:10A77000AA4280F0B580BBF800003C46C0F30B0055
:10A780000BE0118814460A44002900F0A980AA426F
:10A7900080F0A680052940F2A38061888142F0D133
:10A7A00061798B07EDD123885846DBF8081094F8BF
:10A7B00004A0009344F05EFBBBF80010BAEB113F1D
:10A7C00000F0948000230193BBF804100BF11C0BE4
:10A7D0005BF8140CC1F30B015BF8044C49F0FEF973
:10A7E000C3452060BAD3D6F8803B564CC6F8D43B5C
:10A7F000FFF7A4FB96F8983AEA22534D03FB024276
:10A80000A4F18003C6F8AC2A96F8992A03EB421308
:10A81000C6F8A83A1CF046FB4FF0FF33D6F8AC0A56
:10A820002B6620F0CBFB1DF085F904F2845304F273
:10A83000FC5102E00633994262D01A78002AF9D11D
:10A840009C78D878844202D358790028F2D096F8C0
:10A85000403CB6F8441C85F8642003EB8303642273
:10A8600003EB830302FB01F100229B006429C6F87D
:10A87000C02EC6F8C42EB8BF6421642BC6F8C82EFB
:10A88000B8BF6423C6F8BC1EC6F8D41EC6F8B83ECE
:10A890002E492F4BC6F8CC2EC1F83C37C6F8D02E27
:10A8A000A6F8D82E86F8DA2E26F042FF96F8DE1E9D
:10A8B000B6F8DC0E1DF020FF36F054FC18F0A8FDB1
:10A8C00096F8903E013B012B2AD9224B0122019898
:10A8D0001B6886F8D92EC6F8C03E03B0BDE8F08FDD
:10A8E000DBF80810584644F0C5FA6BE7009BA11D41
:10A8F00058469A1F44F0F4FA00287FF465AF61E7E8
:10A9000096F8A72A003A18BF0122A0E7FCF7F4FE48
:10A91000114B0222034486F8B02EC6F8AC3E09E77C
:10A92000FCF7EAFE0223C6F8AC0E86F8B03ECCE790
:10A930000123019357E700BF00430024F0C60B0832
:10A9400000000408C449002464070024F80E002015
:10A95000304F0024EC29002460E31600E4D00B08FB
:10A9600000000208114B0122032810B5044683F8A9
:10A97000442705D9601CBDE81040C0B20EF090B865
:10A980000B4BEA2203F2C46083F8984A04FB0200EE
:10A99000C3F8AC0A20F012FB1EF04EF91EF030FA9C
:10A9A000601CBDE81040C0B20EF07AB8F80E00206E
:10A9B00000430024054B0121D3F8E42E83F8E01E68
:10A9C00042F40012C3F8E42E704700BF0043002495
:10A9D000F8B5066805460F46C6F30B03EBB13F68B2
:10A9E00049F02CFF002838D11D4CE36843F00203E6
:10A9F000E360BFF36F8FBFF34F8F3760BFF36F8F8D
:10AA0000BFF34F8F49F01AFFE36823F00203E360BE
:10AA100018BB2B6804332B6021E0124A124B9A4278
:10AA200003D94AF0FBF84BF0FBF849F007FF88B96F
:10AA30000B4CE36843F00403E3606661E36843F0B2
:10AA40008003E36049F0FAFEE36823F00403E36067
:10AA50000028C4D04FF0FF3001E06FF00200F8BDD5
:10AA6000002000520000020800E01F082DE9F0411C
:10AA70005D4E8AB03378B12B76D1FEF748F880F07E
:10AA80000104E4B2594B04F00104594DB3F84332C8
:10AA9000584FADF80430BD4268D3002C00F0A180BF
:10AAA00000230596CDE907330993534B9B1B06936F
:10AAB000524BDA68D20704D5514A5A6002F1883203
:10AAC0005A6001224FF0000801A905A88DF8252041
:10AAD0004FF00042464D1A6102228DF824804CF05E
:10AAE000D1FF022201A94FF6FF70FDF7F5FF0446E2
:10AAF000BD424BD30025022202A905A8ADF808509B
:10AB00004CF0C0FF022202A92046FDF7E5FF40BA43
:10AB1000022203A9C043ADF80C0005A84CF0B2FF17
:10AB2000089888B107ABC0F104022946184450F0D8
:10AB3000AFFD9DF9240018B907A905A8FFF748FF44
:10AB400000238DF8240008939DF8253023B12B4A6B
:10AB5000D36843F00103D3609DF92400B0FA80F07C
:10AB600040090AB0BDE8F08101248BE7AB691C35D0
:10AB700035F8181CD3F8008055F8140CC1F30B01FC
:10AB800049F02CF8804518BF012484E7AE8803A95A
:10AB900005A88DF81180C6F30B061C35B31DADF862
:10ABA0000C3035F81C3CC3F30B021B0BADF80E2028
:10ABB00006228DF810304CF065FF062203A92046CE
:10ABC000FDF78AFF044655F8141C324605A84CF0E0
:10ABD00059FF204655F8141C3246FDF77DFF044608
:10ABE00086E70120BDE700BF000002083CC9090854
:10ABF000F0C60B08E4D00B08000004080020005247
:10AC00002301674570B5274CFFF798F994F8903EFB
:10AC1000013B012B34D9D4F8C03E01220325224E3A
:10AC200003F2DC5384F8E82EC4F8C03EFFF71EFFA1
:10AC300058B13378B12B08D1FDF769FF013D0AD037
:10AC400058B9FFF713FF0028F3D1013DEED149F0C9
:10AC5000E5FF4AF0E5FF0028F9D094F8903E002285
:10AC6000013B84F8E82E012B14D9104B012100225E
:10AC70001B6884F8D91E84F8E92EC4F8C03E70BD64
:10AC8000FCF73AFD0A4B0222034484F8B02EC4F8C4
:10AC9000AC3EC0E7FCF730FD0223C4F8AC0E84F8EC
:10ACA000B03EE2E70043002400000208EC29002443
:10ACB00060E3160010B5084A0124084B82F84447A7
:10ACC00083F8A64AFFF79EFFFFF72AFD2046BDE85E
:10ACD00010400DF0E5BE00BFF80E00200043002438
:10ACE00090F89230B7EE007ADFED6A6A014607EE1F
:10ACF000903A90F89630684AB0EE476A05EE103AFE
:10AD000090F89430F8EEE77A04EE903A90F89530A7
:10AD1000B8EEC55A05EE903A90F8983067EEA67AEC
:10AD200004EE103A25EE265AF8EEE44AF8EEE55A1B
:10AD3000B8EEC44A25EE275A64EEA64A65EEA65A36
:10AD400024EE264A64EE854A65EEA75A24EE274A89
:10AD5000B0EE473AF0B590F8917000F16F0602F14D
:10AD600018050024137807EE903AF8EEE77A67EEBC
:10AD7000857A67EE867AFDEEE77A17EE903AFA2B3F
:10AD8000A8BFFA2323EAE3730B72537807EE903AD5
:10AD9000F8EEE77A67EEA47A67EE867AFDEEE77A58
:10ADA00017EE903AFA2BA8BFFA2323EAE3734B720B
:10ADB000937803EE903AF8EEE33A63EEA57A67EE05
:10ADC000877AFDEEE77A17EE903AFA2BA8BFFA23BE
:10ADD00023EAE3738B72938807EE903AF8EEE77AF2
:10ADE00067EE847A67EE867AFDEEE77A17EE903AA0
:10ADF000D5ED007AB3F57A7FF8EEE77AA8BF4FF485
:10AE00007A7323EAE3738B812B68002B3FDD90F884
:10AE10009730B0EE436A02EE903AF8EEE22AA2EEE4
:10AE2000E66A63EE863A83EEA76AA2EEA66A65EE4C
:10AE3000A77A013467EE877A67EE867AFDEEE77AC5
:10AE400017EE903AFA2BA8BFFA23BC4223EAE37329
:10AE500006F8013F00DDF0BD012C13D190F89330CE
:10AE600007EE103A90F89B3006EE103AB8EEC77A2B
:10AE7000B8EEC66A27EE267A26EE266A0435083230
:10AE800008316FE7B7EE007AB0EE476AF6E7B7EE43
:10AE9000006ACCE70AD7233CA8CD090890F899307E
:10AEA0006BB3B0F864308BB190F89A20642102EB58
:10AEB0008203C3EB0313B3FBF1F3A0F864309623D2
:10AEC00012FB03F3B3FBF1F3A0F8663043884BB1F8
:10AED00090F89A30642203EB8303C3EB0313B3FBB4
:10AEE000F2F34380B0F850304BB1962290F89A308C
:10AEF00013FB02F36422B3FBF2F3A0F85030704767
:10AF000090F821304BB3438B83B190F82230FA2272
:10AF1000642113FB02F203EB8303B2FBF1F2B3F5FE
:10AF20007A7F4283A8BF4FF47A738383838843B1C7
:10AF3000FA2290F8223013FB02F36422B3FBF2F3FF
:10AF40008380C3884BB190F8223003EB8303B3F5C1
:10AF50007A7FA8BF4FF47A73C380704710B5064C50
:10AF60004FF48072002104F2D44050F091FB002392
:10AF7000C4F8D43510BD00BFF8530024034BD3F8F8
:10AF8000D80508B105F0E4B8704700BFF8530024B5
:10AF900008B50B4605490246D1F8D80528B1044941
:10AFA000FDF744FFBDE80840E8E708BDF85300247A
:10AFB00031760408024B0146D3F8D805FCF73ABBBA
:10AFC000F85300240048F5E77C500A080CB4C30687
:10AFD00007B500D561B905A904980191FFF7D8FF1D
:10AFE000FFF7F0FF012003B05DF804EB02B07047FB
:10AFF0000020F8E708B5FFF7DDFFBDE80840E1E70E
:10B0000010B504460348FFF7D5FF2046BDE81040C1
:10B01000F0E700BF954D0A08034B0146D3F8D80569
:10B0200008B105F081B87047F85300240CB407B597
:10B0300010F020000BD079B92320FFF7EDFF05A910
:10B0400004980191FFF7A4FFFFF7BCFF012003B0B4
:10B050005DF804EB02B070470020F8E70FB407B5C5
:10B0600004A951F8040B0191FFF792FF03B05DF8BA
:10B0700004EB04B0704730B52B4C85B02B48FFF77C
:10B0800099FF94F8C43023B9294805B0BDE8304091
:10B09000B0E7FCF72DFD08B92648F6E7FCF73EFDC2
:10B0A00008B92548F1E7D4F8CC35DB699847002882
:10B0B000F7D0FCF73DFD02680446037D8179520814
:10B0C000407CE51D0C34029020790190E0880090CE
:10B0D0001A48FFF7C3FF15F8010BFFF79DFFAC42BD
:10B0E000F9D1174C1748FFF765FF6378022B06D09C
:10B0F00007D9032B10D11448FFF75CFF0CE013486D
:10B10000FAE704F580541248FFF754FF94F8E43747
:10B11000022B05D0032B05D005B0BDE8304051E728
:10B120000C48E9E70C48E7E7004300249A4D0A0879
:10B13000A44D0A08B34D0A08C14D0A08D04D0A08AB
:10B14000D06A0024FE4D0A08044E0A080A4E0A0876
:10B15000174E0A081D4E0A08364E0A080FB407B5E6
:10B1600004A951F8040B0191FFF712FFFFF72AFF22
:10B1700003B05DF804EB04B070470EB403B503AA46
:10B1800052F8041B0192FDF774FF074BD3F8D83532
:10B190002BB9064B0649D3F8D405FCF74BFA02B09D
:10B1A0005DF804EB03B07047F8530024004300241B
:10B1B0007C500A080EB403B503AA52F8041B01928E
:10B1C000FDF757FF054B0649D3F8D405FCF732FAD3
:10B1D00002B05DF804EB03B0704700BF00430024E9
:10B1E0007C500A082DE9F04798460B7981460F46B6
:10B1F00003F0E0051646402D32D10024614DDFF802
:10B20000A081DFF8A89116E03B7903F00703013B2A
:10B21000042B04D8DFE803F014171A1D2100315D58
:10B220005848FFF71BFF7B79013BA34202DD4846EC
:10B23000FFF7C0FE01347B79A342E5DCBDE8F0876F
:10B2400031572846EDE736F81410FAE736F91410AE
:10B25000F7E756F824104046E3E756F82410F0E7E5
:10B2600003F00703052B56D8DFE803F0031E26285A
:10B270002B3D3478602D54D02BD8002D72D1B7F8E7
:10B280000550B7F8076021463E48FFF7E7FEAC429D
:10B2900038DBB44236DCB8F1000FCFD03246294655
:10B2A0003948BDE8F047D9E696F90040602D38D01E
:10B2B0000FD8002D56D14FE03488DBE7B6F90040B7
:10B2C000F4E7D6F800A0202D54464BD033D9602D9A
:10B2D00027D0802DB2D132782C4B2D48002A14BFB4
:10B2E0003146194634E0202D34683BD0EFD8214652
:10B2F0002448FFF7B3FED7F80510A14202DB4B420A
:10B30000A34220DDFFF75EFE23463A684846214906
:10B31000BDE8F04731E7202D23D01CD9602DD8D1CE
:10B3200000247B7944FA03F3DB07BDE8F0474CBF08
:10B3300019481A4892E651461948FFF78FFED7F888
:10B3400005108A45DED8B8F1000F3FF477AF1548F5
:10B35000BDE8F04782E60024B7F90550B7F9076069
:10B3600091E700247A79104B03EBC20393F89424FD
:10B37000A242C7DDD3F8903453F82400BDE8F0476B
:10B3800018E600BF596F0A089E520A083F690A086A
:10B390004E570A08504E0A08F04E0A0869700A080B
:10B3A000884E0A084A4E0A083CC90908484E0A084D
:10B3B000F0B5067906F0E003402B03D145794FF054
:10B3C000FF3406E0602B4FF00105F8D1447905FA0F
:10B3D00004F40023012006F00706AB4200D1F0BDC3
:10B3E000052E0FD8DFE806F00308101D242448B10D
:10B3F000C85CD75C78400FE020B1C856D756C71B51
:10B40000784278410133E8E70028FBD031F8130097
:10B4100032F81370784080B220420CBF0120002027
:10B42000F0E70028EED031F9130032F91370E6E7A7
:10B430000028E7D051F8230052F82370DAE708B566
:10B44000034610460AB9002008BDDB0601D50029D5
:10B45000FAD0FFF7D5FDF6E7F8B50D4E054696F89C
:10B46000DC3593B9F8BD25B12388C3F30B039D42A6
:10B4700004D0A288D4E9020150F0B2F81C34BC42D6
:10B48000F1D3002386F8DC35ECE7024C024FF6E7F7
:10B49000F8530024F0C60B08E4D00B08037903F03E
:10B4A0001803102B1ED003D833B9B0F80B00704727
:10B4B000182BFAD000207047124BB0F80B0093F90C
:10B4C0000031591C0CD1104B93F8983A03EB43020E
:10B4D00003EB820303EBC30300EB430080B270472E
:10B4E000DBB2F3E7074BB0F80B0093F901315A1CBC
:10B4F00005D1054B93F8993A00EB4310EEE7DBB228
:10B50000FAE700BF640700240043002470B5054635
:10B51000B0F8090043F098FC064B0446284693F81F
:10B52000DC65FFF7BBFF16B1E368184470BDA36884
:10B53000FBE700BFF85300242DE9F04F164685B015
:10B54000334C1A464FF00009A246CDE90101002113
:10B550003046FFF774FF06F0100300900393FFF7E7
:10B560000DFD2379029A03F01803934203D0002AB9
:10B5700044D1182B42D14FF00D0B0BFB09A3B3F8AC
:10B58000090043F061FC80462046FFF787FF07462D
:10B59000D8E90221024401442046FFF709FF80F068
:10B5A00001010546009AC9B23046FFF748FF039BE8
:10B5B000009003B115BB0BFB09FBB3065AF80BB0A7
:10B5C0000ED56DB959461348FFF748FDD8F8082045
:10B5D0002B4621463A440198FFF704FEFFF7F2FCA0
:10B5E00059460D48FFF73AFDD8F80C2000232146B4
:10B5F0003A440198FFF7F6FDFFF7E4FC09F1010971
:10B6000040F28B230D349945A9D105B0BDE8F08FE8
:10B6100014DF09086A4E0A086B4E0A0870B5164610
:10B6200005460C460846FFF771FF334602462146A1
:10B630002846BDE87040D5E52DE9F041037903F0D7
:10B64000E002402A4AD009D82ABB03F00703052BA1
:10B650001CD8DFE803F0161B161B090F602A44D024
:10B66000802A3ED0BDE8F081D0F805102148BDE821
:10B67000F04173E5D0F8052051421F48BDE8F04184
:10B680006CE5B0F80720B0F80510F6E7B0F9072030
:10B69000B0F90510F1E746790024184D184805EB7C
:10B6A000C605FFF787FC012395F89474A74202D8DA
:10B6B000BDE8F04186E4D5F890644FEA840856F876
:10B6C00024204AB113B90F48FFF774FC56F808104C
:10B6D0000D48FFF7C3FC00230134E7E741790B482D
:10B6E000C5E7827941790A48C8E70A48BDE8F041D0
:10B6F00034E500BF754E0A088B4E0A083CC909089C
:10B70000A24E0A089F5A0A084E570A08B34E0A0862
:10B71000C44E0A08DB4E0A0838B505460C46FFF74A
:10B72000F5FE2A7902F0070302F0E002602A29D12F
:10B73000052B0CD8DFE803F0030B0F0B1B1B6A79FA
:10B74000012393400278DBB214B11343037038BD78
:10B7500022EA0303FAE76A790123934002889BB245
:10B7600014B113430380F2E722EA0303FAE76B798B
:10B7700001229A40036814B113430360E7E723EA08
:10B780000203FAE7052BE2D8DFE803F0030305051F
:10B7900007070470DBE70480D9E70460D7E70149B5
:10B7A00008E500BFF34E0A08004903E5024F0A0806
:10B7B00007B5009313460A460249FFF7FBFC03B0A6
:10B7C0005DF804FB194F0A0820B10078B0FA80F048
:10B7D00040097047012070472DE9F74F8146084620
:10B7E000FFF7F2FF0E46054670B1002401A920467E
:10B7F000013447F0A3F901464846FFF7EDFF122C4C
:10B80000F4D103B0BDE8F08F0846FDF7EFFDC4B2F8
:10B81000112C6ED83B4D701CFBF71CFF3A4E05EB0C
:10B8200044088346670098F8E0A5B0B9AAF1020180
:10B830004B424B413D4495F8E025B25C002B52D081
:10B8400095F8E135192040F2EE2100FB0313214663
:10B850002E4803B0BDE8F04F80E4017830464FF049
:10B860002EFF80B1032C2A49A0EB060394BF0022CF
:10B87000012202EB42020A4452FA83F393F860A6D3
:10B88000BAF1030F04D1484603B0BDE8F04F86E794
:10B890005846FBF7DFFEF0B1BAF1020FF3D1FDF726
:10B8A000A5FD40F6CA0380B29842A8BF184640F2F0
:10B8B000EE239842B8BF18461923A0F2EE20B0FB41
:10B8C000F3F088F8E105AAF1020253425341EA1964
:10B8D00082F8E0A5AEE7BAF1020FF4D1484603B012
:10B8E000BDE8F04F60E721460A4803B0BDE8F04FDD
:10B8F00034E411232A460849484603B0BDE8F04F16
:10B9000056E700BFF8530024747E0A08324F0A0835
:10B910003CC90908424F0A084F4F0A082DE9F04F69
:10B920000346A1B00846FFF74FFF054620B1184671
:10B9300021B0BDE8F04F37E7FF23DFF8C09207469C
:10B940004FF0FF388DF82830D9F804360B9093F873
:10B950003820ADF830000D908DF838200F90ADF8FC
:10B96000400011930991CDE90500934909A84FF0D2
:10B9700045FE044618BB01460AAC904F0B019048A7
:10B980001A57002310F9016BB24240F0D2804E1CCE
:10B99000104647F0BBF8024631463846FFF7DEFB5B
:10B9A000022E4FF00101E9D19DF938A09DF9283010
:10B9B000534540F0C5808348FFF7D0FB4DE0237826
:10B9C000002BD2D0032FD4BF00260126062F00F271
:10B9D000A980DFE807F00447509104475000042F86
:10B9E00010D079492046FDF75FFC58B14FF48060D4
:10B9F0000CF070F9002800F0B48190F904000123E4
:10BA000006930AE071492046FAF7EEFC70B9D9F8BE
:10BA1000043693F93800042F22D0119B119320ABE8
:10BA200003EB061606F8580C01379EE7204646F051
:10BA300067FF0028EFDA01230A2212A92046FDF74A
:10BA40004BFC40B2002803DB129B1B78002BE2D09A
:10BA50002246711C5E48FFF781FB21B0BDE8F08FE4
:10BA60000023DBE72046FDF7C1FC20AB03EB061605
:10BA700046F8540CD8E757492046FDF715FCB0F1BD
:10BA8000000A5549204618BF4FF0010AFDF70CFC8B
:10BA900008B14AF0020A3301DFF864C1079320AB12
:10BAA00003EB0616BCE80F0006F850AC12AE0DF121
:10BAB000480A0FC6BCE80F000FC6BCE80F000FC64F
:10BAC0009CE8030086E803000026B346DAF800107D
:10BAD00020464FF04BFE10B19AF804301E430BF194
:10BAE000010B0AF1080ABBF1070FEFD1079B803366
:10BAF0006B4403F84F6C97E738492046FAF774FC1B
:10BB0000A0B137492046FAF76FFC00288CD02046B8
:10BB1000FDF76CFC0328804686D901463148FFF7C3
:10BB20001DFB9AE7224608212F4894E7012305933D
:10BB30007AE701330B2B7FF425AF01312B488AE7DD
:10BB40000B9B1BB9AAF114025542554100235F1CFF
:10BB5000E368002B61D194F900B058460CF08CF8E2
:10BB6000D4F8049018B10668002E40F08A80B9F12C
:10BB7000000F237A14BF4E464FF46146666023B926
:10BB80001B48FFF7EBFA03232372627A2AB1394686
:10BB900018480792FFF7E2FA079A02925846237A6A
:10BBA000CDE9006300231A4619460CF0ADF8E060B9
:10BBB00040BB39461048B2E7B6520A08D94F0A08C6
:10BBC00081CB0908F64F0A08724F0A087D4F0A0810
:10BBD000814F0A089C4F0A088C670A089F4F0A0881
:10BBE000D6610A08A54F0A08BD4F0A08E44F0A08A3
:10BBF0000F500A082A500A0845500A08F853002432
:10BC0000A4CF090858493346584A5948B9F1000F9A
:10BC100018BF0A463946FFF721FA022F04F1100433
:10BC20004FF0010393D1119E0D9F4DB15148FFF785
:10BC3000E1F933681B6A1BB13A464F4930469847D1
:10BC4000059B002B50D04D49474BBAF1140F18BF3C
:10BC500019464B48FFF782FABAF1140F09D1059B38
:10BC6000002B43D03368DB691BB1002245493046C5
:10BC70009847069B002B43D100223146384646F0B8
:10BC800057FEE660B9F1000F2CD04946304601F06E
:10BC9000C1FE3D4AB36839463C48FFF75FFA94F865
:10BCA0000890B9F1000F0CD03279914509D04B467C
:10BCB00039463748FFF752FA3368494630469B69A0
:10BCC0009847637A23B1727939463248FFF746FACA
:10BCD000F36A002BA1D039462F48FFF73FFA002323
:10BCE000F3629AE7204AD5E71F49B2E7B8F1000F9F
:10BCF000BFDB3368DB69002BBBD042462749B6E780
:10BD0000DFF89C900025DFF89CA04FF0030B04F0B7
:10BD1000AFFC0520FBF704FE9AF89035AB42ABD997
:10BD200019F8014FC4B1204604F060FE804698B176
:10BD30002046F5F78DFC0446EBB210B180F806B052
:10BD4000C37120460121F6F77DFC98F806302046A5
:10BD5000DB0703D5F5F754FD0135DDE7F5F75EFCAC
:10BD6000FAE74FF0FF304AE67E500A08574F0A08BC
:10BD700061500A0817510A0815DA0408654F0A08C5
:10BD800040510A086D760408604F0A087F500A087F
:10BD9000A4500A08C7500A08FE500A08D9660408C9
:10BDA000972F0024F80E00202DE9F04F914687B020
:10BDB0000C461A46002180464D46FFF740FB0027FF
:10BDC0000646B9F1000F63D02946062220464FF0FF
:10BDD000E3FC00283246404613BF012100214FF00A
:10BDE000010A4FF0000AFFF72AFB0646287817F0F1
:10BDF0009BFA8346F8B1687917F096FA4FF46171AF
:10BE00004FF0190CAB78EA789BF805E01CFB0313A4
:10BE10001CFB021295F801B0297900B14079CDE9F7
:10BE20000410CDE9023251463B461A4A4046CDE95C
:10BE300000EBFFF7FBF8207817F076FA8346F8B1AD
:10BE4000607917F071FA4FF461714FF0190CA37813
:10BE5000E2789BF805E01CFB03131CFB021294F82C
:10BE600001B0217900B14079CDE90410CDE9023269
:10BE700051463B46074A4046CDE900EBFFF7A6F89E
:10BE8000013706340635142F9BD107B0BDE8F08F7B
:10BE9000CA46D0E763510A082DE9F041054686B04D
:10BEA00008460F46FFF790FC064638B100235B4971
:10BEB00001201A4606B0BDE8F04175E70846FDF7D7
:10BEC00095FA1328044600F3A08006258DF8176024
:10BED000534E4543781CFBF7BDFB074660B1FDF7A9
:10BEE00085FAC0B217F03AFA30B17319027983F8C3
:10BEF000482C01238DF817303846FBF7ABFB07467B
:10BF000068B1FDF773FA0D2809D8062303FB046313
:10BF100083F8490C9DF8173001338DF81730DFF89E
:10BF2000FC80A91C0DF1170238464144FDF762FA66
:10BF3000FBF790FB074668B1FDF758FA012809D8CE
:10BF40009DF817300622013302FB04628DF817308A
:10BF500082F84C0C3846FBF77DFB80B1FDF746FAC2
:10BF6000C0B217F0FBF950B19DF8173006220179E5
:10BF700002FB0462013382F84D1C8DF817309DF8E6
:10BF800017200623042A2FD103FB04630022A3F801
:10BF90004C2C06251BF0CEFD05FB046595F8480CDE
:10BFA00017F0C2F995F84B1C95F84A7C19234FF409
:10BFB0006172804695F84D0C13FB012613FB072791
:10BFC00017F0B2F94379214698F80520039395F8C4
:10BFD0004C3C14480097CDE9016395F8493CFFF7C4
:10BFE000BDF806B0BDE8F081052A05D103FB046366
:10BFF000002283F84D2CCCE7062ACAD0002308EB98
:10C00000050248F805309380C3E7132332460649FA
:10C01000284606B0BDE8F041FFF7CABB484F0024F0
:10C020000043002463510A087C510A082DE9F04FAF
:10C03000904689B01A460C46002181464546FFF7D6
:10C04000FEF93A4E08F184030746DFF8E4B007939F
:10C0500094F904000BF010FE00285CD0B8F1000F3A
:10C0600061D029460C2220464FF096FB00283A4624
:10C07000484613BF012100214FF0010A4FF0000A8A
:10C08000FFF7DDF9074695F9040046F03FFDEA7930
:10C090000346514606EB82024846D2F8A026049297
:10C0A0002A7A06EB8202D2F8A0260392AA7906EB3E
:10C0B0008202D2F8A02602926A7906EB8202D2F8B6
:10C0C000A02601922A6800925A46FEF7AFFF94F923
:10C0D000040046F01BFDE2790346514606EB82025E
:10C0E0004846D2F8A0260492227A06EB8202D2F8C1
:10C0F000A0260392A27906EB8202D2F8A026029231
:10C10000627906EB8202D2F8A026019222680092A0
:10C110005A46FEF75BFF0C35079B0C34AB4297D1B8
:10C1200009B0BDE8F08FC246D1E700BF3CC909089D
:10C1300082510A082DE9F04780468CB00846FFF787
:10C1400043FB054638B10023594901201A460CB07B
:10C15000BDE8F0476AE7CDE909000B9007A8079111
:10C1600054494FF04BFA064646F0CAFB431C0446BE
:10C170000CD12B460A2208A93046FDF7ADF8089BE2
:10C180001B781BB9C4B2132C0BD944B220460BF058
:10C190002DFD054640B94046FFF701FB0CB0BDE858
:10C1A000F087333464B2F1E7424907A88DF828409C
:10C1B0004FF024FAB0B3002302260A221946FDF7F5
:10C1C0008BF809900027DFF8EC90DFF8F0A04946E3
:10C1D00007A84FF013FAF8B1FDF708F9364A002323
:10C1E00052F8041B88421FD1DBB20AEB8302D2F85B
:10C1F000A026904210D1022F20D0032F23D05A1E08
:10C20000012FD2B215D00B2A03D88DF82930013670
:10C21000F6B20137042FDAD1052E1AD84046FFF7BF
:10C22000C3FABBE70126CDE70133102BD8D1002399
:10C23000DBE7052AEDD88DF82A30E8E7092BE8D8A6
:10C240008DF82C30E3E79A1E0D2AE2D88DF82B30BA
:10C25000DDE709AB03CB286018686960A860204659
:10C2600046F054FC154A9DF82B10034602EB810161
:10C27000D1F8A01604919DF82C1002EB8101D1F8A1
:10C28000A01603919DF82A1002EB8101D1F8A016A7
:10C2900002919DF8291002EB81020021D2F8A0261C
:10C2A00008460192099A0092054AFEF78FFE75E74B
:10C2B000F44D0024B6520A08DCCF09083CC909082D
:10C2C00082510A082DE9F04F90468BB000264FF0BE
:10C2D000190A45464FF461790C461A460021074673
:10C2E000FFF7ADF80990B8F1000F49D029460A22AE
:10C2F00020464FF051FA0028099A384613BF012111
:10C3000000214FF0010B4FF0000BFFF798F82A893E
:10C310000990334606925946EA88384605922A79AA
:10C320000492EA780392AA781AFB029202926A783F
:10C330001AFB029201922A780092124AFEF776FEC8
:10C34000228933460136594606923846E2880A3534
:10C35000059222790492E2780392A2781AFB029263
:10C36000029262781AFB0292019214F80A2B009250
:10C37000044AFEF72BFE1E2EB5D10BB0BDE8F08FA0
:10C38000C346DDE79F510A082DE9F04380468BB094
:10C3900008460F46FFF718FA044638B100235E49F5
:10C3A00001201A460BB0BDE8F0438BE70846FDF7C5
:10C3B0001DF81D28054600F3A5800A268DF82740A4
:10C3C0004643781CFBF746F910B101238DF827305E
:10C3D000FBF740F9514C074668B1FDF707F80D2807
:10C3E00009D80A2303FB054383F808069DF8273084
:10C3F00001338DF82730DFF82091711C0DF12702F1
:10C4000038464944FCF7F6FFFBF724F9074668B1C4
:10C41000FCF7ECFF232809D89DF827300A220133C6
:10C4200002FB05428DF8273082F80B063846FBF7F1
:10C4300011F9074668B1FCF7D9FF0D2809D89DF816
:10C4400027300A22013302FB05428DF8273082F89B
:10C450000C069DF82730062B0CD0002309EB0602B2
:10C46000404649F80630536013810BB0BDE8F043F5
:10C47000FFF79AB90A260023384606FB0546A6F8B8
:10C480000E36A6F81036FBF7E5F8074618B1FCF7AC
:10C49000ADFFA6F80E063846FBF7DCF830B1FCF726
:10C4A000A5FF0A2303FB0543A3F810061C4B4FF01E
:10C4B000FF324FF461701A660A2303FB0542B2F89B
:10C4C00010360693B2F80E36059392F80C360493A4
:10C4D00092F80B360393192392F80A1613FB010105
:10C4E000029192F8091613FB0103002101930846FB
:10C4F00092F808360B4A00932B46FEF767FD0BB007
:10C50000BDE8F0831D232246074940460BB0BDE835
:10C51000F043FFF74DB900BF005A0024F853002440
:10C52000640700249F510A087C510A082DE9F04F46
:10C53000804691461E460C4615460027DFF81CA192
:10C540002DED088B95B094ED008AB5EE408AF1EEA2
:10C5500010FA7BD0D4ED019A94ED029AD4ED038ABF
:10C56000B9F1000F49D0D5ED00BA95ED01BAB4EE9E
:10C570006B8AD5ED02AA95ED03AAF1EE10FA6AD105
:10C58000F4EE4B9AF1EE10FA65D1B4EE6A9AF1EE40
:10C5900010FA60D1F4EE4A8AF1EE10FA0CBF0121D4
:10C5A000002132468B46404681F00101FEF747FFED
:10C5B000B0EE6B0A064611A8FAF7C8FFB0EE4B0AB8
:10C5C00007900EA8FAF7C2FFB0EE6A0A06900BA811
:10C5D000FAF7BCFFB0EE4A0A059008A8FAF7B6FFD2
:10C5E0000599069A079B039040460291594601928D
:10C5F000524600933B46FEF719FDB0EE480A11A8DB
:10C60000FAF7A4FFB0EE690A83460EA8FAF79EFF78
:10C61000B0EE490A06900BA8FAF798FFB0EE680A48
:10C62000059008A8FAF792FF069B059A002103904F
:10C6300040460292524610341035CDE900B33B46D5
:10C640000137FEF7C3FC082F7FF47DAF15B0BDECBA
:10C65000088BBDE8F08F0021A3E700BFC2510A0894
:10C660002DE9F14F06460C46DFF894B12046FFF75E
:10C67000ABF8074638B100235A4901201A4601B0E9
:10C68000BDE8F04F52E7052257492046FCF7E8FD88
:10C6900060B9544B00221A601A611A621A631A6454
:10C6A0001A651A661A6701B0BDE8F08F0422594670
:10C6B0002046FCF7D5FD05462046002D45D1FAF76A
:10C6C000C9FF07460028EED04CF000F9DFF834A18E
:10C6D0005FFA80F85AF8049BB9F1000F07D122469F
:10C6E0004249304601B0BDE8F04FFEF763BD424617
:10C6F000494638460135FCF7B3FD84460028E9D1A8
:10C70000384A034600211746013342F8101B082B14
:10C71000FAD1374B03EBC505D5F880E0BEF1000F29
:10C7200005D149463348344CFEF718FD9EE795F88D
:10C730007C50AC45F5DA0EEB0C1307EB0C140CF146
:10C74000010C0FCB84E80F00F3E7FCF74FFE07283E
:10C7500005463DD82046FAF77DFF074658B3F9F75E
:10C76000E1FE204B012403EB051383ED000A38465C
:10C77000FAF770FF074638B1F9F7D4FE194B0134C8
:10C7800003EB051383ED010A3846FAF763FF07460A
:10C7900038B1F9F7C7FE134B013403EB051383EDF2
:10C7A000020A3846FAF756FF38B9304601B0BDE8FC
:10C7B000F04FFEF7F9BF0446D9E7F9F7B3FE094B8E
:10C7C000032C03EB051383ED030A3FF454AFECE7AE
:10C7D00007233A460949304601B0BDE8F04FFEF75D
:10C7E000E7BF00BF745200249F4F0A08DB510A08BC
:10C7F0003CC90908EC510A087E500A087C510A0815
:10C80000D6510A081CD009082DE9F74F92460C466C
:10C810001A46002181465646FEF711FE0025804645
:10C82000DFF864B0BAF1000F2CD031460422204664
:10C830004EF0B2FF00284246484613BF01210021B6
:10C8400001270027FEF7FBFD738880465A460193B7
:10C8500039463AF82530484600932B46FEF7E6FB6A
:10C8600063885A46394648460193043634F8043BF7
:10C8700000932B460135FEF7A9FB042DD2D103B05E
:10C88000BDE8F08F5746EBE7F6510A082DE9F34172
:10C8900005460846FEF798FF0C46074638B10023C8
:10C8A000334901201A4602B0BDE8F041ACE73149F6
:10C8B0002046F9F799FD70B904222D4B4FF47A7098
:10C8C0004FF4FA61013A1880598003F10403F9D159
:10C8D00002B0BDE8F0812046FCF788FD032806463B
:10C8E00041D82046FAF7B6FE074698B1FCF77EFD20
:10C8F0004FF0010804463846FAF7ACFE20B1FCF7C9
:10C9000075FDB8F1000F09D1284602B0BDE8F0412D
:10C91000FEF74ABF40F2EE248046ECE7A4F2EE2296
:10C9200040F2DC539A4203D8A0F2EE229A420AD98E
:10C9300040F6CA0340F2EE220F49284602B0BDE895
:10C94000F041FEF735BF0D4B00210D4A03EB860386
:10C95000A3F83447A3F836073346CDE9004008462C
:10C96000FEF734FBB4E703233A460649E5E700BF88
:10C970002C5B00249F4F0A0807520A08F853002432
:10C98000F6510A084F4F0A082DE9F04F8FB089463B
:10C99000174600211A4606460024FEF750FD0DF109
:10C9A000240B0546DFF86CA059F82480594602A8EC
:10C9B000CDF8088046F05AF84FB357F824302A468D
:10C9C00030469845039313BF012100214FF0010821
:10C9D0004FF00008FEF733FD04A9054603A846F012
:10C9E00045F804A923465246009130464146FEF7D9
:10C9F0001DFB23460134524641463046CDF800B077
:10CA0000FEF7E4FA202CCFD10FB0BDE8F08FB84686
:10CA1000EFE700BF15520A08F0B5074689B008468F
:10CA20000E46FEF7D1FE054638B100231949012014
:10CA30001A4609B0BDE8F040A6E70846FCF7D6FC68
:10CA40001F2804461DD83046FAF704FE014620464A
:10CA500034F0DAFC78B103AE0E48314600EB8400C6
:10CA600046F004F823460C4A294628460096FEF76D
:10CA7000ADFA09B0F0BD384609B0BDE8F040FEF7A8
:10CA80008EBE1F232A460549384609B0BDE8F0404E
:10CA9000FEF78EBE3C5B002415520A087C510A0842
:10CAA0002DE9F04F924685B00C461A46002181468A
:10CAB0005546FEF7C4FC00268046DFF86CB0BAF19C
:10CAC000000F2FD02946042220464EF065FE002894
:10CAD0004246484613BF0121002101270027FEF7E7
:10CAE000AEFCEB7880465A4602933946AB7848460E
:10CAF00001932B8800933346FEF798FAE3785A4661
:10CB00003946484602930435A378019334F8043B30
:10CB1000009333460136FEF759FA102ECFD105B0F7
:10CB2000BDE8F08F5746E9E71F520A08F0B50746FF
:10CB300085B008460E46FEF747FE054638B100238D
:10CB40001C4901201A4605B0BDE8F040A8E7084698
:10CB5000FCF74CFC0F28044623DC3046FAF77AFD3C
:10CB60000146204634F02AFDA8B104F12002124B00
:10CB70002946284603EB820393F84727029293F84D
:10CB800046270192B3F844370C4A00932346FEF738
:10CB90001DFA05B0F0BD384605B0BDE8F040FEF71F
:10CBA000FEBD0F232A460649384605B0BDE8F040D1
:10CBB000FEF7FEBDBC5B0024F85300241F520A0898
:10CBC0007C510A082DE9F04F85B014461A460546F7
:10CBD00002910021FEF733FC4FF0000806460623C1
:10CBE0004FF0000903FB08F7C037029B13F807B0AA
:10CBF000002C7AD0E35D324628469B45039313BF51
:10CC0000012100214FF0010A4FF0000AFEF717FC46
:10CC1000039B0646374A51462846CDE900934346D2
:10CC2000FEF704FA4346334A514628460137CDE918
:10CC3000009B09F10109FEF7C9F9B9F1060FD4D13A
:10CC400008F10108B8F1060FC9D1E427029BA7F14A
:10CC5000E40913F807A0002C49D014F807B03246B5
:10CC60002846DA450DBF4FF001084FF000080121BA
:10CC70000021FEF7E4FB062306461E4A41462846ED
:10CC8000CDE9009BFEF7D2F901370623194A414648
:10CC90002846CDE9009AFEF799F9EF2FD6D1029BED
:10CCA00093F8EF70ACB194F8EF80324628464745D0
:10CCB00013BF0121002101240024FEF7C0FB002343
:10CCC0000C4A2146009328460723CDF80480FEF73E
:10CCD000ADF90023074A2146284600930723019710
:10CCE000FEF774F905B0BDE8F08FA2469AE7A046BA
:10CCF000CAE700BF31520A08F0B5054685B00846BC
:10CD00000B46FEF761FD044638B100231B490120A4
:10CD10001A4605B0BDE8F04054E701AE184F6A4628
:10CD2000174918464EF097FC88B1032C04D12846C9
:10CD3000FEF73AFD05B0F0BDFCF758FB6A4646F831
:10CD4000040B3946002001344EF085FCECE7032C3F
:10CD5000EDD1039FDDE901463A463146E0B234F0B9
:10CD600067FC18B92846FEF71AFDE3E73B46324652
:10CD700021460448FEF7F2F9DCE700BF3C5B0024E3
:10CD8000B6520A0831520A082DE9F04F0E461546F0
:10CD900089B01A4600210446B046FEF750FB2F46E4
:10CDA00081464FF0000B002D7AD039460C224046C8
:10CDB0004EF0F2FC00284A46204613BF0121002114
:10CDC0004FF0010A4FF0000AFEF739FB97F90B20EC
:10CDD00081465B460492514697F90A202046039209
:10CDE000B7F908200292B7F906200192B7F904209A
:10CDF0000092364AFEF71AF998F90B205B460BF1C0
:10CE0000010B51460492204698F90A200C3708F18C
:10CE10000C08039238F9042C029238F9062C01927E
:10CE200038F9082C0092294AFEF7D0F8BBF1080F18
:10CE3000B9D14FF0000BDFF898800C2303FB0BF9FE
:10CE400085B3002755F80900012356F8092003FA95
:10CE500007FA42403AEA020214BF1946002110EADA
:10CE60000A0F07D05B464246204600970791FEF71F
:10CE7000DDF8079956F809201AEA020F05D05B463B
:10CE8000424620460097FEF7A1F801370E2FD9D170
:10CE90000BF1010BBBF1080FCFD109B0BDE8F08F4A
:10CEA000AA46A9E72F46012356F8091003FA07F20C
:10CEB0000A4206D05B464246012120460097FEF713
:10CEC00085F801370E2FEED1E2E700BF45520A0880
:10CED0005D520A08F0B506468BB008460D46FEF7CF
:10CEE00073FC044620B300233D4901201A460BB0D1
:10CEF000BDE8F04048E72D2903D0A1F13003092B0C
:10CF000049D8052C05DD30460BB0BDE8F040FEF7F2
:10CF10004BBC2846FCF76AFA0AAB621C03EB4404DC
:10CF200024F80C0C15F8013F303B092BFAD91446B4
:10CF300029780029DFD1062CE5D1BDF81C20BDF9E8
:10CF40001C30072ADFD8BDF91E50A5F5FA7292B23F
:10CF5000B2F5FA6F18D8BDF92070A7F5FA7292B23F
:10CF6000B2F5FA6F10D8BDF922C065450CDC6745F3
:10CF70000ADBBDF924E00EF1640292B2C82A03D89C
:10CF8000BDF92640112C11DD164930460BB0BDE825
:10CF9000F040FEF70FB9202902D101352246C6E73D
:10CFA00030460BB0BDE8F040FEF7F9BB0C200E4A4E
:10CFB00064B200FB03220846A2F83858A2F83A7877
:10CFC000A2F83CC882F83EE882F83F48074A00953C
:10CFD000CDE903E4CDE9017CFDF7F8FF0BB0F0BD2E
:10CFE0002C5C002472520A08F853002445520A08A7
:10CFF0002DE9F04F89468DB0164600211A460746A6
:10D000000024FEF71CFADFF8DCA00546C4EBC403DD
:10D0100009EB030259F80300918840F3074892791D
:10D020000890ADF824108DF82620B8F1000F53D0E9
:10D03000002E54D0F218F0589188937907220A9064
:10D0400008A8ADF82C100AA98DF82E304EF0A4FBDC
:10D0500000282A46384613BF012100214FF0010B5A
:10D060004FF0000BFEF7EBF99DF82E3005465246C7
:10D07000069359469DF92D30384605939DF92C307D
:10D0800004939DF82B3003939DF92A3002939DF869
:10D09000293001939DF8283000932346FDF7C6FF01
:10D0A0009DF8263052465946384606939DF925305C
:10D0B00005939DF9243004939DF82330CDE9028334
:10D0C0009DF8213001939DF82030009323460134D0
:10D0D000FDF77CFF102C99D10DB0BDE8F08FB34661
:10D0E000DEE700BF88520A082DE9F04F06468BB0F4
:10D0F0000D46DFF8A08228464BF0E8FB034630B926
:10D100000246964901200BB0BDE8F04F70E70522BA
:10D1100093492846FCF7A4F80446C8B9914D014646
:10D12000702205F694004EF0B3FAC5F83448C5F8FD
:10D130004048C5F84C48C5F85848C5F86448C5F893
:10D140007048C5F87C48C5F888480BB0BDE8F08F3A
:10D15000042241462846FCF783F8044630BB2846A3
:10D16000FAF778FA81460028EFD04BF0AFFBDFF8F2
:10D1700028B282465BF8047B3FB92A467A4930469A
:10D180000BB0BDE8F04FFEF715B852463946484699
:10D19000FCF766F840B92046744D1EF03FF839465A
:10D1A0007348FDF7DBFFA6E70134E3E70722714987
:10D1B0002846FCF755F8074600287AD12021284652
:10D1C0004EF07DFA044670BB6B4D6C48FDF746FF90
:10D1D000214601342846FDF741FF0E2CF8D10025E9
:10D1E000DFF8B891664FFDF7EDFEDFF8B4810C264D
:10D1F0000024DFF8B0A129466E434846FDF72EFF14
:10D200000123F2595F48A340013413420CBF414649
:10D210005146FDF723FF0E2CF2D10135FDF7D2FE6A
:10D22000082DE4D191E702AC574D01AA56494EF0C2
:10D2300012FA002848D0022F11D1029A072A07D8E3
:10D24000039C0D2C04D80378722B13D06E2B25D0A1
:10D25000082300224D493046FEF7AAFA75E7FCF78D
:10D26000C5F801AA44F8040B2946002001374EF006
:10D27000F2F9DEE70C233B4903FB02110123D1F84D
:10D280003418A3400B4337490C2000FB02123949E4
:10D29000C2F834383046FFF727FF56E7314B0C20F1
:10D2A000012100FB0233A140D3F8343823EA010303
:10D2B000E9E72846002402AD334F01AA32494EF077
:10D2C000CAF980B1082C03D13046FEF76DFA3CE76D
:10D2D000FCF78CF801AA45F8040B3946002001340C
:10D2E0004EF0B9F9EDE7082CEED1029B0F2B30D8A8
:10D2F000DDF80CE0BEF1070F2BD8DDF810C0BCF153
:10D300000D0F26D8059F07F16402C82A21D8069D73
:10D31000FF2D1ED8079864281BD80899642918D8AF
:10D32000884216DA099C032C13D8C3EBC3020D4BB9
:10D33000134483F8991883F894E80C4983F895C846
:10D3400083F8967883F8975883F8980883F89A4872
:10D35000A0E70F493046FDF72DFFF6E68C5C002470
:10D360009F4F0A08F8530024DB510A087E500A0830
:10D37000EC510A08A5520A08AD520A084F570A088C
:10D380002C5C0024B2520A08B6520A08B8520A08A5
:10D3900072520A08D6510A081CD00908596F0A08A7
:10D3A0006D530A0870520A082DE9F04F9246002684
:10D3B00089B04FF019095546B3464FF461780C46D1
:10D3C0001A4600210746FEF73AF80790BAF1000F17
:10D3D00027D02946062220464EF0DEF90028079A7B
:10D3E000384613BF012100214FF0010B4FF0000B15
:10D3F000FEF725F86A790790334619FB02825946F1
:10D40000384605922A7919FB02820492EA7803923F
:10D41000AA7802926A7801922A780092104AFDF75F
:10D4200005FE627933460136594619FB02823846B9
:10D4300006350592227919FB02820492E278039262
:10D44000A27802926278019214F8062B0092044AA4
:10D45000FDF7BCFD0A2EB9D109B0BDE8F08F00BFC1
:10D46000BE520A082DE9F04F074689B008468B46A0
:10D47000FEF7AAF9044638B100234F4901201A46A5
:10D4800009B0BDE8F04F8FE74C4B084693F870ADFC
:10D4900093F8719D93F85A8EFBF7A8FF092805466B
:10D4A00000F3818006268DF81F40454C46430BF162
:10D4B0000100FAF7CFF8834640B1FBF797FF0D283C
:10D4C00004D8A319187301238DF81F305846FAF7B2
:10D4D000C1F8834660B1FBF789FF504508D80623A1
:10D4E00003FB054358739DF81F3001338DF81F303F
:10D4F0005846FAF7AFF8824660B1FBF777FF484528
:10D5000008D8062303FB054398739DF81F300133A9
:10D510008DF81F305046FAF79DF8814660B1FBF751
:10D5200065FF804508D3062303FB0543D8739DF8A8
:10D530001F3001338DF81F30DFF87C80311D0DF175
:10D540001F0248464144FBF755FF9DF81F30062B4C
:10D550000BD0002308EB0602384648F806309380CB
:10D5600009B0BDE8F04FFEF71FB903FB05424FF4C9
:10D5700061701923517C13FB01010591117C13FB90
:10D580000103002104930846D37B0393937B02930A
:10D59000537B0193137B0B4A00932B46FDF716FD3B
:10D5A00009B0BDE8F08F092322460749384609B083
:10D5B000BDE8F04FFEF7FCB80454002400430024FB
:10D5C000F8530024BE520A087C510A082DE9F04F96
:10D5D00014468BB00F461A4600210646FDF72FFF72
:10D5E0000546002C00F0D78022783B789A4202460C
:10D5F00030460DBF4FF001084FF000080121002117
:10D60000FDF71DFF237805469B4A41463046FDF74E
:10D610000DFD3B784146984A3046FDF7D7FC002C7B
:10D6200000F0BB80627830467B789A422A460DBF74
:10D630004FF001084FF0000801210021FDF7FFFE27
:10D64000637805468D4A41463046FDF7EFFC7B780E
:10D6500041468A4A3046FDF7B9FC07F1C90307F194
:10D66000020A04F1CA0B0593A31C4FF000090693AC
:10D67000822307933B784B4500F39180002C00F008
:10D68000F58097F8EA30304694F8EA209A422A4624
:10D690000DBF4FF001084FF0000801210021FDF7F8
:10D6A000CEFE94F8EA300546754A41463046FDF70D
:10D6B000BDFC97F8EA304146714A3046FDF786FCDA
:10D6C000002C00F0D58004F1EA0307F1EA0204F12E
:10D6D000FA014FF0010833F802CF32F8020F844507
:10D6E00018BF4FF000089942F5D188F001012A4691
:10D6F0003046C9B2FDF7A3FE0821054604F1EC004F
:10D70000FBF730FD5F4A034641463046FDF78EFC8D
:10D7100097F8EA1007F1EC00FBF724FD594A03469D
:10D7200041463046FDF752FC002C00F0A3804FF03C
:10D73000FC094FF0010807EB090104EB0900F8F7B9
:10D7400053FE09F10409002818BF4FF00008B9F58D
:10D750008E7FF0D188F001012A463046C9B2FDF72C
:10D760006EFE082104F1FC00F9F786FF464A0346E5
:10D7700041463046FDF75AFC97F8EA1007F1FC00E5
:10D78000F9F77AFF404A0346414630460BB0BDE800
:10D79000F04FFDF71BBCA0463BE7A04657E7079BB1
:10D7A000FB180993002C5FD0079B0998E3181946D2
:10D7B0000893F8F719FE059B5A789BF800309A42B7
:10D7C0004FD1B0FA80F84FEA5818069AAAF102032E
:10D7D0000AF10E01023A33F802CF32F8020F844503
:10D7E00018BF4FF000088B42F5D188F001012A469E
:10D7F0003046C9B2FDF723FE6278069905469BF8CC
:10D800001800FBF77FFC02909BF8003041461F4A4E
:10D8100030460193089B009309F10103FDF706FCD4
:10D82000059B51467A7809F10109587E0AF1100AE0
:10D83000FBF768FC059A0290414612F8013F30461A
:10D840000BF1010B0193099B059200934B460F4A84
:10D85000FDF7BCFB069B10330693079B0933079328
:10D8600008E74FF00008B0E7A046D9E7A04620E758
:10D87000A0464DE7A0467FE7D7520A08E9520A08BA
:10D8800017530A082F530A0846530A08FE520A087B
:10D890000379062B12D1C9B2C268072996BF084B7B
:10D8A0000021595C4FF001039CBF013149B28B400C
:10D8B000134214BF08464FF0FF307047481C7047B2
:10D8C000C8BF090838B5074C074DAC4203D3074B16
:10D8D00001221A7038BDA288D4E902104DF080FEF2
:10D8E0001C34F2E7F0C60B08E4D00B08D45900242E
:10D8F0001B4BB0F5FA6F1A680346A8BF4FF4FA63E2
:10D90000B3F57A7FB8BF4FF47A73D20416D540F2DC
:10D91000DC52904220D040F2DB5207EE903A904227
:10D92000F8EE677A99BF9FED0F7A9FED0F0A9FED92
:10D930000F7A9FED0F0AA7EE870A7047B0F57A7F3E
:10D940000AD907EE903A9FED0B7A9FED0B0AF8EE9D
:10D95000677AA7EE870A70479FED080A704700BFF5
:10D96000D44E0024D52000C010903E45D520004064
:10D9700040A0F4C4671000401160F4C4000000002F
:10D98000704700BF00207047704700BF00207047FD
:10D9900001207047704700BF704700BF704700BF4D
:10D9A000704700BF9FED010A704700BF00000000F4
:10D9B00000207047064B1B78834281BF00EB40007C
:10D9C000044B03EBC003586998BF0020704700BFA9
:10D9D0004C0500205005002000EB4000024B03EBFB
:10D9E000C003587C704700BF50050020024B1878D8
:10D9F000003818BF012070474C050020C3B25E2BD1
:10DA00009ABF024B53F820000148704724000A08CF
:10DA10002CB10A0803681B6903B11847704700BF9F
:10DA20000023084901E0152B09D003EB4302013321
:10DA300011F802C00A448445F5D110467047002011
:10DA4000704700BF202D0024F0B1B1FA81F35B09CB
:10DA5000D1B110B50D4C4FF0010E224602E001335A
:10DA60004E2B0FD092F804C01C328445F7D10EF132
:10DA7000010C71455FFA8CFEF1D1C3EBC30304EBDB
:10DA8000830010BD002010BD00207047B0C0090801
:10DA90002DE9F0434FEA101887B015461F46DDF810
:10DAA000389008F1400800F00F0431B3FFF7CCFFC5
:10DAB000C3790646164A29463846CDE9004343460F
:10DAC000C847B8B130684AF069FDB279737912F08D
:10DAD000020F1049104A03F1010318BF0A46F179F9
:10DAE0000094CDE90321CDE901030C4A434600210E
:10DAF0003846C84707B0BDE8F0834346084A294680
:10DB00003846CC460E9407B0BDE8F043604700BFEE
:10DB10008B530A08F14E0A087E500A089D530A08E2
:10DB2000BF530A082DE9F04FDFF878B00F4601F136
:10DB300009080124BBF8003004339DB217F8011B1B
:10DB4000AC464FF0000E04FA0EF2ACF104030A40AA
:10DB50009BB21BD103F1010A00EB83091FFA8AF380
:10DB6000C9F814209C45F5D10EF1010E0CF1040CFE
:10DB7000BEF1080F1FFA8CFCE5D120354745ADB248
:10DB8000DCD10023ABF80030BDE8F08F868903F1CB
:10DB9000010900EB83021FFA89F356616345F6D150
:10DBA000E2E700BF24A300242DE9F047DFF87CA0C2
:10DBB000884601F106090024BAF8023001260B3329
:10DBC0001FFA83FE18F801CB71460025A1F10B0363
:10DBD0009BB23DB1092D20D06A1E06FA02F212EA6C
:10DBE0000C0F1AD0878900EB830201339BB2576177
:10DBF0009942F8D10B1D01350C3100EB83030A2D3E
:10DC000089B25C60E2D10EF1780EC8451FFA8EFE33
:10DC1000D8D1AAF80240BDE8F0871A1D01339BB2A3
:10DC200000EB82028B425460F7D1E3E724A3002487
:10DC30002DE9F8430E780446057B00F11003F64306
:10DC400000F13802F6B243F8045F9342FBD1282278
:10DC5000002104F13C0005274DF01AFD4FF00008AB
:10DC60004FF0140E46FA07F2734602F00102002A42
:10DC700042440CBF4FF00A094FF0190917F0010F89
:10DC80005FFA82F80EEB090C14BF284600201FFA39
:10DC90008CFC591C04EB83028BB250616345F8D1B4
:10DCA000013FF1447B1C1FFA89FEDBD118F0010F04
:10DCB000734614BF19200A200EEB0006B6B2591C99
:10DCC00004EB83028BB25561B342F8D1421E0EF1D0
:10DCD00001030EF10200074992B2134402449BB2C1
:10DCE00092B204338A80002104EB830359602261DD
:10DCF000BDE8F88324A3002470B5094CA36873B170
:10DD00000546002606E099681A681E73A1609047D0
:10DD1000A36823B15A681846AA1A002AF3DA70BD1C
:10DD200024A30024154B1B682DE9F041044688B05C
:10DD3000F3B11A6804A91846D56A6A46A847064688
:10DD400088B104AC6D460027DFF83C80013735F818
:10DD5000022B34F8021B4046FDF700FABE42F5DC08
:10DD600008B0BDE8F08106492046FDF723FAF7E741
:10DD7000044908B0BDE8F041FDF71CBAEC5300249B
:10DD8000EB530A0803540A08D1530A08034904480C
:10DD900001F5FD610EC9FDF7E1B900BF00F0F01F0C
:10DDA0000A540A0870B5054608461646FBF71EFBDE
:10DDB0000D4B041E1A780EDB944205DA21460B48FF
:10DDC000FDF7CCF9204670BD2EB1FF2C03D10848D9
:10DDD000FDF7C4F9F6E7013A064928464FF0FF344B
:10DDE000FDF7E8F9EEE700BF881400201E540A088A
:10DDF0002F540A0842540A0870B50A4C00250A4EEE
:10DE000094F8913013B12046FCF76AFF20460135A3
:10DE1000FDF744F83046FDF773F8042D04F1EA04E9
:10DE2000EED170BDC44900246C4D002438B50C46B9
:10DE3000054616492046F8F7D7FA30B9FFF7DCFF58
:10DE40001348BDE83840FDF7D5B812492046F8F729
:10DE5000CBFAA8B9104B83F8910083F8990083F8A6
:10DE60007B0183F8830183F8650283F86D0283F8F0
:10DE70004F0383F85703094B83F821000848E0E774
:10DE80002846BDE83840FDF78ABC00BF68540A0840
:10DE90006E540A0889540A08C44900246C4D0024B1
:10DEA00091540A0870B5054608460C464AF00EFD26
:10DEB000024670B1072804D1214609484DF025FCDF
:10DEC00038B12846064B074A0749BDE87040FDF7C0
:10DED00071B903490548BDE87040FDF73FB900BF7F
:10DEE000AD540A08B5540A08C0540A08EA540A088E
:10DEF00070B5054608460C464AF0E8FC024670B18B
:10DF0000032804D1214609484DF0FFFB38B12846CB
:10DF1000064B074A0749BDE87040FDF74BB9034976
:10DF20000548BDE87040FDF719B900BFF8540A086C
:10DF3000FC540A08C0540A080C550A08F8B54E1ECD
:10DF4000054601F11F04054F16F8012F28463946F2
:10DF50000235FBF7C1F8A642F6D1F8BD1F550A08F5
:10DF600002460846531C05D1044B1A681B790A6007
:10DF70000B7170470249FBF7AFB800BFE05C0A08BD
:10DF8000596F0A0810B501311446FFF75DFD28B935
:10DF9000064B1A681B792260237110BDC279204696
:10DFA0000349BDE81040FBF797B800BFE05C0A08E2
:10DFB00098530A082DE9F04307469BB008460C46E3
:10DFC0004AF084FC06462022002101A84DF060FBA7
:10DFD00036B3402E08D040233246394938461BB06C
:10DFE000BDE8F043FDF7E6B801AD04F140084FF09D
:10DFF00000090222214668464DF099FB00231022B9
:10E0000009A968468DF80290FBF766F9099B0DF1A6
:10E010000202934222D1023405F8010BA045E8D157
:10E0200009AC41220021274D20464DF031FB002E46
:10E030003BD02E7BD6B1202205F10D0101A84DF079
:10E04000ABFB98B105F10D012046FFF777FF2346A2
:10E050001D4A38461D49FDF7ADF804E01A783846E8
:10E060001B49FDF7A7F81BB0BDE8F083194B1B78DF
:10E07000DBB9D6B901AB184E1A46083603CAA2421C
:10E0800046F8080C46F8041C1346F5D10123204637
:10E09000114985F82D30FFF751FF1048FCF7B0FF0C
:10E0A00021460F48FDF75AF8DDE795F82D3013B9F2
:10E0B0002B7B002BF4D008492046FFF73FFFEFE70A
:10E0C00024550A0824A3002462550A08C0540A08EB
:10E0D00046550A08D459002431A300246C550A0877
:10E0E0007B550A0873B50E4610490546F8F77CF9CA
:10E0F00018B93070012002B070BD2C78602C8CBF34
:10E10000613C413C082C0FD8013501230A2201A9AA
:10E110002846FBF7E1F8019BAB4205D00F2803D856
:10E12000013440EA0410E4E70020E4E7E05C0A0878
:10E130002DE9F04F0F46904689B0002187EA080884
:10E140000646139A00250393FDF779F9DFF88490CA
:10E150006FEA080304460693284609F027FB129B42
:10E16000184230D0069BDFF870B0034014BF4FF068
:10E17000010A4FF0000A049310EA070328460CBF77
:10E180004A465A460593079209F022FB039B8046B4
:10E19000079A514600903046FCF748FF049B224600
:10E1A0003046B3FA83F14909FDF749F9059A044667
:10E1B000039B002A0CBF5A464A4651463046CDF8CA
:10E1C0000080FCF703FF0135172DC5D109B0BDE86C
:10E1D000F08F00BF88550A08D0510A0810B5114BBE
:10E1E00086B0114904460493104B11480393114B18
:10E1F000114A0293114B0193114B0093114BFCF701
:10E200002DFFFCF7DFFE10491048FCF7A7FF3CB1DB
:10E210000F4A1049104806B0BDE81040FCF79EBFF9
:10E2200006B010BDD2550A089C550A08D7550A08F1
:10E23000A7550A08E1550A088F550A08EA550A0841
:10E24000F6550A089F4D002400560A0808560A0889
:10E25000AD540A08F8540A0819560A080120BDE707
:10E2600038B50B4D0C4605EBC00595F97C01FFF761
:10E27000C5FB01460748FCF7F1FE95F8823133B142
:10E28000611C0548C9B2BDE83840FCF7E7BE38BD9F
:10E2900024000A084E570A08586F0A0810B50446A9
:10E2A000012022F09FFA28B920460549BDE8104018
:10E2B000FCF780BF0348BDE81040FCF74FBF00BF2C
:10E2C00046560A0855560A082DE9F743804608467F
:10E2D0000C46FDF779FA054628B14046FDF764FA89
:10E2E00003B0BDE8F083204601AA2C492F464DF02B
:10E2F000B2F92E460446DFF8A4907CB9022DECD189
:10E30000A7F57A73B3F57A7F21D94FF4FA634FF406
:10E310007A7223494046FDF74BFAE1E74DB1012DF2
:10E3200010D001AA4946002001354DF094F9044669
:10E33000E3E7012221464046FFF734FD431C064631
:10E34000EFD1CDE72046FBF751F80746E9E7154B3B
:10E35000B8B21B685B689847FCEEC07AFF2E17EED8
:10E36000902A0BD1104BB6EEC00A19780F4BA14280
:10E3700010DC11460E48FCF7F1FEB1E70D4B3146BB
:10E380000D48B6EEC00A03EB860383ED0C0AFCF7DA
:10E39000E5FEA5E70134A3EC010AE8E7B6520A0856
:10E3A000CF620A08401600208814002054A30024DD
:10E3B0006D560A0824A3002460560A08064B10B5BF
:10E3C0000446186832F022FE28B920460349BDE809
:10E3D0001040FCF7EFBE10BDFC5900247C560A0823
:10E3E00070B50024144E96F82330651CE340DB071B
:10E3F0001CD5E4B229461148FCF7B0FE7521204631
:10E4000023F058FE01460E48FCF7A8FE1A212046CC
:10E4100023F050FE01460B48FCF7A0FE1B212046CE
:10E4200023F048FE01460848FCF798FE022D4FF005
:10E430000104D8D170BD00BF6C4D002492560A086B
:10E440009E560A08B1560A08C4560A08F8B5074687
:10E4500008460C46FDF7B8F9C8B11F4B1E680136D7
:10E460003046344609F0B4F90546F0B90134182CA9
:10E47000A8BF0024204609F0ABF90546A8B9B4426C
:10E48000F4D138461549BDE8F840FCF793BE204664
:10E49000FAF7ACFF044609F09BF9054628B9214676
:10E4A0000F48BDE8F840FCF759BE0B4B1C6009F063
:10E4B00005FD2A460B482146FCF750FE172C9BBF52
:10E4C000094B0C22002002FB043398BF93F8DC02B6
:10E4D000BDE8F84009F02EBDEC130024D7560A0819
:10E4E000EB560A0801570A0824000A0870B50546C9
:10E4F0000C46114E2046FDF767F960B10F4B1048EE
:10E5000093F900104B1C0ABF0E4BC9B21978BDE835
:10E510007040FCF723BE2046FAF768FF032804D8B2
:10E52000C0B23446FCF71EFAE4E728460322064947
:10E53000BDE87040FCF73EBE7E500A086408002427
:10E540001A570A08984D00242A570A0870B505463C
:10E550000C46114E2046FDF737F960B10F4B1048BD
:10E5600093F900104B1C0ABF0E4BC9B25978BDE895
:10E570007040FCF7F3BD2046FAF738FF032804D8B3
:10E58000C0B2344615F0D6FBE4E72846032206491C
:10E59000BDE87040FCF70EBE7E500A0865080024F6
:10E5A00016570A08984D002425570A080329F0B584
:10E5B000054685B00C46164614D80B4F3970FCF74B
:10E5C00001FD0A492846FFF791FF2246084901A8A4
:10E5D000FAF782FD01AB324608212846FCF7ACFF72
:10E5E000FF233B7005B0F0BD640800247E500A088C
:10E5F0001A570A080329F0B5054685B00C46164699
:10E6000014D80B4F3970FCF7DDFC0A492846FFF798
:10E610009DFF224608496846FAF75EFD6B46324682
:10E6200010212846FCF788FFFF233B7005B0F0BDA2
:10E63000650800247E500A0816570A082DE9F84F8D
:10E64000002607460C461D4DB046DFF87890DFF8EF
:10E6500078A02046FDF7B8F8D5F800B048B92146B3
:10E660005846FAF721FE20B921466868FAF71CFEE1
:10E6700080B15846FCF79EFC696811B15046FCF722
:10E68000EDFCA96811B14846FCF7E8FC4FF0010821
:10E69000FCF798FC01361035362EDAD12046FDF70E
:10E6A00093F848B9B8F1000F06D12246384604491C
:10E6B000BDE8F84FFCF77EBDBDE8F88F20040A08DE
:10E6C00051570A084B570A0845570A08434B2DE98A
:10E6D000F74F1A780546009141495B780A70414A24
:10E6E0001370414B1B780BB9FFF7ECF83F4C002639
:10E6F00040F0E4FBB046A3460D23009973435BF85A
:10E7000003904846FAF7D0FD002840D0B8F1000F3A
:10E7100001DDFCF757FC49463548FCF79FFC002219
:10E7200021462846FCF77AFFFCF74CFC237903F0DE
:10E730001803082B44D0102B47D02046FCF77CFF51
:10E740000D2303FB06B3B3F8090040F07DFB8246BE
:10E75000D8B12046FCF7A2FE0746DAE902210244BE
:10E7600001442046FCF724FE78B94946019021482F
:10E77000FCF774FCDAF80810019A28461346CA1907
:10E780002146FCF72FFDFCF71DFC08F101080136BE
:10E7900040F28B230D349E42AED10020FCF75CFE8C
:10E7A000FF230F4A13700F4A1370B8F1000F11D1F5
:10E7B000009A2846104903B0BDE8F04FFCF7FABCB8
:10E7C0000E492846FFF792FEB7E70C492846FFF7A7
:10E7D000BDFEB2E703B0BDE8F08F00BF984D002446
:10E7E0006408002465080024D459002414DF0908B3
:10E7F0006F4E0A0865570A08DB510A087E500A085E
:10E800002DE9F04F3B4C89B00A4600210546FCF744
:10E8100016FE059094F90000FFF7F0F88146608835
:10E8200040F012FB344BD0F808B01F7817B15F46A8
:10E83000D0F80CB0A3790026012B38BF0123069332
:10E840002279637906FB02331BF80380002F3AD04C
:10E85000FB5C4345059A2846079313BF012100211D
:10E860004FF0010A4FF0000AFCF7E9FD079B013663
:10E87000059053B303F00F021B095146284640335D
:10E8800002921E4ACDE900634B46FCF7CFFBB8F17C
:10E89000000F24D008F00F034FEA1818174A51460A
:10E8A000029308F140032846CDE900634B46FCF78C
:10E8B0008DFB069BB342C3DC0834114BA342A9D1A4
:10E8C00009B0BDE8F08F3B46C3E7002FDFD04B46D1
:10E8D0000C4A514628460096FCF7A8FBD7E76B0682
:10E8E000E7D44B46074A514628460096FCF76EFB94
:10E8F000DFE700BFA0010A08D459002475570A08B1
:10E9000000030A088B570A082DE9F04F0C4607460A
:10E910008BB040F2162040F097FA224605460021BF
:10E920003846FCF78CFD404B064615221B7800212B
:10E9300004A8002BD5E9024504BF25461C464CF02F
:10E94000A7FE05F13F03039395F80090B9F1000F7E
:10E9500030D095F801A0002C63D022460023117816
:10E96000494557D1283392F8018001226B4403F8BE
:10E97000182CD0453246384613BF012100214FF0F4
:10E98000010B4FF0000BFCF75AFD064654B1B8F1ED
:10E99000000F07D0254B5A464146484600933B4658
:10E9A000FFF776F8224B5A465146484600933B46BD
:10E9B000FFF76EF80335039B9D42C5D13CB3651C40
:10E9C0000DF110084034DFF86490DFF864A018F807
:10E9D000013BCBB915F8013CB3B116B13046FCF799
:10E9E0000FFB29783B4615F8010C0022CDF800906A
:10E9F0000026FFF74DF8002215F8010C3B461146A2
:10EA0000CDF800A0FFF744F80335A542DFD10BB0E5
:10EA1000BDE8F08F01330332152BA0D14FF0000871
:10EA2000A7E7A046A5E700BFD45900242DB00408ED
:10EA3000CDAF0408234870B5FCF7BCFA224B93F81D
:10EA40005030002B38D0214B93ED010A4BF00CFED7
:10EA500001461F48FCF782FB1E4C1F48FCF7AAFA30
:10EA60001E4B94F821001E4A00280CBF1046184681
:10EA7000FCF7C0FA94F8213013B31A4C1A48B4F8D2
:10EA80009210FCF7EBFA194E94F89000184D0028FC
:10EA90000CBF30462846FCF7ADFAB4F89410154880
:10EAA000FCF7DCFA94F8910000280CBF30462846A9
:10EAB000BDE87040FCF79EBA0F48FCF79BFACBE725
:10EAC00070BD00BFAF570A0824A30024EC13002434
:10EAD000C9570A08C04D0024D8570A08F04E0A0842
:10EAE00069700A084C160020E9570A08A8570A0856
:10EAF0009F570A0810580A08CE570A086B4B1B7814
:10EB00002DE9F04F87B0002B00F0CA80684D4FF020
:10EB100000086848A968FCF721FB69686648FCF7AB
:10EB20001DFB664B6648D3E90031C91A654B1A686C
:10EB3000B1FBF2F2FCF712FBFCF744FA6248FCF777
:10EB400059FA6248FCF756FA614B5FFA88F41B7871
:10EB5000A34221D85F4D00245F4EFCF733FA013405
:10EB600055F8041F3046FCF779FA162CF7D15B4DA7
:10EB70000124594EFCF726FA2B46696801343046C9
:10EB80001B680435C91AFCF769FA162CF4D107B0D2
:10EB9000BDE8F04FFCF716BA514B14264FF03C0B72
:10EBA000671C03EB840306FB045693ED280A4BF025
:10EBB0005BFD96F81EA081B2B6F80E901AF0010F18
:10EBC00080B20CBF2D2252221AF0020F0490454849
:10EBD0000CBF2D2354231AF0040FB1FBFBF10CBF23
:10EBE0004FF02D0C4FF0560C1AF0080F05914FF016
:10EBF00064010CBF4FF02D0E4FF0430E1AF0800F42
:10EC000001FB09F10CBF4FF02D0A4FF0530ACDE97B
:10EC100000CECDE902A13946FCF720FAB37FDB072D
:10EC20003AD55C23304A6343D118D05891ED010A9C
:10EC300070B1B8EE400ADFED2D7A20EE270A07EE1C
:10EC4000900AF8EE677A80EE270A4BF00DFD00B2CD
:10EC5000642290FBF2F102FB11022548FCF7FEF959
:10EC60001421244808F1010801FB075701FB045453
:10EC7000F988628A0491218B02F0030392080391C0
:10EC8000E18A0291A18B0191A18A009119214B4344
:10EC9000218AFCF763FA57E71748FCF78BF9DFE79F
:10ECA000164807B0BDE8F04FFCF7A4B948050020AE
:10ECB000F40C002030580A0840580A08E80E0020DA
:10ECC00057580A08082A002484580A08E0580A08F5
:10ECD000881400209C0D002090590A08A00D0020E7
:10ECE0004C1600203C590A08140A002000401C461B
:10ECF00059590A086E590A0865590A0894590A08A8
:10ED000008B5224BF0EE407A1B68DB0420D5B5EE47
:10ED1000400AF1EE10FA32D09FED1D7AB4EEC70A28
:10ED2000F1EE10FA2BD49FED1B7AB4EEC70AF1EE88
:10ED300010FA99BF9FED187A9FED180A9FED187A87
:10ED40009FED180AA7EE870A4BF08EFC80B208BD33
:10ED50009FED0F7AB4EEC70AF1EE10FA09DB9FEDD2
:10ED6000127A9FED120AA7EE870A4BF07DFC80B263
:10ED700008BD9FED0F0A4BF077FC80B208BD9FEDF8
:10ED80000D0A4BF071FC80B208BD00BFD44E0024C8
:10ED90000000404200E0824466BEFFBE3B5FBE44CE
:10EDA00066BEFF3E9261744437DFFF3EC540744447
:10EDB00000007A440080BB44B54BB6491A68B64B94
:10EDC0002DE9F04FB2FBF3F291B00746B3480024AF
:10EDD000FCF744F9B24EFCF7F5F8B24AB249B34831
:10EDE000FCF73CF9B24DFCF7EDF8B24BB24AA9463C
:10EDF000997BB24B06EB8101B148D31AB14AD1F8E5
:10EE00005C171288FCF7AAF9DFF86883FCF7DAF8D8
:10EE1000AD48FCF7CFF8AD4BAD481978FCF71EF9BB
:10EE2000AC48FCF7C7F8AC4BAC481A88AC4B92B274
:10EE3000DFF844A31978FCF711F9DFF840B3FCF7C9
:10EE4000C1F8A849A848FCF709F9234698F81F20FB
:10EE5000E240D1072DD513B1A448FCF7ABF8611CF3
:10EE60005046FCF7FBF8A24BA248E35C5BF823108A
:10EE7000FCF7F4F899F86A35E340DA0702D59E48C2
:10EE8000FCF7ECF895F81831032B09D09B48FCF7F8
:10EE9000E5F895F81831012B02D19948FCF7DEF816
:10EEA000EB6C2BB15B7B012B02D99648FCF7D6F8B3
:10EEB000012305F5CE75002C00F0E580002B40F015
:10EEC000E4809148FCF796F8904DDFF8B482D5F8CD
:10EED0005890DFF8B0A208F1180B0123A34013EA01
:10EEE000090F15D01AF8042058F824305BF82410C4
:10EEF00053F822208648FCF7B1F8012C06D1854B47
:10EF000093F8DD1011B18448FCF7A8F8FCF75AF823
:10EF10000134062CE1D18148FCF74CF8804B1B688A
:10EF20001B0640F1628195F87830DFF85C82032B94
:10EF30008CBF7C487C48FCF73DF898F80030022BE9
:10EF400040F024817948FCF735F895F87830042BA7
:10EF500000F242817648FCF72DF895F88830002BB6
:10EF600000F0418106EBC303D3F898177148FCF712
:10EF700075F8FCF727F8704B70481C68704B1A78CE
:10EF8000704B53F82210FCF769F824B1227A617AA9
:10EF90006D48FCF763F8FCF715F86C493846FCF748
:10EFA0006AF8FCF70FF86A4B6A4819684FF47A73ED
:10EFB000B1FBF3F1FCF752F805A8FAF71BFB38B1E7
:10EFC00005A908A848F0D6FF08A96348FCF746F849
:10EFD000FBF7F8FFD5F81471002F00F00A8107EE57
:10EFE000907ADFED5E6AB8EEE77AC6EE877AFDEEDC
:10EFF000E77A17EE903A95F8500030B1584A0393EB
:10F0000092ED010A4BF030FB039BD5F894405CB1C4
:10F0100007EE904ADFED516AF8EEE77A86EEA77ABE
:10F02000FDEEC77A17EE904A3A4AB2F82C113A46EA
:10F030006429CDE90004A8BF64214A48FCF78EF892
:10F04000B5F84C2964234848B2FBF3F103FB1122C5
:10F0500095F85D3906EB830692B2D6F8CC37254E8B
:10F06000009395F85C390125FCF778F83F48FBF7E9
:10F07000A1FF3F4B1C68002C40F0BD80FBF7A2FFB6
:10F0800011B0BDE8F08F0124E0E6FBF79BFF1BE722
:10F09000AC030024B8590A0840420F00C1590A08BD
:10F0A00024000A08F8FF012000080000D3590A08CC
:10F0B000F80E0020984D002400000408000002080B
:10F0C000E5590A08D0480024FC590A08B82E002443
:10F0D0000E5A0A08484E0A088C310024165A0A08AB
:10F0E000B92E00242A5A0A082F5A0A089F5A0A08D9
:10F0F00078A30024BE5A0A08A7590A08395A0A08F0
:10F10000415A0A08465A0A084E5A0A0824A30024FB
:10F1100070640A084C160020535A0A08575A0A0805
:10F12000D44E00245D5A0A08695A0A08795A0A0816
:10F13000E26A0A08B25A0A08F4560024CE5A0A08AB
:10F14000F3560024C4D00908D75A0A087E500A088A
:10F15000EC290024E15A0A08FB5A0A0800247449E1
:10F16000EC1300240E5B0A08545B0A08795B0A085A
:10F17000E45100246C4D0024345A0A0890D1090847
:10F1800088070A08F4130024844E0024022008F0A3
:10F19000A1FD044608B91F48D5E690F9040043F0E4
:10F1A000B5FCDFF894A0814631F0C8FF5AF8202062
:10F1B00049461948FBF752FF98F80330012B04D158
:10F1C0001648FBF7F7FE1648BDE6A37915485AF82E
:10F1D0002310FBF743FFF6E798F802300BB912480B
:10F1E000B9E61248B7E61249C0E61248FBF7E2FE5C
:10F1F000BFE63B46FFE694FAA4F0B0FA80F005FAC9
:10F2000000F024EA000408F0B7FA01463046FBF7A4
:10F2100025FF30E77F5A0A08895A0A08995A0A08CE
:10F220009E5A0A089B510A08A25A0A08A84D0A08C1
:10F23000B0590A08C25A0A08DCCF09082DE9F04F74
:10F24000DFF8748199B098F80330002B00F09780B4
:10F2500050480025504EDFF864B1FBF7CBFE2F4637
:10F26000DFF85C91DFF85CA10BA9E8B214F04AFB6F
:10F270009DF83430002B53D0139C54B107EE904AC4
:10F280009FED460AF8EE677A80EE270A4BF0ECF91C
:10F2900004460B9A29465846FBF7E0FE109A002ACE
:10F2A0006FD002FB04F04FF47A73B0FBF3F30993D1
:10F2B000DDF848C0BCF1000F65D00CFB04F142F250
:10F2C0001073B1FBF3F1082D98F8033018BF7F18C5
:10F2D000002B5AD017984FF47A7E0A23079015987E
:10F2E0000690169805901198B0FBFEFECDF810E040
:10F2F0000998B1FBF3FE03FB1E11CDE902E1099968
:10F30000B1FBF3F103FB1100BCFBF3F3CDE90010FB
:10F3100021465046FBF722FF0023B362C6E90D33B6
:10F3200001354036232D9FD198F8033023B31C4C70
:10F330004FF47A731B48D4F86019D4F86429B1FBF0
:10F34000F3F3D208D4F86819FBF708FF0A2216482D
:10F3500097FBF2F102FB1172FBF700FF134B1B78D6
:10F36000432B06D1D4F86C29D4F870191048FBF758
:10F37000F5FE0023C4F8683919B0BDE8F08F0D48D8
:10F3800067E7099294E761469DE721464846FBF707
:10F39000E5FEC1E78F5B0A08B0A300248096184BF6
:10F3A00024A30024365C0A08565C0A08F0290024CD
:10F3B0007A5C0A08ED5B0A08984D0024F75B0A089E
:10F3C00055590A08065C0A082DE9FF47914604468C
:10F3D0008A461E46FEF75CFA421CBDF830700546B0
:10F3E000DDF834801FD0B9F1FF3F1FD0154A3146F8
:10F3F000CDE9000938462368C0474A465FFA8AF1DA
:10F400002079F3F703F8024600B10288D3B23146FF
:10F4100038460393C2F30323120B0293CDE9005243
:10F42000094A2368C04704B0BDE8F0877B06FAD4D8
:10F430000C90314623683846044AC44604B0BDE8FF
:10F44000F0476047A45C0A08B15C0A08D65C0A0869
:10F450002DE9F043154685B0894619466A1CBDF86A
:10F4600030600D9F28D04FEA101800F00F04194AA1
:10F47000304608F14008CDE900454346B847C0B1E1
:10F48000EBB2D9F8000099F805100F2B11D82A46D5
:10F49000F3F704F868B1038800210278304603923C
:10F4A000C3F303221B0B02920B4ACDE900434346F0
:10F4B000B84705B0BDE8F0837306FAD4030900F03D
:10F4C0000F00064ABC460C904033304605B0BDE8FC
:10F4D000F0436047E55C0A08F75C0A08215D0A080A
:10F4E0002DE9F04F714C8DB0DFF8CC910A4604F154
:10F4F000800A00218346FBF7A2FF03900025A37A30
:10F5000099F80060AB4200F3908010345445F5D177
:10F5100040F216200DF1180A3FF096FC0027002E4D
:10F520004FF015024FF00001D0E90245504604BFEC
:10F53000254634464CF0ACF82E78002E3CD0697845
:10F540003046FEF781FA95F90290049009F1010224
:10F5500053425341002C00F0A5800022A05CB04231
:10F5600040F09C80224492F90280C14540F0948092
:10F5700052788A4208BF0123012203F001030AF8EE
:10F58000072083F00101039A58460593FBF757FFC4
:10F59000059B039044B1464A30460499CDE900B238
:10F5A0004246FFF755FF059B424A30460499CDE994
:10F5B00000B24A46FFF74CFF01370335152FBBD188
:10F5C00084B3564604F13F07DFF8E480DFF8E490A7
:10F5D00016F801ABBAF1000F21D12078F8B194F9F7
:10F5E000023001331BD06178FEF72EFA0546039AEC
:10F5F00001215846FBF723FF94F902205346294680
:10F6000003902078CDE900B8FFF722FF2078534619
:10F610004FF0FF322946CDE900B9FFF719FF033457
:10F62000BC42D5D10DB0BDE8F08FE0883FF00CFCB6
:10F63000002E627AD0E90231207A04BF194633469F
:10F6400005FB00228F5623B39E56B742039A5846B5
:10F65000049313BF012100214FF001084FF000086F
:10F66000FBF7EDFE049B039043B1114B3246294654
:10F670002046CDE900B34346FFF7A6FE0D4B2946D1
:10F680003A4620460135CDE900B34346FFF79CFEDC
:10F6900035E74FF0FF36D8E700236DE703323F2A06
:10F6A0007FF45CAF4FF0FF386BE700BFFC13002422
:10F6B0002DB00408CDAF0408D4590024AA4B1B6810
:10F6C000002B38D05B69F0B585B0984788B3A74D5B
:10F6D000D5F8CC36002B01DDF9F788F9A44C637816
:10F6E000022B33D0032B24D195F8E83713B1A1486E
:10F6F000FAF70EFA95F8D43613B19F48FAF708FADC
:10F7000095F8183713B19D48FAF702FA95F85C3767
:10F710007BB19B4805B0BDE8F040FAF7F9B99948CC
:10F720000321302305220090A1709748974948F0A3
:10F730000DFD05B0F0BD7047A26801209449F8F7AF
:10F740000BFC012840F074810623A370A378072BDB
:10F75000EFD801A252F823F025F80408BBF70408FB
:10F760001FF70408AFF7040895F7040839F70408F1
:10F770007FF7040879F7040803236370D9E70021B1
:10F780008148F8F7B3FC012840F05281A378013397
:10F79000A370DBE72378032B14BF4FF48076802619
:10F7A000207D002800F0C580012850D0FEE795F8A4
:10F7B000A037002BBDD07448ACE70023092203A971
:10F7C000D5F82C08F8F7E0F90128B2D10022039B04
:10F7D0002270B3F80B20B2F5007F1DD11A7C022AEB
:10F7E0001AD193F8FE21552A16D193F8FF21AA2A9F
:10F7F00012D1B3F80EC0D5F82C280CEB0207C5F8CF
:10F8000030785E7B721EC5F840687F2A04D8724249
:10F8100036EA020200F014810322012385F8E4276E
:10F82000637086E70023092203A91846F8F7ACF9AC
:10F8300001287FF47EAF039B93F8FE21552A00F048
:10F84000AD800222012385F8E427637071E7D5F8C3
:10F8500040284FF0FF3300215202B3FBF2F36268FD
:10F860009A18D5F8383803F1020341EB01009342AE
:10F87000814148494FF0020038BF1A46F8F7D6FADE
:10F8800003288DD801A353F820F000BF33F70408F4
:10F890009DF8040833F704089DF80408D4E901131F
:10F8A00027695A1ABA4288BFC4E9031203280BD049
:10F8B0000133B3FBF6F206FB12320AB133449B1A52
:10F8C0000022636022756BE723690622652BA27014
:10F8D0007FF63CAF2278653B032A15BF6FF0FF012E
:10F8E0006FF07F014FF4807280220B4001339A4207
:10F8F0002361BFF42BAFE268D5F8381898180231AD
:10F90000884207D395F8E41711B9012185F8E41767
:10F9100001216170D5F84018C5F8C42701FB03F335
:10F9200005215B02A170C4E901201B4A42E90233B0
:10F930000CE7D5F8382816490232F8F777FA032889
:10F940003FF62EAF01A353F820F000BF33F70408B1
:10F950005DF9040833F70408C9F804080122636854
:10F9600013442275A3601BE7CC480024D07A0024FE
:10F97000D06A0024B8820024A4810024E8810024F5
:10F980002C8200241D6304087082002434B10A080C
:10F99000D46A0024D86A00248082002493F8FF21CE
:10F9A000AA2A7FF44EAFD3F8C6215AB193F8C211F8
:10F9B0000639C9B2082905D840F2611020FA01F1D0
:10F9C000CF0730D4D3F8D6215AB193F8D2110639E3
:10F9D000C9B2082905D840F2611020FA01F1C80720
:10F9E00021D4D3F8E6215AB193F8E2110639C9B20D
:10F9F000082905D840F2611020FA01F1C90712D494
:10FA0000D3F8F621002A3FF41CAF93F8F231063BFD
:10FA1000DBB2082B3FF615AF40F2611121FA03F378
:10FA2000DB077FF50EAF0123C5F82C28A3708DE608
:10FA300002287FF47EAE012385F8E437637078E610
:10FA40007202013AC5F84828D88A00B9586AC5F840
:10FA50003408B3F81120520102F2FF125212C5F815
:10FA60005028B3F8131001B9196A94440CEB400CF8
:10FA7000A1EB0C01B1FBF6F1460040F6F470C5F8BD
:10FA80003818814213D94FF6F470814212D90321FC
:10FA90002170D96ABB180020C5F84C183344C5F84A
:10FAA0003C38F8F76DFFA3780133A37041E60123DA
:10FAB0002370B1E6022300212370EBE7294B30B518
:10FAC00083B09A790190AAB393F82420DFED266AD7
:10FAD00007EE902ADB79254AF8EEE77AA3F10203D4
:10FAE000234CB3FA83F3157886EEA77A5B0984F882
:10FAF000343184ED4C7ADDB11E4BDDED017AB3F883
:10FB00007E39F8EE677ADFED1C0A00EE103A67EEF8
:10FB1000A00AB8EE400A4BF0F7FF04F59C730021F1
:10FB200003EBC5021960083303ED010A9A42F9D1CB
:10FB300003B030BD114A12681001F9D593F82420A2
:10FB4000DFED096A07EE902ADB79094AF8EEE77AD9
:10FB5000991E4B4286EEA77A4B4182F8343182EDF2
:10FB60004C7AE5E7902F00245555554010060020AB
:10FB70004C16002024A30024BD378635D44E002423
:10FB800038B5094D2B7963B100242B6820465B6B97
:10FB900013B10134984708B9002038BD2B799C4235
:10FBA000F3D3012038BD00BF401600200C4B93F862
:10FBB000902012B90B4B987970470A4A906800B9A7
:10FBC0007047094940F6B83C0968091A614504DDE7
:10FBD0000021907983F8901070470020F0E700BF73
:10FBE000EC13002440160020EC2900242DE9F04FEE
:10FBF000DFF840921F46531E83B016460546D9F8DB
:10FC00000040142B00F2D280DFE803F05E5E5E5EFF
:10FC10005ED00B0B0B0BD00B0B0BD0D0D0D0D00B7E
:10FC20000B004FF47A734FF00A0A0193012F51D061
:10FC3000002F46D1794A7A4B14781878631C03F068
:10FC4000030383423DD0137004EB4403DFF8E081EB
:10FC50004FF47A724FEA440908EBC30383F80CA00F
:10FC60009A60C1B11822A5F1FF0002FB0482B0FA2C
:10FC700080F00C32400905E038B9013702F8013F45
:10FC80008F4208D0AF420346F6D1013733468F4248
:10FC900002F8013FF6D1FFF773FF002800F0AE80B5
:10FCA00009EB04035F4A0120DB00D2F8942008EB43
:10FCB000030108F8030042F20F731344B3FBF2F39D
:10FCC0004B6003B0BDE8F08F574B012F4FF0010A96
:10FCD0000193ADD1554A537C012B03D0022B00F088
:10FCE0009880002799F8040008B34D4B1821A5F11E
:10FCF000FF0E1A780C23BEFA8EFE11FB02314C4B1C
:10FD00004FEA5E1E1944002307E0BEF1000F08D140
:10FD1000013301F801CF984209D0DAB2F446AA4281
:10FD2000F3D10133B446984201F801CFF5D142F244
:10FD30002830F7F757FD4FF47A70F7F753FD97B374
:10FD4000236A03B1984799F80430EBB1A5F1FF0895
:10FD50004FF0000BB8FA88F858464FEA5818E26B93
:10FD600090475D45A26A314603D0B8F1000F00D13B
:10FD70004146584690470BF1010399F804205FFA79
:10FD800083FB93455846EAD3A36903B19847E36AD6
:10FD900098478FB90AF1FF3A1AF0FF0A18D04FF4CA
:10FDA0007A70F7F71FFDE3699847C9E74FF47A7354
:10FDB0004FF0010A019339E70AF1FF3AE3699847E6
:10FDC0001AF0FF0A04D04FF47A70F7F70BFDB7E78B
:10FDD0000198F7F707FD99F80420002A3FF471AF66
:10FDE0000F4C0D2118231248247813FB0413002113
:10FDF000184403B0BDE8F04F4BF04ABC09EB0403D4
:10FE0000DB0008EB030208F80300506003B0BDE814
:10FE1000F08F9778083F18BF012763E74029002437
:10FE200041290024EC130024A0860100902F002417
:10FE300044290024401600202DE9F041144C94F888
:10FE400080490CB9BDE8F08180460F4616461D4634
:10FE5000BBB1012BF6D10F4B98792F2EF2D8002889
:10FE6000F0D10D4B0D4A1B781278013303F00303D8
:10FE70009342E7D02B46324639464046BDE8F04132
:10FE8000B4E6FFF793FE80F00100C0B2E5E700BFE3
:10FE900024A30024401600204029002441290024E6
:10FEA0002DE9F04F074691B082480E46824DFBF790
:10FEB00055F9002381494024062285F888393046C7
:10FEC00001230978C5F884D985F88949FFF7B4FF7B
:10FED0000A20F7F725FD95F888390C2BDAB240F2A5
:10FEE000E4809DF80C60FE2E32D0FF2E15BF0F244B
:10FEF000152400250125944240F0D780611E6846F4
:10FF0000C9B239F07FFA04F140030DEB030414F891
:10FF1000413C834240F0C4806A1E9DF80D30684821
:10FF2000012A87BF03F01F075C099DF80E701E466B
:10FF30008CBF61379DF80F40FBF73CF8022D33D0A2
:10FF4000013C042C2ED8DFE804F00527292D2B00D6
:10FF50000225D0E75B486C464FF00008DFF8BC9103
:10FF6000FBF748F8DFF8B8A1DFF8B8B15648FBF75F
:10FF700021F808F1010814F8011B4846FBF76EF858
:10FF8000B8F10C0F16D00AFB08F3B3F1553FF0D8C7
:10FF90005846FBF70FF8ECE74C48DCE74C48DAE74B
:10FFA0004C48D8E74C48D6E700230DF11F008DF8E8
:10FFB0003F30D0E7FBF706F8022D3AD064223B46EB
:10FFC0004648B6FBF2F102FB1162C9B2D2B2FBF7AE
:10FFD000C5F885F001035B42DBB2012B59D8404ADA
:10FFE000404B9DF81010404800290CBF114619469F
:10FFF0003E4EFBF7B3F89DF811103D4B3D480029EC
:020000040805ED
:100000000CBF31461946FBF7A9F8022D41D19DF8E6
:1000100012403948FAF7CEFF8CB1FF2C1FD00A23CB
:100020003648B4FBF3F103FB1142D2B2FBF796F86A
:1000300008E03A4631463248FBF790F8CFE73046C1
:10004000FAF7D8FF9DF813402E48FAF7B3FF44B1F2
:10005000FF2C21D021462C48FBF780F804E02B48E8
:10006000EEE72248FAF7C6FF0DF1130500241F4EF4
:100070001F4FDFF8988015F8013F7BB1FF2B14BFAD
:100080003A464246214601342148FBF767F8042CE2
:10009000F1D111B0BDE8F08F1C48E3E73246F1E73B
:1000A0001C493846FBF786F8F3E71B48FAF7A2FF2E
:1000B000EFE700BF555D0A0824A300248814002040
:1000C000665D0A08715D0A08975D0A08785D0A088E
:1000D000805D0A08885D0A08B0590A08A95D0A0807
:1000E0003E5D0A08355D0A08E05D0A08455D0A08BC
:1000F0005F670A08F75D0A08FE5D0A08125E0A08D3
:10010000C55D0A081A5E0A08596F0A08495D0A089F
:100110002A5E0A08355E0A08455E0A081F550A0865
:10012000ABAAAAAA3F690A0810B5437B04468268B5
:10013000581C6073D154627B237B934200D802B970
:1001400010BD2368D4E9010198470023637310BDF3
:10015000427B42B1036810B50446D0E901019847DB
:100160000023637310BD7047036810B51C7882B01C
:10017000012C0DD0022C02D0002002B010BD1B6A51
:10018000002BF9D101F07F013BF032FD0120F4E7B3
:1001900093F9044096460DF107030A46017920467B
:1001A0008DF807E045F026FE0028E6D02046F5F75A
:1001B000CBFE02B010BD00BF036810B51C78012C47
:1001C0000CD0022C01D0002010BD1B6A002BFAD1EC
:1001D00001F07F013BF00CFD012010BD84469646E6
:1001E00093F904002C22094B02FB00335B7E002BA9
:1001F000E9D1074B0A469CF8041083F88AE903F614
:100200008A13BDE8104045F0F5BD00BF80280024EA
:1002100024A3002470B5066894B00446154696F8E9
:1002200000C0BCF1010F43D0BCF1020F02D000208E
:1002300014B070BD1A46336A002BF8D161F07F010B
:1002400005938DF81C300D93109312938DF80F10B9
:10025000CDE90A520DF10F0204920122CDE90833D3
:10026000069200238DF830208DF844200022CDE93D
:100270000E23EFF31185102383F3128803681B6AA2
:10028000002B30D004A8069B02461BB1D369143260
:10029000002BFBD1336AEBB1996839B99A4219D076
:1002A0001968A9B15B6899680029F7D01433F3E79E
:1002B00096F904600A46017930460095F5F780FE0C
:1002C0000028B5D0304614B0BDE87040F5F73CBE0C
:1002D000C3E90040EDB285F311882268136A002B50
:1002E000FCD10120A4E704ABEDB2336285F31188A1
:1002F000F1F70CFBF1E700BF70B5066894B0044657
:10030000154696F800C0BCF1010F42D0BCF1020FB7
:1003100002D0002014B070BD1A46336A002BF8D109
:1003200061F07F0105938DF81C300D9310931293AB
:100330008DF80F10CDE90A520DF10F02049201223F
:10034000CDE90833069200238DF830208DF8442043
:100350000022CDE90E23EFF31185102383F31288D9
:1003600003681B6A4BB304A8069B02461BB1D36902
:100370001432002BFBD1336AB3B1996839B99A4270
:1003800012D0196871B15B6899680029F7D01433ED
:10039000F3E70A46217996F904000095F5F710FE77
:1003A00014B070BDC3E90040EDB285F31188226836
:1003B000136A002BFCD10120ACE704ABEDB2336231
:1003C00085F31188F1F7A2FAF1E700BF036810B5D1
:1003D0009B68044698470122FF236273A37310BDF4
:1003E000036810B504461B6898470121236820461E
:1003F0009B689847E37B0133E37310BD2DE9F0411F
:10040000069F0D46044616463846984648F05EFA62
:100410002844E672A072387850B1069729462568BC
:10042000204643463246AC69A446BDE8F0416047E9
:10043000BDE8F08103689B6A184700BF03685B6DE5
:1004400003B11847704700BF0368DB6C03B118475E
:10045000704700BF0B46002110B5C17304464274BB
:100460009A6C0360017302B1904723680121204612
:100470009B689847FF2123680122A173DB6C62739C
:100480001BB12046BDE81040184710BD01380F28A9
:100490000DD8084B4FF02C0C0CFB003393F92000C7
:1004A00028B9012083F8201083F82120704700200C
:1004B000704700BFB0030024064A002301E0102B60
:1004C00006D0516801332C328142F8D1184670476A
:1004D0000023FBE7B00300240D4B012210B482403F
:1004E0000C4C1B7854F82000134051B1003B18BF4E
:1004F000012318B1026881883BB191615DF8044B1A
:100500007047B3FA83F35B09F3E79162F6E700BF44
:10051000804300248443002410B50A4C23681B6BDD
:100520009847094B094A40F2DC5099780023032987
:1005300098BF1046A360A4F80530BDE81040F7F757
:1005400051B900BF40160020902F0024FCA60700E0
:1005500008B504460848FAF72DFDFAF70FFD074BDA
:10056000186807F027FCFFF7D7FF012C01D145F0F1
:1005700057FBF3F77DFE00BF4E5E0A08FC590024CE
:1005800038B50546FAF7FAFC094B0024186807F05D
:1005900011FCFAF7E3FC074B83F88B4983F88C498D
:1005A00018F05AFD15B12046FFF7D2FF38BD00BF45
:1005B000FC59002424A3002410B508460749F5F788
:1005C00013FF002815BF0124002405480548FAF749
:1005D00017FD2046BDE81040D2E700BF5A5E0A086A
:1005E000635E0A088A5E0A0838B505460C460AF0BA
:1005F0006FFF58B32046FBF7E7F868B92046F8F7D5
:10060000F5FE00F54370B0F5C36F05D928461249D1
:10061000BDE83840FAF7CEBD1048FAF7F1FC1048B3
:10062000FAF7C8FCFAF7AAFC0E4B186807F0C2FBF1
:10063000FFF772FF0C4BCA225A6253225A620322FE
:10064000DA65FF225A6272B6F3F712FE0748BDE878
:100650003840FAF7D5BC00BFA65E0A08BE5E0A089D
:100660004E5E0A08FC59002400400058DE5E0A086D
:1006700010B5044C23681B6998470023A371A3603D
:1006800010BD00BF4016002010B5074C63791BB1A8
:100690002368DB68984700B910BD044B01221B6832
:1006A000A271A36010BD00BF40160020EC290024F9
:1006B0002DE9F74F054608460E46FBF785F8044638
:1006C00018B9334B93F880792FB9284603B0BDE8A9
:1006D000F04FFBF764B83046DFF8C8902646DFF8E5
:1006E000C8A001AA2B494AF0B6FF10B9FFF7CCFF0A
:1006F00008E056B9012201462846FDF753FB421C8B
:1007000004461AD103B0BDE8F08FF8F76FFE2F282A
:10071000834636D80FB1FFF7ABFFBBF1060F13D0FE
:100720001D4901235FFA8BF20978E0B2FFF784FBE1
:10073000002759464846FAF711FD01AA154900203D
:1007400001364AF088FFD0E7DAF800301B0114D5F3
:10075000FF2C0ED0E1B22846FFF7A2FBE8E70137F5
:100760002846FFF79DFBF9B298F800208A42F6D898
:10077000DEE70027DFF82080F5E70848FAF73AFCC3
:10078000D6E72F2206492846FAF714FDD5E700BF21
:1007900024A30024B6520A088814002046560A08EA
:1007A0001C5F0A080B5F0A08D44E00240D4A0E4B4A
:1007B000B2F84C295B8C07EE902A9FED0C6A07EE8D
:1007C000103ADFED0B6AF8EEE77A9FED0A0AB8EE11
:1007D000C77A67EE877A67EE867AA7EEA60A27EED3
:1007E000800A704724A30024902F00240AD7233CBA
:1007F0003F89B6B6FCA9713F044B1A79824203D9EE
:100800001B689B6B03B118470020704740160020FF
:100810002DE9F041104D00244FF0520853272E1DB2
:10082000013415F8010BF0F713FF2021E4B220B1D9
:1008300080F80680C471F1F7DDFE16F8010BF0F7C1
:1008400007FF402118B18771C471F1F7D3FE042C62
:10085000E6D1BDE8F08100BFB4AC002438B50C4649
:1008600014F8011B41B105462B6828461B689847C0
:1008700014F8011B0029F7D138BD00BF03681B68BD
:10088000184700BF03682DE9F0415F6A1FB13B467E
:10089000BDE8F041184704460D46164600E02368BF
:1008A0009B68204698478642F9D8002E08DD2E44E2
:1008B0002368204615F8011B1B689847B542F7D1FD
:1008C000BDE8F08103685B68184700BF03689B6858
:1008D000184700BF0368DB68184700BF03685B69FF
:1008E000184700BF03689B6A03B11847704700BFF1
:1008F0000368DB6A03B11847704700BF03682DE93E
:10090000F04116469A6A04460D460AB1904723689C
:100910005F6A5FB1324629462046B8472368DB6AE2
:10092000C3B12046BDE8F041184723689B682046C4
:100930009847B042F9D3002EF0DD2E4423682046BC
:1009400015F8011B1B689847B542F7D12368DB6A8D
:10095000002BE6D1BDE8F08170B504460E46154681
:10096000236820469B689847A842F9D32A46314617
:100970002046BDE87040C1E7164B1B888BB9164A6C
:10098000164B12781B682AB143B11A689B8830B1A4
:100990009361704780F00100002BF6D1704793629D
:1009A00070470F4B5A69002AF8D00E4A1288002A65
:1009B000F4D010B41C6848B10B490120B1FBF2F22D
:1009C0000241226058745DF8044B704720605874EF
:1009D000F9E700BF90430024984300249443002487
:1009E0009C430024B443002440420F0000231849D4
:1009F00001E0152B26D003EB4302013311F802C0AE
:100A00000A448445F5D130B45478ECB1B0FA80F39F
:100A10005B09C8B10F4D4FF0010C2A4602E00133CB
:100A20004E2B11D011791C328142F8D10CF1010109
:100A3000A4455FFA81FCF2D1C3EBC30305EB83004D
:100A400030BC704700207047002030BC704700BFAA
:100A5000202D0024B0C009082DE9F04F3D4D83B092
:100A60004FF0000A0646DFF8F090DFF8FC800191B5
:100A70002878697818B3B1FA81F46409F9B1364B72
:100A80004FF0010C02E001344E2C18D01A791C33BF
:100A90008242F8D10CF1010261455FFA82FCF2D189
:100AA000C4EBC4034FEAC40B59F8230009EB8307D6
:100AB000F3F7FEFC072834D90022964237D00AF11A
:100AC000010A0335BAF1150FD2D1244BD3F80090A7
:100AD000B9F1000F39DD224C0025DFF88C8004E0ED
:100AE000013504F58874A9452FD0A768002FF7D0E9
:100AF0003868F3F7DDFC07284FF000029EBF18F8B6
:100B00000020013252B29642EAD17A79019B9A4290
:100B1000E6D194F90C21002AE2D0384603B0BDE8B2
:100B2000F08F18F80020013252B29642C7D1ABEBD9
:100B30000402019B09EB820252799A42BFD1094B10
:100B400013F91A20002ABAD0E7E70027384603B085
:100B5000BDE8F08F202D0024B0C00908040000205B
:100B600008000020BCAC0024C8BF0908F0B5DFF8BD
:100B7000A4E00025224F06469EF800009EF80140A2
:100B8000D0B1B4FA84F35B09B4B11D4A4FF0010C43
:100B900002E001334E2B0FD011791C328142F8D183
:100BA0000CF1010164455FFA81FCF2D1C3EBC30390
:100BB00007EB83039E421DD001350EF1030E152D68
:100BC000DAD1104B1C68002C18DD0F4800230246B8
:100BD00002E001339C4211D0916802F5887200292D
:100BE000F7D08E42F5D103EB031300EB031000F5B1
:100BF0008670F0BD054800EB4500F0BD0448F0BD2F
:100C0000B0C009080400002008000020BCAC00248B
:100C10000C080A08202D0024F8B5B8B316460F4674
:100C200000231D4A01E0152B30D003EB430C5D007F
:100C3000013312F80C1094448142F4D19CF8014025
:100C4000B4B1DFF85CE001210023F44602E0013397
:100C50004E2B1ED09CF804200CF11C0C8242F6D1C5
:100C60004A1C8C42D1B2F2D1C3EBC3030EEB830416
:100C70002046FFF77BFF90F900303BB9074B204639
:100C80002B4483F8987983F89969F8BD00242046AD
:100C9000F8BD0024ECE700BF202D002424A300248D
:100CA000B0C00908644B2DE9F04F1B68C6B2DFF8ED
:100CB000CCA1DA04614CBAF82080614F48BFB4F887
:100CC000C88994F8D2392DED048B9AF8025097B068
:100CD0003E71042D039308BF4FF000081BB394F836
:100CE000801951BBC02257484AF0D2FC9AF8042020
:100CF000554B003A55491E7018BF0122544B3960BC
:100D00001A70039B042D00F24183DFE815F076038F
:100D10003F03910267036C03089B002B40F04C8358
:100D20000023039A1370464900234A4A0B710A6054
:100D300017B0BDEC048BBDE8F08F9AF806209AF846
:100D40001130101E18BF0120012B00F0D881B5F121
:100D5000080118BF0121022B18BF0021002940F013
:100D6000CE813D4B072D36490B603C4B1E700393E3
:100D70003B4B0493187000F22A83042D0ED9394B93
:100D8000394919609AF80530012B05D0022B08BFAC
:100D9000002A0CBF01230023344A1370294B4FF063
:100DA0000009DFF8DCB00793314BCDF814900A93BB
:100DB000304B0693039B059A1B78934240F3DF82E6
:100DC000069A032112F8013F06920AEB030201334F
:100DD000147ADFB220463A46FFF71EFF0546002888
:100DE0009ED02046F0F734FC079B586118B14FF0B5
:100DF0000303C77183719AF802209AF8033095F8BB
:100E0000069009920BB189F001092846F1F772FBAF
:100E1000164B1B78089300283FF47EAF002B40F060
:100E2000CB82D0E901630D93002E3FF479AF124BD2
:100E300000241A4629E000BFD44E002424A3002435
:100E400040160020500500204C05002010080A081C
:100E500031070024DC080A0890080A081006002060
:100E600048050020F40E002001000000E40E0020E0
:100E7000802B0124A22F0024B0030024902F0024F3
:100E800014060020102C3FF44BAF5168A0462C32C2
:100E900001348E42F6D12C22089802FB083292F9D6
:100EA0002010002800F004832868CDE90B1247F0D9
:100EB00075FB0B990C9A39299F4B40F01F8392F8D0
:100EC0002120824213D0286847F068FB9A4BC0B2B9
:100ED0002C2202FB083393F92020002A7FF420AF54
:100EE000392283F8210083F82020002308932F68FB
:100EF000CBF874603846F4F789FF059B8F4A8BF86E
:100F000011308F4BCBF808501B780B90013B0C93A2
:100F100003B203EB430302EBC303CBF87830287929
:100F2000F0F796FB09F00101049B01311B784901A0
:100F300089EA030941F00601CBF8141010B1EA79EF
:100F4000F1F774FCDDE90B32934200F0FF82099B5C
:100F5000063B0F934FF0000860223846CBF85E80C6
:100F6000CBF86280CBF8668069793FF0B9FC754BAD
:100F70009BF81110602223F8112019F002030E9340
:100F800000F088824FEAC903ABF8688003F00803D9
:100F9000ABF864300423ABF8603000226A4B38466B
:100FA00023F8112069793FF0F1FC684B0BF16A02DC
:100FB0003846CBF86A304FF40033CBF86E3069799D
:100FC0003FF054FD624B1B78002B00F07E82DBF873
:100FD000783001229E60002130468BF81820F1F70E
:100FE000A1F83046F1F766F8089B002B00F0698203
:100FF000574B1B78002B40F006820D9A8BF8183067
:10100000CBF81C200A9ACBF82030CBF87C20CBF808
:1010100028204022CBF83030CBF838200122296834
:10102000CBF82420CBF82C203431CBF83420CBE97A
:101030000F336879CBF82C30122301EB8001CBF809
:101040003420CBF83C304FF48053CBE90812CBF876
:1010500030304FF40033DBF87820CBF840309DF887
:101060003C30CBF87460022B00F2118209990829F8
:10107000384901EB8303D3F8AC18374BB3FBF1F3DA
:1010800018BF132103F1230308BF5F21CBF85830A9
:10109000584691804AF044FD2D4B1B78002B00F000
:1010A000EB81089B002B00F0E7813B68384643F05A
:1010B00001033B600E9B6979002B00F0E58144F051
:1010C00019FEDDE90B32934200F09B82049B1B78F2
:1010D000002B40F00A820A9B0BF1800B059A5833D3
:1010E000079901320A930123082A05920BF8713CF3
:1010F0004B7401F1180307937FF45CAE3FE1174B8B
:101100000027174A1D703946164B3D46DFF86C80A4
:1011100013604FF46072144BC346A0461E700393D5
:10112000124B134E1F700327124B18701248049372
:101130004AF0AEFA31E000BFB0030024240E0020D4
:10114000200E0020702F0024802F00240A000100B0
:10115000E40E002024000A0800D01213B62F002449
:101160004016002050080A0810060020B72F00245F
:10117000A22F002448050020405E012448040020DE
:10118000282930386F12833A00007A44F0F738FB90
:10119000082D0BF1200B00F0F280039B1B78AB4273
:1011A00040F3ED8016F8013F534493F80890484609
:1011B000FFF71CFC04464846F0F74AFA9AF8031079
:1011C000A379044609B183F0010303F00101049AF5
:1011D0000131107888F8D31983EA0009002C00F057
:1011E000218294F9060030B1A0F1410358425841E0
:1011F000002800F0DB80A08849010135CBF80C40C5
:10120000B0FA80F041F005018BF81090C0F11F009A
:10121000CBF81410CBF804002046A771E571F1F764
:10122000E9F919F0010F2046B0D1F0F7F7F9AFE76F
:101230001FED2D8AF0EE488A38EE887A5FED2F7A1E
:10124000F5EE006A1FED309A28EE278ADFF8F4B237
:101250000027AB4CC6EE879A0393AA4B1B78BB4280
:1012600040F38D801BF8019F03210AEB090309F16C
:1012700001091D7A5FFA89F928464A46FFF7CCFC36
:101280000646002800F0BC802846F0F7E1F96061CE
:1012900038B1032280F8079002218271F279F1F7C8
:1012A000C5FA994B1878002877D0BAF8003007EEC5
:1012B000903AF8EEE77AFCEEE77A17EE90CA3368D8
:1012C0009249934A8B42126865D001F580618B4246
:1012D00061D0DFF874E201F580418B4218BF73459D
:1012E00059D001F580618B4255D092084FF6FF73BB
:1012F000B2FBFCF11944090CB2FBF1F208B1B2FBEC
:10130000FCF39AF8021007EE902ACDF80080042929
:10131000F8EEE76A9AF80300314608BF07EE903A04
:101320009BB211BF26EE887AB8EEE77ADFED797AC4
:1013300027EE277A69EE477A84ED027AE6EEA87AFC
:10134000C4ED037A01902046F3F7CEFC002F37D08E
:1013500061686B4B01E0A34226D05A6818338A4279
:10136000F9D1039B83F001030137183404F8083CDA
:10137000082F4FF0010304F8073C7FF46EAF664975
:10138000002201238A60A1F80530D1E49FED638A31
:10139000F0EE488A50E75208A8E7FAFE697AFCEEB8
:1013A000E77A17EE90CA8AE70023DBE70399012367
:1013B0005B4A08701370B6E4D5E904630D9333E516
:1013C0000127183404F8087C04F8077C45E7082D49
:1013D0007FF4E4AC534B544A1A60DFE49FED538A28
:1013E000DFED538A28E79FED538A01224649F0EE4C
:1013F000488A4FF000080A701EE79FED468AF4E71E
:10140000404B18708FE4099B4FF490720B994FF08A
:10141000000C082B484B286802FB01334FF00101F8
:10142000DBF8782000F1E40E8BF818101361CBF88C
:101430002C304FF040030D98CBF8483014BF1223E6
:101440000623CBF81C00CBF820E0CBF84C304FF44F
:101450008053CBF834C0CBF824304FF48043CBF822
:101460002810CBF830304FF40033CBF84410CBF8D1
:101470005030CBE90ECCF2E520469BF8113090229B
:101480002E49F0F7ABFC10E644F05EFC19E68D2324
:101490001321FBE54FEA490303F00203ABF8623086
:1014A0000123ABF85E304FF48073ABF8663074E51F
:1014B00000297FF435AC032382F8217082F82030B4
:1014C00013E52046F0F768FC92E56A79DBF87800CE
:1014D000032A818A9CBF1A4B33F812300022ABF8E2
:1014E0000C3021EA0303838275E52B686A79343373
:1014F00003EB82034FF6FF721A60ECE5C0B2E7E43B
:10150000500500204C050020310700240000014058
:10151000AC0300246F12833A401600206F12033987
:10152000B72F0024F40E002035000000ACC5A7370B
:10153000ACC5A73600000000802201241D04000075
:1015400040BF0908A22F0024004001400023D5F825
:1015500000803C49CDF84230ADF85030159351F839
:10156000332001EBC3000133904559D00E2BF6D147
:10157000002044F0ADFE3B6823F001033B60099B73
:10158000082B4FF000030CBF5F221322CDE912237A
:101590002D4A2E4B90451B6840D002F58062904545
:1015A0003CD02B4902F58042904518BF884535D084
:1015B00002F58062904531D09B0807EE903A099B76
:1015C000DFED246A063BF8EEE77ADAB20F93022ADF
:1015D00097BF214B214B03EB8203D3F8AC3807EEC6
:1015E000103AB8EE477A87EE870A30EE260A49F0BD
:1015F0003BF8431E10A93846ADF840303EF0F2FFEC
:10160000A8E43B6843F080033B607B6C43F40043F9
:101610007B643B6843F001033B6057E55B08CCE724
:101620008088A6E749010135CBF80C4041F005015F
:101630008BF81090CBF814104FF0FF31CBF804105A
:10164000EFE500BFD0BE090800000140AC03002454
:10165000004001400AD7233C24000A08C0C62D00E0
:101660000D4B30B593F80F2A002A14BF0122002237
:101670001A730FD003F6D41503F10D0403F6F41317
:101680002A46083403CA9A4244F8080C44F8041C59
:101690001546F5D130BD00BF24A3002470B5174E08
:1016A000044633786BB1164D2B7853B11549F9F7D1
:1016B00081FD20461449F9F77DFD00203070287027
:1016C00070BD124B93F82D20AAB11A7B9AB903F181
:1016D0000D0203F6D41503F12D061068083252F8F6
:1016E000041C2C46B24203C42546F6D1012283F8DD
:1016F0000F2AFFF7B5FF0120E2E700BFD84800241A
:10170000D94800243C5F0A08735F0A0824A3002418
:1017100010B50C46FFF7C2FF78B1084B01229A734F
:10172000F9F770FA0648F9F76BFC06492046F4F71A
:101730005BFE10B10020FEF70BFF10BD984D00249A
:10174000915F0A085A5E0A082DE9F74F4FF0000B27
:10175000064601AA08462D495D4649F07CFF01274F
:101760000446DFF8BC80DFF8BC90DFF8A0A014BB13
:10177000BBF1000F27D1002D44D029462448F9F7AA
:10178000EDFC244B1B780BB9FCF79CF83DF096FB65
:10179000214B00221A70FCF72FFB15B12846F9F7F0
:1017A0005BFE9FB13046FFF779FF78B1F9F72AFA6F
:1017B0000020FEF7CDFEBBF1000F0AD02046F7F760
:1017C00015FE85B2C5B93046F9F7E9FF03B0BDE8AB
:1017D000F08F41462046F7F767FD80B9494620461D
:1017E000F7F762FD0028EED05F4601AA51460020BF
:1017F00049F031FF0446BAE74FF0000BF5E74FF030
:10180000010BF2E70548F9F7FBFBBFE7B6520A0800
:10181000A15F0A08D4590024D9480024C45F0A08EB
:10182000985F0A08ED660A0808B501210020FEF756
:1018300053FE01212B4C0846FEF74EFE01210220EB
:10184000FEF74AFE237803F00502052A2AD003F0AA
